:08000000FC7F002005AA0000AE
:100400000000000000000000FFFFFFFFBE03FFFF31
:1004100061202A2106F09EBE6120292106F09ABEA5
:100420007FB5422306A88DF81030002340F8143D14
:100430000AF046F8012804D1612014210C2207F0AB
:10044000E5F807B05DF804FB08B5144B20281880C8
:100450000BD002D8E0B1082805E0802818D0B0F50C
:10046000807F0AD0402818D112E0612041F27071DB
:100470000622BDE8084007F0C9B8062261204FF403
:10048000966107F0C3F8064B1A78064B1A7008BD40
:100490006120BDE8084007F0F1B808BD0083FF1FE8
:1004A000948BFF1F0D82FF1F084B10B51868084C76
:1004B00040222146183006F0DFFC064B2146186822
:1004C000402206F0D9FC002010BD00BF2882FF1F8B
:1004D000C0B400002482FF1F054B064A1978117032
:1004E00010B9054A127800E0FF221A70704700BF69
:1004F0000D82FF1FF081FF1F948BFF1F024B1A78A4
:10050000024B1A70704700BFF081FF1F0D82FF1F62
:1005100030B51F4B1F4D1B6885B093F824208DF814
:100520000B208022ADF804204FF4C062ADF8062005
:1005300061228DF80C2093F84E208DF80E2093F850
:100540004F20DB698DF80F200024014600932046E0
:1005500001236A468DF808408DF80D3006F066FBE1
:10056000287088B12246052106F0A2FA009B5A069F
:100570000AD540F204412246287806F099FA2878F4
:100580008121224606F094FA287805B030BD00BFDC
:100590002882FF1F948BFF1F2DE9F0416B4C867B57
:1005A0002568A0B0002D56D1402006F045FE684BCE
:1005B0001860582006F040FE664B18602846FFF78A
:1005C00073FFB0F5004F07D161204FF4166103228D
:1005D00007F01CF8042300E001235F48236008F0C3
:1005E0008BFA01F0CDF86D20042106F0DDFF032029
:1005F000FFF78EFF002800F0A680584B58481A7865
:10060000584B1A7006F08CFD7520042106F0CCFFC3
:1006100004214D2006F0C8FF534B009309238DF8A9
:10062000043006238DF8053002238DF8073040236F
:100630000293684612238DF806300AF0C7FA4B4B36
:10064000009303238DF807306846102302930AF0C5
:10065000BDFAFFF7E5FE414FDFF8F080304669460E
:10066000052206F03DFA00283FD09DF803509DF882
:10067000042015B1012D15D032E0032A02D10AF071
:1006800083F9EBE70C2A02D1FFF7CAFEE6E7062A58
:1006900005D138783649162206F020FDDEE7832A98
:1006A000DCD1ECE7DD2A05D12368082BD6D1C8F8C8
:1006B0000050D3E7283AD2B2042ACFD82D4806F00A
:1006C0002FFD9DF80430292B06D02A2BC6D12846B1
:1006D0000AF0F0F8284800E0284806F021FDBDE7C0
:1006E0003046694606F0FCF9B8E7236813F0370F87
:1006F00029D01A4D287806F003FA20B3204F2E4651
:1007000028786946402206F0EBF90446D8B16846DD
:10071000214600F0D9FD3A88684621467AB901F0B1
:100720009DFF0028ECD04FF4807000F0D9FE022825
:10073000E6D130781349172206F0D0FCE0E700221A
:1007400001F08CFFDCE720B0BDE8F0812C82FF1FB8
:100750002482FF1F2882FF1F70B40000948BFF1FAC
:1007600000B500000D82FF1F1904000011040000F5
:100770003CB400001DB500003BB5000026B50000EC
:100780000083FF1F58B400007047013911F8013F82
:1007900033B110F9012B5BB29A42F7D000207047B9
:1007A00090F90020202A07DC03461846013390F90F
:1007B0000020202AF9D070471846704710B503680A
:1007C00093F90020202A07D01A461346013293F9E4
:1007D000001031F02004F8D11A46013392F90010CC
:1007E0002029F9D0026092F90000D0F1010038BF51
:1007F000002010BD08B5054806F092FC044806F03C
:100800008FFC0448BDE8084006F08ABCC4BE000066
:100810002CCF0000D7BE00002DE9F047DFF8D090C4
:100820002D4E99F800204FF00C0808FB02F2B31887
:1008300088B08246B5581F795C7901A820211B2217
:1008400006F012FBBAF1000F04D054450FDD0C3551
:10085000013CFAE7214806F063FC99F8003008FBF8
:100860000366B06806F05CFC1D4806F059FC1D4E9E
:100870000C3554B330780021422206F02FFC50B9D9
:10088000184B4021187841F26D0206F011F9164B11
:1008900001201C601CE055F80C0C06F041FCB8422D
:1008A0000246307802DB01A9012202E0BA1A01A94E
:1008B00092B206F013FC55F8080C06F031FC0B4818
:1008C00006F02EFC013C0C35D3E7074B20461C609C
:1008D00008B0BDE8F08700BFE0BC0000D6BE000055
:1008E000DABE00000D82FF1FFC82FF1FD7BE000092
:1008F0007983FF1F08B5094B1B78082B08D1084BDB
:100900001B681BB1186808B106F00AFC054800E036
:100910000548BDE8084006F003BC00BF7983FF1F0F
:100920003082FF1F8ECB0000CAC30000B0F5000F5D
:1009300008B505D34008002106F0F8FB054804E09F
:100940004002002106F0F2FB0348BDE8084006F033
:10095000E7BB00BFF2BE0000FABE00002DE9F04F79
:10096000ADF5037D09280546019100F04482112868
:1009700000F04182082800F0CF81152800F0F881AE
:10098000A0F11D03DBB2012B40F2C4830B2800F061
:100990001D839F4E306820B94FF4807105F0CEF969
:1009A000306031680C8F04F00204A4B24CB92046C8
:1009B00005F0E6F908B1974875E2954B1A68964B31
:1009C0001A60202D00F2A683DFE815F02600F7025A
:1009D00057024E0208010801A4038402A601150271
:1009E0001502A4036302A403A403A403A403150231
:1009F0001502A403A403D201C6022600A403F50035
:100A0000A4032100F500A403A403A40326000023EB
:100A1000DDF80490019301E04FF000097F4F3C683E
:100A20003CB901987C4905F04DFB002801DA7C486F
:100A300039E27C4C0123A3810DF108089023172D86
:100A4000C4F80080238101D1022302E01B2D02D1D2
:100A50000623237504E0202D01D00023F9E7257536
:100A60003B68C3B9704806F05BFB3368186806F052
:100A700057FB3368DB8E032B02D96C4806F050FB22
:100A8000019820B190F900300BB106F049FB68489D
:100A900006F046FB02E0614B00221A60654EB34649
:100AA00030780021932206F019FB78B9614B402180
:100AB000187841F26D0205F0FBFF172D01D10423D8
:100AC000FCE0202D0CBF05230123F7E052485549D7
:100AD00004F0A6FF63898246002B38D0172D03D17E
:100AE000554806F01DFB2CE01B2D2AD10022023BAD
:100AF00019F9021031F0200EC2EB030001D00132CF
:100B0000F6E7F2B14044494606F039FBC8B9B4F8FB
:100B10000A904148A9F10209C14404F0F5FD10B161
:100B20004846464901E04649484606F04DFB0D233C
:100B300003700A2343700230C8EB000060814FF05D
:100B400000099BF800006289414606F0C7FA1AF1D5
:100B50000F0FA5D10021608A06F0E8FA394806F0A7
:100B6000DFFA0021606806F0E1FA374806F0D8FAAB
:100B70000021208A06F0DAFA344806F0D1FA002182
:100B80001822284806F070F9002005F06BFF038B4F
:100B9000590709D5036B5A1C06D090F82B0058430F
:100BA000FFF7C4FE2A48CAE003236D2100203B6002
:100BB00005F0E6FE83E04CF2010344F201041C2D33
:100BC00018BF23460198326802A905F02FFD0028BE
:100BD00002DA204806F0A4FA02A89AE00F4F1E4954
:100BE0003A686D2381F83F3040F61203042D18BF98
:100BF0001123022A884602D1042D4CD12EE00198FF
:100C0000326805F013FD022840F0B781F4E700BF19
:100C10003082FF1F01BF00004C83FF1F0483FF1FB2
:100C200011BF00004082FF1F25BF000020D200003E
:100C300030BF00000D82FF1F34BF000038BF00002E
:100C400054BF000061BF00006EBF000077BF00000E
:100C500086BF00008EBF00000883FF1FA44C4FF426
:100C60008072217802A806F0FFF823780133237000
:100C7000A04C02A920464FF4807205F0A9FA05465F
:100C800008B19D482CE09D4806F04AFAA068294624
:100C900006F04CFA39E09A4DDFF858922E46287843
:100CA00000214FF4807206F019FA50B9944B40219C
:100CB000187841F26D0205F0FBFE02233B6001242F
:100CC00029E202AC00238B483B6021464FF480723E
:100CD00005F096F918B9B9F83C202E2303E08948AD
:100CE00006F01EFA11E0904207DA215C0A39C9B217
:100CF000702988BF23540130F5E73078214606F08B
:100D0000EDF9B8F83C30FF2BC9D87F4806F008FA57
:100D1000784805F039FAFDE1019806F064F80446D8
:100D20007A4806F0FDF92046842106F009FA2246A9
:100D3000002002A905F054FE044618B1744806F0DC
:100D4000EFF9E7E1704806F0EBF9254602AF00261F
:100D50002F44B8599421043606F0F2F9402EF8D108
:100D60006948403506F0DCF9B5F5007FEED1D2E1F7
:100D7000019806F038F8044601A8FFF71FFD20B9D6
:100D8000019806F030F8C0B200E00020002302AD68
:100D9000C218B3F5007FD2B202D0EA540133F7E7AC
:100DA0005C4806F0BDF92046842106F0C9F95A4B8B
:100DB00040221A6001A8FFF701FD08B1012005E0FB
:100DC000019806F010F8C0B20028F7D00319DEB27F
:100DD00000202946224605F01DFE08B14F4800E0DC
:100DE0004F48013406F09CF9E3B29E42F0D14A4BE1
:100DF00040221A608EE14B4806F092F9019B93F96C
:100E000000202D2A16D193F90120312A12D193F90D
:100E10000230322B06D0362B0CD1434806F080F935
:100E2000042203E0414806F07BF90222019B0433CF
:100E3000019303E03E4806F073F900220A2D01D029
:100E4000122D01D142F00102113DEDB2012D98BFEA
:100E500042F008020020019905F0F6FC044608B1B2
:100E600034486CE734481EE00198316805F0A8FC6E
:100E7000002800F04F81314861E70198326802A9EB
:100E800040F2026305F0D2FB022800F043812C48B7
:100E900055E7019A154612F8014B63B2202B05D095
:100EA000002CF7D1274806F03BF934E100222A70E4
:100EB0000198326802A905F0B9FB002801DA22483E
:100EC0003DE7681C02A905F011F9002800F0228115
:100ED0001E4834E70198316805F014FC431C01D129
:100EE0001B482CE7002800F015811A4827E700BFAF
:100EF000F881FF1F0883FF1FA9BF0000B6BF0000D5
:100F00000D82FF1FC9BF000009C00000F0BF000034
:100F100000C000000CC000008CF00F401FC000009B
:100F200036C000003EC0000051C000004DC00000AF
:100F300055C0000059C0000068C0000087C0000014
:100F400099C00000AEC00000C1C00000CDC00000CC
:100F5000DDC00000EDC00000019805F061FF07460C
:100F6000019810F9012B202A0190F9D102A93268C9
:100F7000022305F05BFB022801D06948DFE6002070
:100F800005F070FD3946046B0546002202A805F005
:100F90001BFA02A805F0A8FC68B9624806F0C0F880
:100FA000286B001B05D0102106F0C0F85E4806F043
:100FB000B7F85E48C3E65E48C1E60198316805F0BF
:100FC000BDF9002800F0A6805A48B8E6002005F0D8
:100FD00049FD0446584806F0A3F8238B03F48072B9
:100FE00092B20AB15548AAE69F0601D454480DE0D2
:100FF000134602A8E11891F8491019540133202929
:1010000018BF1A460B2BF5D10023835406F088F83D
:101010004C4806F085F82069FFF788FC4A4806F03E
:101020007FF8238B5E0602D5484806F079F84848D9
:1010300006F076F8238B9D060FD513F4C04F09D028
:10104000580402D5434806F06BF8238B990404D565
:10105000414800E0414806F063F8238BDA0602D5E8
:101060003F4806F05DF8314806F05AF8238B9B069E
:1010700050D53C4806F054F81821208D06F056F85B
:10108000394806F04DF894F82B30208D182158433C
:1010900006F04CF8354806F043F89C21606806F0ED
:1010A0004FF8334806F03CF89C21206A06F048F8D7
:1010B000304806F035F89C21E06906F041F82E48EA
:1010C00006F02EF8182194F82A0006F02FF82B4885
:1010D00006F026F89C21A06806F032F8284806F0B1
:1010E0001FF89C21606A06F02BF8264806F018F8D5
:1010F0009C21E06A06F024F8234806F011F89C21B0
:10110000206B06F01DF8214806F00AF8606B9C2160
:1011100006F016F8002420460DF5037DBDE8F08F9B
:10112000DFBF0000FDC0000019C1000009C00000C1
:1011300029C100003DC100004CC1000057C10000A2
:1011400066C10000CDCF00005ACC000074C1000081
:1011500048C000007AC100007DC1000080C10000CD
:1011600083C1000094C10000A6C10000B4C100000A
:10117000C4C10000CFC10000D9C10000E9C1000016
:10118000EEC10000FEC1000009C2000018C200004C
:1011900030B587B00446082301A88DF8103009F057
:1011A0008FF9A01D05F03CFE0025ADF80800657123
:1011B000E01C05F035FEA5708DF80A00204605F00C
:1011C0002FFE01238DF80B0001A88DF8103009F0D7
:1011D00077F9024805F0A4FF07B030BD23C2000034
:1011E00070B5344D847B8AB00DF10906204602A902
:1011F000052205F075FC00285AD09DF80B309DF8AB
:101200000C20012B02D0412B37D04CE0DD2A1BD122
:101210002B6893B1012B02D1002001460BE0042B77
:1012200001D1172006E0052B01D1202002E0022B7E
:1012300003D105200021FFF791FB1F4B1868002800
:10124000D4D0FFF7E9FAD1E7BF2ACFD12B68032B1F
:10125000CCD1002005F006FC036B5A1C09D090F895
:101260002B005843FFF762FB144805F059FFFFF7C6
:1012700041FB104B00221A60B8E7204602A905F096
:101280002FFC9DF80830042B07D10DF107003146E3
:10129000012205F0F1FD0A4802E0032BA6D109481E
:1012A00005F03EFFA2E7204602A905F019FC9DE7E4
:1012B0000AB070BD0483FF1FFC82FF1F86BF0000C1
:1012C00032C2000043C200000A46034903460878C0
:1012D000194605F003BF00BF948BFF1F184B194A36
:1012E0001B681268D8695168884210B50BD1B3F8F1
:1012F0004E00D18E884206D193F82440117B641AA7
:1013000018BF012400E0012452895B8C53409BB23A
:1013100013F0280F18BF44F002045A0748BF44F0E6
:101320000404DB0648BF44F008040120FFF7BCF8C2
:10133000E00704D50420BDE81040FFF7E9B810BD70
:101340002882FF1F2482FF1F70B586B0064608233F
:1013500001A80C468DF8103009F0B2F896BB6CB3BA
:10136000314622469DF80B0005F082FC3A250570B7
:10137000024602219DF80A00013205F079FC057051
:1013800002463146BDF80800013205F071FC122119
:1013900002469DF80D0005F06BFC05700246022127
:1013A0009DF80E00013205F063FC0246022102F8AE
:1013B000015B9DF80F0005F05BFC00E02046001B80
:1013C000C0B218E0A01D05F02BFD00258DF80F0020
:1013D0006571E01C05F024FDA5708DF80E00204617
:1013E00005F01EFD01238DF80D0001A88DF81030C9
:1013F00009F066F8284606B070BD0000F8B51D4B30
:101400001D4D1E681423B6FBF3F6B6FBF5F4024639
:101410000021204605F02CFC44214170612181709F
:1014200005FB146679214FF461652023B6FBF5F4C2
:10143000C170024673210370437101710632204668
:10144000002105F015FC05FB14663C253A27B6FB88
:10145000F5F40246077002212046013205F008FC2F
:1014600002460770022105FB14600132BDE8F84016
:1014700005F0FEBBC487FF1F8051010038B50F4B3C
:101480001B68D9789C789D7901EB04245979024630
:101490000904D87901EB05210144187901EB0060BA
:1014A000022105F0E5FB2D23A4B2024603700A21B8
:1014B00020460132BDE8384005F0DABB2882FF1F24
:1014C0007FB5064805F02CFE01A8FFF7D7FF01A85D
:1014D00005F026FE07B05DF804FB00BF5DC200000A
:1014E000B0F5807F10B508D1154B1B882BBB154B71
:1014F0001B8813BBFEF7A8FF03E0124B4FF40072EA
:101500001A80114B1B88B3F5807F02D12020FEF793
:101510009BFFFFF7D5FFFFF76DF90C4805F000FEC4
:101520000B4B1868393005F0FBFD0024094B2046B1
:101530001C70FFF771F9204610BD022010BD00BFDE
:10154000F882FF1F3C82FF1F0083FF1F6FC2000055
:101550002882FF1F7983FF1F313803283FD8DFE837
:1015600000F00211202F1F4B1F491A6809681868E4
:10157000043B1B6823EA000001EA02031843C0F39E
:1015800040107047174B18491A6809681868043BDF
:101590001B6823EA000001EA02031843C0F380102D
:1015A0007047104B10491A6809681868043B1B689B
:1015B00023EA000001EA02031843C0F3C010704799
:1015C000084B09491A6809681868043B1B6823EA34
:1015D000000001EA02031843C0F300207047002016
:1015E000704700BF94F00F4080F00F402DE9F843A2
:1015F000114B1A6892F85070B2F8528001253120D0
:1016000000249946461C40B2F6B2FFF7A5FF00B190
:101610002C436D00392EEDB201D0F0B2F2E7FFF7A6
:101620005DFED9F8003083F8507083F85140A3F87C
:101630005280BDE8F88300BF2882FF1F313803289D
:101640001FD8DFE800F0020910170F4B186880F070
:101650002000C0F3401070470B4B186880F040002A
:10166000C0F380107047084B186880F08000C0F30A
:10167000C0107047044B186880F48070C0F30020DD
:1016800070470020704700BF94F00F40303838B5E5
:1016900003284AD8DFE800F002090406202405E008
:1016A000802403E04FF4807400E04024642945B2B4
:1016B0000AD002DC612938D003E0692904D06F29FF
:1016C0001BD04FF0FF3038BD194B1A6842F400624E
:1016D0001A6002202146032209F068FA154B1A68A5
:1016E00022EA04041C60144B1B68012093F850206C
:1016F00000FA05F522EA050515E00D4B1A6842F4DB
:1017000000621A6002202146042209F04FFA094BB8
:101710001A6814431C60084B1B68012093F8502082
:1017200000FA05F5154383F85050002038BD00BF7E
:101730003880044094F00F402882FF1F21B10E4BE7
:101740001A6842F400621A6010F0010F14BF2023DF
:101750000023810748BF43F040034207074A48BFC0
:1017600043F080030107116848BF43F4807321F4FC
:10177000F0710B43136070473880044080F00F40D5
:101780002DE9F84FB64E336893F8510093F8505056
:10179000284083F851000121FFF7D0FF01243020B9
:1017A000B0462C4200F1010614BF6F216921F6B248
:1017B00040B2FFF76BFF6400382EE4B201D0304630
:1017C000EFE7A84CA84EA94D61235F1C5BB2623BBA
:1017D000FFB20E2B09D8DFE803F0162433414F5D2A
:1017E0006B798795A3CDCDB1BF00236843F48053B7
:1017F000236003204FF48071042209F0D7F92B688D
:1018000043F480731AE0236843F480532360032079
:101810004FF40071042209F0C9F92B6843F40073F6
:101820000CE0236843F48053236003204FF480616D
:10183000042209F0BBF92B6843F480632B6099E024
:10184000236843F48053236003204FF40061042293
:1018500009F0ACF92B6843F40063EFE7236843F425
:101860008053236003204FF48051042209F09EF935
:101870002B6843F48053E1E7236843F480532360EB
:1018800003204FF40051042209F090F92B6843F42F
:101890000053D3E7236843F48053236003204FF4BD
:1018A0008041042209F082F92B6843F48043C5E7A4
:1018B000236843F48053236003204FF40041042243
:1018C00009F074F92B6843F40043B7E7236843F445
:1018D0000063236002204FF48051042209F066F96E
:1018E000336843F4805344E0236843F40063236087
:1018F00002204FF40051042209F058F9336843F4F0
:10190000005336E0236843F40063236002204FF461
:101910008041042209F04AF9336843F4804328E007
:10192000236843F40063236002204FF40041042243
:1019300009F03CF9336843F400431AE0236843F4A8
:101940000063236002204FF48021042209F02EF965
:10195000336843F480230CE0236843F4006323607E
:1019600002204FF40021042209F020F9336843F4E7
:1019700000233360712F01D0FBB226E7D8F8003086
:101980003B4A3C483C493D4CB3F852A0102501234A
:101990004FF400462F464FF4802C4FF400284FF0B0
:1019A000080913EA0A0F70D0802B4CD016D8082BE8
:1019B0003ED009D8022B35D0042B36D0012B40F075
:1019C000C0804FF4807B3BE0202B34D0402B35D0BF
:1019D000102B40F0B6804FF4805B31E0B3F5006F20
:1019E0003BD00CD8B3F5007F2FD0B3F5806F2FD04C
:1019F000B3F5807F40F0A5804FF4805B2AE0B3F51B
:101A0000005F3DD005D8B3F5805F08BFC1F80090F6
:101A100097E0B3F5804F35D0B3F5004F08BFC4F859
:101A200000808EE04FF4007B0AE04FF4806B07E00B
:101A30004FF4006B04E04FF4005B01E04FF4804B87
:101A4000C1F800B07DE00E607BE04FF4005B01E088
:101A50004FF4804BC4F800B073E0266071E000BF23
:101A60002882FF1F3880044094F00F40D4F00F40CC
:101A7000C8F00F4088F00F40C4F00F4084F00F40D2
:101A80000F605EE0C4F800C05BE0802B49D014D842
:101A9000082B3BD008D8022B32D0042B33D0012B9B
:101AA0004FD14FF4807B39E0202B32D0402B33D004
:101AB000102B46D14FF4805B30E0B3F5006F3AD085
:101AC0000BD8B3F5007F2ED0B3F5806F2ED0B3F5D1
:101AD000807F36D14FF4805B2AE0B3F5005F2CD0D5
:101AE00005D8B3F5805F08BFC2F8009029E0B3F5D0
:101AF000804F24D0B3F5004F08BFC0F8008020E02D
:101B00004FF4007B0AE04FF4806B07E04FF4006B6A
:101B100004E04FF4005B01E04FF4804BC2F800B0EA
:101B20000FE016600DE04FF4005B01E04FF4804BD6
:101B3000C0F800B005E0066003E0176001E0C0F8FF
:101B400000C05B00013D9BB27FF42BAFBDE8F88F76
:101B500010B52B4B1A78110604462FD41A78920729
:101B60002ED41A7850072DD41A7891062CD41A78CE
:101B70001B78D20704D513F0400F2249224B1AE0FC
:101B8000580623D4214B1A78D10721D41A7892070A
:101B900020D41A7850071FD41B7819071ED41B4B6A
:101BA0001A78D2061CD41A7890061BD41B781849D0
:101BB00013F0800F174B18BF194614E0164912E0B6
:101BC000164910E016490EE016490CE016490AE0E5
:101BD000164908E0164906E0164904E0164902E0F5
:101BE000164900E0164924B9084605F099FA20463E
:101BF00010BD204605F0E8FA001BC0B210BD00BFC2
:101C000000F007409CBC0000C7BA000001F007408C
:101C1000D4BA0000BBBA000093BC00002CBB00008B
:101C200088BC0000C2BA000014BA000014BB000057
:101C30006CBB0000EDBD0000DFBD0000B4BA0000C9
:101C400019BB000038B508F0DDFD00240546631E11
:101C5000082B06D8DFE803F007090B0D0F11131549
:101C60001700104810E010480EE010480CE0104833
:101C70000AE0104808E0104806E0104804E0104868
:101C800002E0104800E0104805F04AFAA54202D1EF
:101C90000E4805F045FA0E48013405F041FA0A2CC9
:101CA000D5D138BD87C200008FC2000098C20000A5
:101CB000A1C20000AAC20000B3C20000BBC2000063
:101CC000C5C20000CFC20000D9C20000E3C20000BC
:101CD00009C000002DE9F0470C468EB015460B28D0
:101CE00000F2A284DFE810F00C004500A102A0047D
:101CF000A004D6021E048804A004A004A0049C0230
:101D000009B9084605E0042908D10122994B0020B1
:101D10001A70FEF781FD044600F094BC052908BF47
:101D20000222F3D0062908BF0322EFD0072908BFFB
:101D30000422EBD0092908BF0522E7D00A2908BFF1
:101D40000622E3D00E2908BF0722DFD00F2908BFE3
:101D50000822DBD0102908BF0922D7D0112908BFDB
:101D60000A22D3D012294FF00000D4D1814B187031
:101D7000CFE70292202900F25784DFE811F021001A
:101D80003800C3005504B0007700550455045504CD
:101D9000550458006200AD0055045504DC00BE0136
:101DA000BE01550455045504550455045504550405
:101DB00055042500DC00BE01BE0133022D003100B8
:101DC00008F0E2FD00F030BC6B4805F0A9F90020F6
:101DD000FFF7BEFE00F028BCFFF734FF00F024BC84
:101DE00092F90000303808F065FD00F01DBC634832
:101DF00005F096F9624805F093F9624805F090F90C
:101E000005F082FA822105F09BF95F4805F088F918
:101E100005F06EFA822105F093F95C4805F080F92F
:101E200005F05AFA822105F08BF95948F6E304A827
:101E3000FFF7E4FA00240470564805F071F904A88D
:101E4000E9E11378313BDBB2032B01D95248E5E3DA
:101E5000524805F065F9029B93F90000FFF7EEFB8D
:101E6000044608B94E48D6E14E48D7E31078A0F1B1
:101E70003103DBB2032B01D94B48CFE340B2FFF76C
:101E8000DDFB044608B14948C8E305460126312078
:101E9000471C40B2FFB2FFF75FFB08B13543EDB21C
:101EA0007600352FF6B201D0F8B2F1E7029804F0CF
:101EB0009AFFC0B2461E02980123184403FA06F6A0
:101EC000029004F090FF01280CBF3543B543E8B2FF
:101ED0000021FFF733FCB5E3FFF788FBA4E3137899
:101EE000313BDBB2032BC7D8314805F019F9029B0F
:101EF00093F90000FFF730FB044608B12D488DE34D
:101F00002D4888E10EAC104644F8282D04F06BFFF4
:101F100005462046FEF752FC08B128487EE3049BA4
:101F200005F12F0040B293F90010FFF7AFFB002836
:101F300000F07A83F1E792F900300BB9102652E0F5
:101F4000104604F050FF1E4B186002A8FEF736FC46
:101F5000029B1A78002AF1D002F0DF0252B24C2A1A
:101F600001D1042102E0572A2ED10221154A013362
:101F700011602FE07983FF1FEDC2000001C3000054
:101F8000DDBE000018C30000C2D0000025C3000061
:101F9000D7BE000037C300005CC300006EC3000062
:101FA00081C300008AC3000092C30000A1C30000E7
:101FB000B1C30000BEC30000C2C30000C6C300001E
:101FC0003482FF1FFC81FF1F422A04D1A44A012151
:101FD00011600B440293029890F90030002BADD0B1
:101FE00004F01EFF06469F48DFF874A205F098F83B
:101FF00020238DF810308DF811305746002E40F315
:102000001383994D8421286805F09AF8974805F0C4
:1020100087F80DF112084FF01009DAF80020022AB3
:1020200017D0042A28D0012A40F0FE821B2C07D1A9
:1020300028680DF1060108F03DFA9DF8063001E030
:102040002B681B783968039341F010019DF80C0050
:1020500020E01B2C07D128680DF1060108F02AFAB0
:10206000BDF8063001E02B681B883968039341F006
:102070001001BDF80C000DE01B2C04D1286803A949
:1020800008F018FA02E02B681B680393396803987C
:1020900041F01001C9B205F053F83B682A68039873
:1020A0001A44022B2A60C3EB090904D0042B0CBF8D
:1020B0001822002200E00822434498450ED020FA5E
:1020C00002F1A1F1200C5FFA8CFCBCF15A0F94BF15
:1020D000C9B22E2108F8011B083AEEE7013E02D0F2
:1020E000B9F1000F99D10D221A700A225A700022FC
:1020F0009A7004A805F014F880E792F90030002BDC
:1021000000F09282104604F06EFE112C054601D0BC
:102110001D2C01D1564800E0564805F001F802A8F0
:10212000FEF74CFB029B1A78002A00F07D8202F039
:10213000DF0252B24C2A01D1042102E0572A04D115
:1021400002214D4A0133116005E0422A04D14A4A76
:10215000012111600B44029302A8FEF72FFB0298A5
:1021600004F041FE049002A8FEF728FB112C01D0D8
:102170001D2C06D1029890F9003013B104F050FEE6
:1021800000E001201C3CE4B23B4F012C8CBF00243A
:1021900001240646B846002E40F346823A68022AD9
:1021A0000AD0042A13D0012A17D1049B14B18DF848
:1021B0000C3005E02B7010E0049B34B1ADF80C300E
:1021C000284603A908F024F907E02B8005E014B1A4
:1021D000284604A9F6E7049B2B60D8F80030013E9E
:1021E0001D44D8E792F90030002B00F01D82104604
:1021F00004F0F9FD044602A8FEF7E0FA029890F90F
:10220000001011B104F0EFFD0146204608F0EAF895
:10221000044618B9194804F083FF13E21848FDE199
:1022200008461146FEF79AFB75E549B1032940F0CF
:10223000FB81144B10461C6804F0F2FD2084F3E18E
:10224000114D2B88042B05D1104804F069FF102391
:102250002B80F7E10E4B08461980FEF7F5F8F1E107
:10226000FC81FF1FCEC300003482FF1FCFD20000CD
:10227000DFC30000E6C30000F481FF1FEEC30000CF
:10228000F7C300002882FF1F3C82FF1F07C4000025
:10229000F882FF1F1D2900F2C781DFE811F01E0040
:1022A0006500320047008200C501C501C501C501B6
:1022B000C501C501C501C501C501C501C501C501EE
:1022C0009F00C501C501C50113011301C501C50169
:1022D000C501C501C50127013D01A84BA84F1E68D6
:1022E00000244FF0070808FB0470294604F056FF4D
:1022F00010B986F8244094E101340C2CF3D1A148A4
:102300008CE192F90030372B05D19C4B1B68DA69C0
:1023100042F0010206E0382B06D1984B1B68DA69BF
:1023200022F00102DA617CE1974877E1934B974F05
:102330001E6800244FF0050808FB0470294604F0CD
:102340002DFF60B9F36923F006032CB1012C40F096
:10235000638143F002035FE143F004035CE1013475
:10236000032CE9D18A4859E1844B8A4F1E68002426
:1023700007EB8400294604F011FF68B9F369012CCA
:1023800023F0180305D0022C40F0468143F01003DF
:1023900042E143F008033FE10134032CE8D17E48D9
:1023A0003CE1764B7D4F1E68002407EBC4002946B4
:1023B00004F0F4FE68B9F369012C23F0600305D042
:1023C000022C40F0298143F0200325E143F0400333
:1023D00022E10134032CE8D171481FE1674C7148B8
:1023E00004F09EFE704804F09BFE236893F82430AE
:1023F0000B2B97BF624A6D48072000FB032004F0B7
:102400008FFE6B4804F08CFE2368DB69DF074CBF4E
:102410006848694804F084FE684804F081FE236837
:10242000DB699E0705D413F0040F0CBF02230023C1
:1024300000E00123554A052000FB032004F070FE54
:102440005F4804F06DFE23685248DB69DD0654BF27
:10245000C3F3C003022300EB830004F061FE59487C
:1024600004F05EFE2368DB69580605D413F0200FE4
:102470000CBF0025022500E00125534804F050FE62
:10248000464800EBC50004F04BFE494804F048FE06
:10249000002D00F0C9804D4804F042FE2368002161
:1024A00093F84E0004F042FE494804F039FE4948D2
:1024B00004F036FE2368002193F84F0004F036FE46
:1024C0004348ABE0104604F0ABFCC0B2632803D82D
:1024D000002808BF012000E06320284B1B68152C52
:1024E0000CBF83F84E0083F84F009AE03A4804F09E
:1024F00017FE3A4804F014FE012007F001FB1821F2
:1025000004F014FE364804F00BFE002007F0F8FA41
:10251000182104F00BFE87E04FF0FF3007F0F0FACF
:1025200030487BE08C1E082C7ED8DFE804F0057D67
:10253000107D7D7D61211800FEF7C2FFFEF75AF97C
:10254000294804F0EDFD0D4B1868393066E00B4B5F
:10255000186811463930142204F08EFC64E004A996
:102560000020FEF7F1FE04A804F0DAFD104855E063
:1025700001201146FEF7E8FE1C484FE02882FF1FAD
:1025800064BD00001CC5000013C40000D0BD0000E5
:1025900035C5000021BA000048C50000ACBE0000EF
:1025A0005EC500002BC4000044C400004CC4000001
:1025B00009C0000055C4000057C4000059C4000001
:1025C0003EC5000061C4000070C400007EC400006D
:1025D0008AC400008EC4000099C40000AEC400008C
:1025E000BFC40000D0C400006FC20000EBC40000F4
:1025F0001046FEF7CDFD17E0062915D11348114608
:1026000004F0CCFD044688B11148294604F0C6FD0B
:10261000044688B10F4801E0F36102E004F080FD58
:1026200002E00420FDF774FF00240BE00A4B1B6856
:102630005A8C42F0400204E0074B1B685A8C22F08F
:1026400040025A8420460EB0BDE8F087FAC400006C
:1026500001C5000009C500002882FF1F2DE9F04FC9
:102660008B4C8C4E85B00546029289464FF000088F
:10267000A246B9F1000F00F006812A78082A09D194
:10268000237823B1013B8448237004F049FD0023E3
:102690003370F3E01B2A04D05B2A05D133781B2B5F
:1026A00002D132700135E9E033785B2B4BD1A2F1D6
:1026B0004103032B47D8DFE803F00E0E080223780E
:1026C000002B00F0DB80013BD7E02378272B00F2C2
:1026D000D5800133D1E0714FDFF8D0B13A682820BE
:1026E00000FB02B004F07AFD2A780390412A3A6890
:1026F00006D10AB9032200E0013A3A60684805E0D1
:102700000132032AC8BF002266483A6004F008FD7F
:10271000039A32B16448019204F002FD019A013A31
:10272000F7E7604804F0FCFC3868282202FB00B0A0
:10273000019204F0F5FC3868019A02FB00B004F045
:102740004DFD20709AE00A2A00F09880002A00F0DF
:102750009580DFF848B194F800C0DBF800005349D9
:10276000282303FB00C00A542A780D2A78D10A22B4
:102770000A54029801910093FDF7AEFE0199DBF82F
:102780000020009B4A4803FB02134A49227809783B
:102790004FF00C0E0EFB01F10132D2B200EB010E34
:1027A00050F801809EF805E09918002001F8010C0E
:1027B0000299CDF80CE029B93F49098800293FD09A
:1027C00049053DD4002A38D04FF0000C039A6245E9
:1027D00018461ED0D8F800108DE80810FDF7D5FF78
:1027E000DDF804C0009B0CF1010C024670B13348C7
:1027F000019204F095FC98F8080098F80910019AE5
:10280000FFF768FA90B9FEF775F80FE008F10C08C9
:10281000DCE72B49FDF7B9FF024670B1042009211E
:10282000FFF758FA10B9274804F07AFC029B3BB92D
:10283000214B1888FDF708FE02E0234804F070FCE5
:10284000FDF75CFEDBF80010144B01310022032978
:102850008AF80020D4BF19601A604FF0010803E025
:102860000CF1010C84F800C0002333709AF800309A
:10287000272B05F1010501D92723237009F1FF3921
:102880001FFA89F9F5E6404605B0BDE8F08F00BFB4
:102890007883FF1F7A83FF1F1EBA00003882FF1F54
:1028A00077C50000D8BE0000D2D200005882FF1FBA
:1028B000E0BC00007983FF1F0083FF1F09C00000F8
:1028C0007BC50000CAC30000C6C30000022AF8B5D9
:1028D0000C4641D0042A02D0002A2FD109E0037807
:1028E000822B3BD11F4B204918780D2204F0F6FBB8
:1028F00034E0067826F08003212B31D18179C37929
:102900001A4D41EA032736062F8029D52A804278BE
:10291000FE2A02D0FF2A0DD022E0827802BBC278C4
:10292000F2B901291CD1DBB9114B124918780122E7
:1029300004F0D4FB082C0FD9083CA4B20B4B1A8826
:1029400052B10D4800219442017001D3198005E075
:10295000141B1C800620F8BD0020F8BD0320F8BD24
:102960000420F8BD8C83FF1F0082FF1F7C83FF1FA4
:10297000A085FF1FD4CF00007B83FF1F2DE9F04708
:10298000204D214F287800210A4604F0A7FBB846C5
:10299000044640F2FF1A3B6853B3544520D9DFF890
:1029A00078901A4E99F800003268002104F018F867
:1029B00080B999F80020164B287853F822304FF44C
:1029C0000072596904F08AFB3368A4F5007401337E
:1029D000A4B23360D8F80030013BC8F80030DAE721
:1029E0002878402141F27502BDE8F04704F060B854
:1029F0000C2CF5D9287807490D22BDE8F04704F0E2
:102A00006DBB00BF8C83FF1F9885FF1F8483FF1F52
:102A10009C85FF1F0082FF1F9485FF1F38B5364B32
:102A20001B6804467BBB35482146042204F0A7FB03
:102A300028BB637B324A13700BBBA37B013BDBB229
:102A40000F2B1CD894F90C30002BE37B2DDA232BB1
:102A500023D016D9282B32D0A82B30D0252B1CD030
:102A6000284D211D0422281D04F006FA05F1080056
:102A700004F10801042204F0FFF901232B73042060
:102A800038BD122B01D1072038BD1A2B01D0032BE2
:102A900030E0237C5B0929D0E2E71B4B1B681B8BD2
:102AA00003F08803002BDBD0EDE71E2BEBD002D820
:102AB000002BE8D0D4E72A2B01D0AA2BD0D1124B7F
:102AC0001A68138B03F08803002BC9D0A37C617CA8
:102AD0001B0443EA0163217D0B43E17C43EA0123AC
:102AE0000A490B6012699342BAD2CCE7637C03F0C7
:102AF0003F033F2BB4D1C6E78083FF1F55CF0000B3
:102B00009485FF1F0082FF1F9C85FF1F8483FF1F8A
:102B10002DE9F047B64F867B3B78A6B01BB1B54C8C
:102B20000DF11D057AE0B44BD3F8008008F12100C7
:102B300004F054FBB14B44001A681ABFA51CEDB257
:102B4000042599463AB9284604F076FB0323C9F8D0
:102B5000000005704370D9F8003024B1023308F149
:102B60002001002002E09C70DC7008E011F8012FC9
:102B7000023322B103F8022C03F8010CF6E700241B
:102B80009F4B8DF81240012521464FF002084FF06F
:102B9000750901AA05200193ADF80A40ADF8084077
:102BA000ADF80E508DF814508DF815808DF81690F4
:102BB00004F03CF84023ADF82430924B38704FF4C9
:102BC00080620693ADF81E204FF400732146052065
:102BD00006AAADF82240ADF81C30ADF820308DF8D3
:102BE0002A908DF827508DF8268004F01FF8864B28
:102BF000864C874F18702578284603F033FF2378DA
:102C000047F825000133DBB22370002BF3D086E7B1
:102C10009DF81B00012809D0752828D0304606A948
:102C2000052203F05DFF0028F2D136E09DF81C304C
:102C3000CB2B17D007D8CA2BF0D10220002105F0EA
:102C400051FC744826E0CC2B04D0DD2BE6D1FFF7F5
:102C500095FEE3E7704A714800231360704A2360D1
:102C6000136017E0002105F03DFC6E4812E030468D
:102C700029469DF81C2003F033FF9DF81D30FE2BE4
:102C8000CCD1694804F04CFA9DF81E00012104F0F3
:102C90004DFA664804F044FAC0E75B4E554FB04623
:102CA000307803F02DFF002800F05C813C68DFF8ED
:102CB00044A1307844B35A4C5D4D2168C1F500728F
:102CC00092B2294403F00CFF3B681B1A3B60236857
:102CD0001844B0F5007F206011DB4C4B1878554B41
:102CE0001A68511C1960294603F094FE00232360E2
:102CF0003B6823B17520042104F056FC32E1DAF878
:102D00000030002BCCD126E14B4DDFF8009106A915
:102D1000802203F0E5FE042207A9281D04F0ACF888
:102D200030782C7201216C72AC72EC722C7303F04F
:102D3000F9FE9DF924309DF82520002B89F800200C
:102D40009DF8273080F2D980232B00F08C8007D8A3
:102D5000122B2AD01A2B2ED0032B40F0FC80B0E08F
:102D6000282B3DD0A82B6BD0252B40F0F480284B8E
:102D7000307853F8222013698DF808408DF8094007
:102D8000128D013B110A8DF80B201A0E8DF80420CC
:102D90001A0C8DF805201A0A8DF80A108DF80620F5
:102DA0008DF8073001A90822D3E09DF828305B098F
:102DB00000F0CC80ADE02149042201A804F05CF8C9
:102DC00099F80020124B98F8000053F822301B8B22
:102DD000D90644BF80238DF8063001A90422B8E04B
:102DE0009DF82E209DF82F3043EA022236E000BFE6
:102DF000A085FF1F8083FF1F2482FF1F8883FF1F82
:102E0000CD2800001D2A00008C83FF1F9485FF1F22
:102E10009C85FF1FB6CF00009885FF1F9ACF00004A
:102E20009083FF1FA6CF0000C3CF0000D0CF0000CB
:102E30009483FF1F8483FF1F0082FF1F74CF000055
:102E40009DF82E209DF82D30120442EA03629DF871
:102E500030301A439DF82F3042EA0322434B1A6068
:102E6000FFF78CFD1CE79DF82F309DF82E40404960
:102E70000C2201A843EA042403F0FEFF99F8002085
:102E80003C4B53F82230198B11F0880F11D08A0671
:102E90004CBF022201228DF80C201B691A0A8DF802
:102EA0000B308DF80A201A0C1B0E8DF809208DF8B6
:102EB000083098F8000001A90C2C34BF22460C22DF
:102EC00047E0122201A82C4903F0D6FF99F8002010
:102ED000284B53F822301B8B03F0880343B970232F
:102EE0008DF8043002238DF806303A238DF8103027
:102EF00098F8000001A912222BE02A2B0CD0AA2B53
:102F00000FD043BB1B4B53F822301B8B03F08803BD
:102F10000BBB01232B731EE09DF82E209DF82F3054
:102F20000BE09DF82E309DF82D201B0443EA026330
:102F30009DF8302013439DF82F2043EA02233B6085
:102F4000DAF800305B02CAF80030A9E630780B49A5
:102F5000242204F0C3F898F8000009490D2204F077
:102F6000BDF89DE626B0BDE8F08700BF9885FF1F3D
:102F700016D000009C85FF1FD5CF0000E8CF0000D1
:102F80000082FF1F122303800048704778CF0000A3
:102F9000202303800048704735CF000005280346F2
:102FA0000DD8094A52F82000027832B9032B08D113
:102FB000064B186803780B8070470A807047002022
:102FC00070471046704700BF5CCF00008883FF1F2A
:102FD00003688B4270B504460D461CD0038BDB079B
:102FE0000ED50E4E94F84830616956F823302268A9
:102FF000204698470130F5D0238B23F0010323832B
:1030000094F84820064B256053F822306269204628
:103010002946984770BD002070BD00BFEC86FF1F99
:10302000B485FF1F10B500231A46C45CD101C9B294
:1030300004EB5202013351FA82F20B2BD2B2F4D1DB
:10304000104610BD30B5446885680B6804EBC505B3
:10305000184C2C40002C03DA013C64F007040134C6
:10306000072C25D8DFE804F004070A1215181E21E2
:10307000C3F30B031CE0C3F30B3319E01B0EBAB10F
:103080004A6802F00F0243EA02230FE0C3F30B1376
:103090000EE0C3F30B430BE01B0F4AB10A7943EA7E
:1030A000021303E0C3F30B2302E01B0D0022C260F6
:1030B000184630BD0700008010B58468406800EBFA
:1030C000C4042D482040002803DA013860F00700CE
:1030D000013007284DD8DFE800F0040B132028301A
:1030E0003E46136823F47F6323F00F0319433FE048
:1030F000136823F47F0323F4704343EA013137E07C
:10310000106820F07F4040EA016010608BB3536884
:1031100023F00F0343EA11211BE0136823F47F43DC
:1031200023F0F00343EA011122E0136823F07F63E8
:1031300023F4702343EA01411AE0106820F0704044
:1031400040EA01701060A3B1536823F0FF0343EA23
:10315000111151600DE0136823F47F2323F4706391
:1031600043EA012104E01368C3F3130343EA015166
:103170001160002010BD00BF070000802DE9F04F56
:10318000874B542404FB0134ADF5057DA56894F804
:103190002B30266A401BB0FBF3F563681D44238B7C
:1031A00003F4C0438B4617463BB106EB15264FF69A
:1031B000FF731F3DEDB2029307E06FF0704C06EB1A
:1031C000D516CDF808C005F07F05764B204653F89C
:1031D0002B30314604AA9847824618B90390DFF88D
:1031E000C89148E06FF0030AD4E004A951F82530F3
:1031F000DDF808C003EA0C01614549D061688B42E3
:1032000046D9022FD4F820807CD0002A00F0A48078
:1032100015F0010F4FEA5505EDB204A900F09480B6
:1032200031F8250041F82500DDF80CC00CF1010C47
:10323000CDF80CC0002A00F0938008EB1328DDB213
:10324000B04518D04FF0000C94F82A30634500F2D6
:103250008C8059F82B30204604A93246984701301B
:10326000F7D0504B204653F82B30414604AA9847DC
:103270000028B7D14646208B10F4C042B5D004A92F
:103280006B0851F82330E9074CBF1B0C9BB2AFE72A
:10329000022F7FD09AB115F0010F4FEA5505EDB21C
:1032A00005D004A931F8253041F825300AE004AAF8
:1032B00052F825301B0C1B0442F8253002E004AB09
:1032C00043F82520410707D5236B039F01333B4477
:1032D00040F00200236320830025334F284694F8F2
:1032E0002A30AB420CD9E26957F82B3002FB056259
:1032F000204604A99847421CF5D00135EDB2EEE70F
:10330000824647E0CAB115F0010F4FEA5505EDB20C
:1033100009D004A830F825206FEA02426FEA124271
:1033200040F8252034E004A951F825206FEA124224
:103330006FEA024241F825202AE004AF6FF07041A5
:1033400047F8251017460BE051F82500010C04A89A
:10335000090440F8251067E704A941F8252063E730
:1033600008EBD31803F07F056AE7E26959F82B30C0
:10337000CDF804C002FB0C62204604A99847013036
:10338000DDF804C0F1D00CF1010C5FFA8CFC5BE7B6
:10339000002752E750460DF5057DBDE8F08F00BFD0
:1033A0004887FF1FB485FF1FEC86FF1F37B5BDF8A8
:1033B00018401D19B5F5007F0568C4BFC3F500743A
:1033C000A4B28D4207D1416910461944224603F048
:1033D00053FD002006E090F848500094024C54F849
:1033E0002540A04703B030BDB885FF1F08B549028E
:1033F00001F5B43011464FF4007207F05BF800207D
:1034000008BD08B503F5B43303EB41201146BDF800
:10341000082007F04FF8002008BD70B5520202F5F1
:10342000B43626F4FF64ADF5006D24F007040D46B4
:10343000204669464FF4006207F03CF8361B00ABAB
:103440001E44304629464FF4007203F098FE78B1CE
:103450004FF400722946304603F00EFD002120464D
:1034600006F0C0FF204669464FF4006206F0D0FF28
:1034700000200DF5006D70BD30B5ADF5017D054640
:103480000C46684600214FF4007203F0EDFC28461C
:1034900069462246FFF7C1FF0DF5017D30BD73B5CA
:1034A00004460E4601A80DF1060107F0D3F838B125
:1034B0004FF4C043ADF8043044F2EB43ADF80630AE
:1034C000BDF80400BDF80630C5B2DAB2000A1B0A26
:1034D000A575E0752276A2746376E3741EB1A573B8
:1034E000E0732274637402B070BD10B50B0A81766C
:1034F000C3760B0C090E04464175C2720375002198
:103500001C30042203F0B0FC20460121BDE810402D
:10351000FFF7C5BF2DE9F0411D4BC76A90F8488001
:10352000ADF5007D53F8283039466A460446984781
:10353000064610B16FF0030624E0256B636B8DF82F
:10354000E8512A0A8DF8E9212A0C8DF8EA212D0E7E
:103550001A0A8DF8EB518DF8EC318DF8ED210D4DF7
:103560001A0C1B0E8DF8EE218DF8EF3155F828302E
:10357000204669463A4698470130F7D0238B23F01E
:103580000203238330460DF5007DBDE8F08100BFC6
:10359000B485FF1FEC86FF1F08B5084B08481A8B3F
:1035A00042F008021A83074B32221A6003F0B8FD7A
:1035B0000548BDE8084003F0B3BD00BF4887FF1FC2
:1035C0003CD000009C87FF1F4BD0000010B50C4C76
:1035D0000C4B94F84820216853F822306269204649
:1035E000984758B9636993F8FE21552A02D06FF0C5
:1035F000020010BD93F8FF31AA2BF8D110BD00BF17
:103600004887FF1FB485FF1F4FF4C07300EB4002D3
:10361000B2FBF3F2032330B5B2FBF3F403FB142344
:103620000A601BB1012B0CBF022301230324B2FB50
:10363000F4F2074D8B6092025D43801A04FB005048
:1036400090FBF4F423444B60082390FBF3F030BD6F
:1036500000FCFFFF70B54B6801334B600D4681687D
:1036600090F82B20591AB1FBF2F602FB16118AB022
:103670000446002964D1068B06F4005292B2FAB1D6
:10368000C2680232934252D05AD306A92868FFF783
:10369000BBFF082186B2226A00910699B30011444B
:1036A0009BB2204604AAFFF781FEE0B9A92E06A826
:1036B00004A98CBF00220122FFF7C4FC039027E07D
:1036C000760417D5C16802318B4233D038D32A68CB
:1036D000016AD3B2022601EB1221009606AA5B0012
:1036E000FFF764FE10B16FF003002AE0BDF8183058
:1036F00003930DE02A68016A02F07F03042601EBC0
:10370000D211009603AA9B00FFF750FE0028EAD1D1
:10371000039B6268934210D9626A93420DD82B6072
:1037200094F82B10E26803FB01236B6008E06FF054
:10373000070006E06FF0080003E06FF0060000E00D
:1037400000200AB070BD0A7A0132D2B20A7210B5F6
:10375000048DB2EB541F05D300220A72BDE810405D
:10376000FFF778BF002010BD30B5436A90F83E20C7
:1037700085B001460BB3144B542404FB023401A85A
:1037800020310C2203F078FBE525238B029943F0CE
:10379000010323832046FFF71BFC80B99DF80C3002
:1037A00062695B01D15CD55421F04003012B04DD3B
:1037B000204601A9FFF7C7FFE7E7002001E06FF00F
:1037C000030005B030BD00BF4887FF1F2DE9F04F53
:1037D00089B00D4614460393029008B1A04800E05A
:1037E000A04803F09DFC284603F09AFC636ADFF8CA
:1037F000F8B20BB99C4848E09C4803F091FC9C4807
:1038000003F08EFC812194F8280003F099FC99487C
:1038100003F086FC8421606A03F092FC964803F072
:103820007FFC8421206A03F08BFC944803F078FC31
:1038300021464FF0540951F8203B93F83A3005A83F
:103840000C2209FB03B903F017FB4FF000084646B2
:10385000474648460699FFF7BBFB024600287CD145
:103860009DF81C30D9F814105B01CD1811F803A095
:103870003FBBBAF1E50F0DD1814803F051FCEA7A64
:1038800002F03F020F2A03D07E4803F049FC64E0B7
:1038900016BB12E01AF0400F0AD00AF0BF0A7A48AD
:1038A00003F03EFC5046082103F040FC012704E0F1
:1038B000764803F035FC01260EE095F80D8056465B
:1038C0000AE0013EF6B2564505D07148019203F078
:1038D00027FC019A164601276E4803F021FC0023BD
:1038E000E85C0193912103F02BFC019B0133202B19
:1038F000F6D1694803F014FCEB7A03F03F030F2B79
:1039000001D066481EE02B7B1BB9AB7E0BB9EB7E6A
:10391000A3B1634803F004FC2B7B13B1614803F0AF
:10392000FFFBAB7E13B1604803F0FAFBEB7E13B1F3
:103930005E4803F0F5FB5E4803F0F2FB6B7B43450A
:1039400002D05C4803F0ECFB012E06D0484605A9E6
:10395000FFF7F9FE07307FF47CAF574803F0E0FB38
:103960008121207F03F0ECFB424803F0D9FB842146
:10397000A06903F0E5FB404803F0D2FB84216069B5
:1039800003F0DEFB3D4803F0CBFB2368A16993F80D
:103990003A30542505FB03B52846FFF719FB0646C8
:1039A000002840F0CA80277F6B693A4803EB47172D
:1039B00003F0B6FBB85D9121013603F0C1FB202E68
:1039C000F8D13E4803F0ACFBFB7A042B10D005D8AD
:1039D000012B0BD0022B11D1394810E0102B09D04C
:1039E000202B09D0082B09D1364808E0364806E0DC
:1039F000364804E0364802E0364800E0364803F036
:103A00008FFB364803F08CFB00232E21FA5CA2F1D9
:103A10002000C0B25E2805A894BFC254C15401332F
:103A20000B2BF3D100238DF81F3003F079FB636A71
:103A300043B12B4803F074FB039B812193F86C0284
:103A400003F07EFB029B002B50D0264803F068FB5E
:103A5000A068002103F06AFBE66A246B4DE000BF1A
:103A60005CD0000063D000006FD0000079D000006F
:103A700082D00000DFD1000097D000006CC40000AD
:103A8000A2D00000B0D00000B6D00000C9D0000025
:103A9000DED00000F1D0000009C00000F8D0000026
:103AA00010D1000029D20000CDC200007EC100006C
:103AB0002AD1000038D1000053D100006ED100009F
:103AC00085D1000093D100007BD100008CD1000093
:103AD0009DD10000A7D10000AFD10000B3D10000FC
:103AE000B8D10000C5D100004887FF1F039B95F89F
:103AF0002B40DE68EB6806FB043411482D6A03F0A6
:103B00000FFB8421204603F01BFB0E4803F008FB4B
:103B10008421304603F014FB05EBD6150A4803F068
:103B2000FFFA8421284603F00BFB084803F0F8FA5B
:103B300006F07F00892103F003FB09B0BDE8F08F98
:103B4000D6D1000097D00000EBD10000F9D10000E1
:103B50002DE9F04FADF23C4D9046056A90F848A033
:103B6000102204460F4606A8002107F05FFC0AA8B1
:103B70000021102207F05AFC18F00C0F07D1238BFC
:103B8000590703D5676B236B9F4200D96768238B66
:103B90009A040DD506A93846FFF736FD069B8146E7
:103BA000EB180AA806A91022029303F065F90EE0AB
:103BB0005E0407D505EB17255FFA87F902954FF0EC
:103BC000FF0B06E005EBD715029507F07F094FF0D4
:103BD0007F0B02993E4603914D46B24A039952F833
:103BE0002A300DF1380C6246CDF800C020469847C7
:103BF000DDF800C0002840F06F816346228B9004FE
:103C00000ED5A92D4FF00101099106A803EB8501FE
:103C10008CBF002201220193FFF714FA019B0DE0F3
:103C2000510409D5022195FBF1F253F82200EA076D
:103C30004CBF000C80B201E053F82500002840F092
:103C4000378118F0030F11D1238B13F4005F0DF1AE
:103C5000380B69D0A92D06A840F6FF710BEB850241
:103C60008CBF00230123FFF727FA76E094F82B306E
:103C700004930499E36801FB063305939C46049B77
:103C8000059A1344CCEB030313F0FF03DCD094F844
:103C90002B209A4239D118F0010F36D00DF50E7B4A
:103CA00000214FF400725846CDF800C003F0DCF854
:103CB00020210B22584603F0D7F82E238BF8003032
:103CC0005846394610220193FFF70FFC20210B22A2
:103CD00096A803F0C9F8019B96A88BF820308BF8C2
:103CE000213002211022FFF700FCDDF800C06E4AEF
:103CF000204652F82A30CDF800C06246594698470F
:103D00000130DDF800C0F2D00BE06849204651F8E0
:103D10002A30CDF800C0614698470130DDF800C078
:103D2000F3D00CF1010CAAE75B0412D5022295FB3B
:103D3000F2F215F0010F5BF8223015BF6FEA034372
:103D40006FEA13436FEA13436FEA03434BF82230E1
:103D500003E06FF070434BF8253018F0040F30D0BB
:103D6000238B03F4005292B26AB1B9F1A90F0AA8E9
:103D700031460BEB89028CBF00230123FFF79CF92E
:103D80004FF000081DE003F480439BB2F3B115F03F
:103D900001084FF002030AD099FBF3F990465BF853
:103DA00029301B0C1B0433434BF8293009E0A9F1DF
:103DB000020999FBF3F93BF8293043EA06434BF833
:103DC00029304FF00009DFF8E0C017E04BF8296018
:103DD0009846F6E7E269DDF80CE05CF82A30CDF8A9
:103DE00000C02046594602FB09E298470130DDF841
:103DF00000C0EFD009F101095FFA89F994F82A307F
:103E00004B45E7D818F0080F10D1238B5F0747D533
:103E1000626B43F002032383236B964228BF721C1C
:103E200003F1FF3328BF6263236339E01D4B02991E
:103E300053F82A3020465A46984700284CD1238B05
:103E400003F4C043A3B1FFB215F0010F4FEA5707C7
:103E500005D05BF827301B0C1B04334303E03BF811
:103E6000273043EA06434BF8273000250E4F12E077
:103E700007F07F074BF82760F7E7E269DDF808E015
:103E800057F82A302046594602FB05E29847013090
:103E9000F3D00135EDB294F82A30AB42EDD8B4E757
:103EA00030461BE0B485FF1FEC86FF1F4487FF1FD1
:103EB0005D4506F1010608DA079A01320792099A70
:103EC000002A7FF49BAE013598E60399013108F092
:103ED000FB080391002580E66FF003000DF23C4DD6
:103EE000BDE8F08F7FB5038B0A6803F4C0430D462D
:103EF0000446016A9BB1D3B2022601EB122100965F
:103F00000DF10A025B00FFF751FA10B16FF00300E8
:103F10002FE0BDF80A3003934FF6FF730DE002F077
:103F20007F03042601EBD211009603AA9B00FFF742
:103F30003DFA0028EAD16FF07043039A61688A4223
:103F400001D99A4205D3204629680E22FFF700FEC8
:103F500003902A68636A9A4209D8039BE2682B603F
:103F600094F82B1003FB01236B60002001E06FF03D
:103F7000060004B070BD00002DE9F04F8FB0C2F311
:103F8000C03390E8C0000992069391F83A20A64BFE
:103F90008B46542101FB02310291044639460BA89D
:103FA0000C2202F069FF96F900305C2B01D02F2B18
:103FB00000D101360023059304F11E0A2021E66298
:103FC00050460B22CDF81CA002F04EFF1823002112
:103FD00084F82930B1468C460B4601254FF0050880
:103FE00016F8012B50B20D2813D003DCB0B10A280B
:103FF0000FD016E02F2811D05C280FD02E2810D11A
:10400000002B00F08280082B66DC01210823B146DA
:10401000E6E7002B00F081804E4682E0002BF6D0D0
:10402000FAE7D0B2202804D8002BF0D0202AEED115
:1040300050E07E283AD8DFF8F4A14AFA82F919F85C
:10404000219C19F0210F09D0BCF1000F02D019F00A
:10405000200F41D119F0400F3CD1D8E7BCF1000F3F
:104060003AD119F0040F0CD094F8290021B920F0AE
:10407000080084F829002FE020F0100084F82900BF
:1040800041E019F0080F27D0A0F12002D2B294F835
:10409000290029B940F0080084F8290003251BE015
:1040A00040F0100084F8290003252CE000F17F097E
:1040B0005FFA89F9B9F11E0F03D92030C0B21C286C
:1040C000A5D84BB950B21B301FD1012384F81E80F4
:1040D0009C469CE75F220425072B16DD09B10A2BBD
:1040E00013DD324612F9013B0D2B19D003DCBBB1B5
:1040F0000A2B04D114E02F2B03D05C2B01D01646E1
:10410000EFE702250DE0072BE9DCDDF81CA04FF0FE
:10411000000C0AF80320013379E74FF0FF3500E087
:104120000425A561013561D06663266396F90030E8
:104130005C2B01D02F2B00D101364FF000090298E3
:104140007968FEF745FF8046002847D1029B97F823
:1041500008A05B694FEA4A1A1D4603935544B9F11A
:10416000000F2FD1059BC3B904F138031846394617
:104170000C22089302F080FE0398069910F80A308A
:1041800011B9E52B35D1D0E19BB32B7B8BBBAB7E3B
:104190007BBBEB7E6BBB012364E0059B013B05937E
:1041A00040F0FE81236D132B00F2F5815A1C22652D
:1041B0000D2202FB034029460B2200F5B47002F0E9
:1041C0005BFEEDE12846FEF72DFF94F86C3283424A
:1041D00040F0DD810120A0618146D9E16FF0030844
:1041E00000E296F90030002B00F0CE806FF002085C
:1041F000F8E1EA7A02F03F030F2B32D0039810F86F
:104200000A1031B9082B0CBF6FF004036FF00103E3
:1042100010E0E5290CD1216BE36A994208D1636B68
:10422000236302235FE000BF4887FF1FE4D2000042
:104230006FF00203082A00F07D81226D132A00F23C
:104240007C81511C21650D2101FB024000F5B470F9
:1042500029460B22019302F00FFE00210491019BDD
:1042600072E10023039A049312F80A3003F040022B
:1042700002F0FF002AB1E52B00F0FC80636B012007
:1042800023630D2212F1FF3280F0FB80002800F042
:10429000428104F1440008990C2202F0EDFD002354
:1042A00084F86E326B7B84F86C3294F86E3203982B
:1042B000226BE16A013384F86E3210F80A3003F0A1
:1042C0003F03012B40F02D818A4240F03B81626B1D
:1042D0002263049A3AB1039810F80A30E52B14BF10
:1042E0004FF0FF33012394F86D2272B1501E0C225F
:1042F00002FB00406C3004F16001019302F0BCFD50
:10430000002284F86D22019B6266DA1C052A00F205
:10431000478101A151F822F039430000E341000038
:10432000A1450000A14500009D450000314300006B
:104330000322A2614FF00109A16921F002010129C4
:1043400040F02E81039810F80A2012B1E52A1ED001
:1043500024E0636918070BD5BBF83830ABF836207A
:1043600003F00103ABF83830DBF8003003B11A700A
:10437000A369002B3FF43AAFA38B190704D5384645
:104380000BA90C2202F078FD6FF005082AE1069ACD
:104390000AB1DA1C12D0022B40F00281B9F1000FF1
:1043A0000CD1EB7A180700F1FB80284607990B2205
:1043B00002F0E5FE002840F0F38001E04FF0010933
:1043C0002B7D6A7D1B0403EB0263EA7E03EB022371
:1043D000AA7E1344E360CBF80450EA7AD1060CD4E9
:1043E0000298CBF82C3090F82B10C26801FB032305
:1043F000CBF830304FF00208F4E0A2691AB1A28B7A
:10440000D20600F1EF80029A3B6092F82B10D2683E
:1044100001FB03237B6002233B7296F90030A3B9B2
:104420006369022B23D01D0740F1DC800BF11404DB
:1044300021460BF108000C2202F01EFD0BF12000BA
:1044400021460C2202F018FDCCE00BA839460C22C4
:1044500002F012FD2660B9F1000F01D00423A36120
:1044600004F16C000021FC2202F0FEFCA4E54FF0F8
:104470000308B7E0226B636B9A423FF4FFAE002063
:10448000FFE6531E0B2B1FD8DFE803F01C1A18168B
:104490001412100E0C0A0806AB7F16E02B7F14E0F6
:1044A0002B7E12E0AB7D10E02B7D0EE0AB7C0CE0B0
:1044B0002B7C0AE0AB7B08E06B7A06E0EB7904E04A
:1044C0006B7902E0EB7800E06B78591EC9B2FD29E8
:1044D0003FF6D8AE216B01F1FF3CC4F830C011F8B3
:1044E000011C8B423FF4CEAEA3F1410C5FFA8CFC71
:1044F000BCF1190F02D82033DBB208E0A3F1610C44
:104500005FFA8CFCBCF1190F1CD82031C9B28B4268
:104510003FF4B8AE16E094F86C126B7B99420FD161
:10452000C3E68A420ED30023DDE6069B04936FF0B8
:10453000030309E00020049006E00021049103E059
:10454000134601E04FF0FF33626B22630022A26446
:10455000049A42B9591C06D1039911F80A2002F0B5
:104560003F020592BFE61A1D7FF4BDAE94F86D328E
:104570002BB904F1600039460C2202F07DFC94F85E
:104580006D32142B07D8013384F86D3208E0C14630
:104590006FF00203D0E60023059301E04FF001091C
:1045A00002983946FFF7CFF800283FF4C8ADA36959
:1045B000002B3FF41BAEA38B1C077FF5E5AE073045
:1045C0007FF4DDAE099B58057FF5D9AE7B68029874
:1045D000013B7B603946FFF785FC002814BF80460D
:1045E0006FF0050840460FB0BDE8F08F2DE9F04FA1
:1045F000876893B097F8483007925FEAD27905460A
:104600000C46089303D1AB69022B2EDD37E0084638
:10461000FFF7AAF80028F6D058E240463146FFF7E7
:1046200092F8C31D06D17368013B73604046314662
:10463000FFF758FC002840F0498240467168FEF7B9
:10464000C7FC002840F03E82327AD8F81430039933
:1046500003EB4213059A914280F03E81049921B107
:1046600018460AA9202202F007FC6E6838467168D5
:10467000FEF7AEFC8246002800F0C08122E2AA4686
:10468000D5F808805AF81E3B6E680593184602F06C
:10469000A5FD059B83460344002150460C2203934D
:1046A00002F0E2FB2023AB772F2385F8263002F0BF
:1046B000FBFE009002F0F8FE009B43EA004000F091
:1046C0001F300A900028F2D00AA9042205F1200028
:1046D00002F0D2FB02F0E8FE41F61F7303400AA984
:1046E000022205F124000A9302F0C6FB5046FEF7B1
:1046F00099FC0BF1010B0990CDF808B04FF0010ABD
:10470000029B0D2B07DD029B0AF1010A0D3B5FFAAC
:104710008AFA0293F4E7B9F1000F08D10FFA8AF38D
:104720009A0005EB03139A1A0C2100232FE0636A09
:10473000002BF3D094F840305345EFD304F1200B15
:10474000304659460C2202F097FB94F8403053450E
:1047500058D0CAEB030384F8403094F840303BB1A2
:1047600040463146FEF7EFFF94F84030013BF2E758
:1047700084F840A0584631460C22009302F07CFB9E
:10478000009B40E0013301FB0320406E20B903EBA6
:104790000A0BBBF1140FF5DDB9F1000F02D1CDF812
:1047A00010901FE040467168FEF712FC002840F0B0
:1047B0008981337AD8F814C05B010CEB0301202205
:1047C0000AA88DE8081002F057FB9DE80810E522C2
:1047D0000CF80320B8F8183043F00103A8F818309B
:1047E00001230493BBF1140F04DD304605F154019D
:1047F0000C2204E00C2202FB0B5130466C3102F01B
:104800003BFB01E00023049340467168FEF7E0FBA8
:10481000002840F05781327AD8F814304AF0400A24
:104820004FF0FF0B03EB4213CDF818A04FF0FF320F
:10483000DA4602990D2904D1039991F800A04FF0AE
:10484000000B511C202900F2CA800FF2080E5EF8FE
:1048500021F000BFD94800001B46000003490000BA
:10486000174900001F490000274900002F49000098
:10487000374900003F490000474900004F49000008
:1048800057490000DF490000DF490000DF49000010
:104890005F490000674900006F4900007749000048
:1048A0007F490000874900008F49000097490000B8
:1048B0009F490000A7490000AF490000B749000028
:1048C000DF490000DF490000BF490000C749000080
:1048D000CF490000D749000018460021202200934C
:1048E00002F0C2FA009B069A09991A7002F0BF0200
:1048F000013AD2B206920F22DA72597318461F2279
:1049000097E780F801A0B8F8182042F00102A8F853
:104910001820002264E080F802B0012289E780F8C4
:1049200003A002225CE080F804B0032281E780F853
:1049300005A0042254E080F806B0052279E780F84B
:1049400007A006224CE080F808B0072271E780F843
:1049500009A0082244E080F80AB0092269E780F83B
:104960000EA00A223CE080F80FB00E2261E780F82A
:1049700010A00F2234E080F811B0102259E780F81F
:1049800012A011222CE080F813B0122251E780F817
:1049900014A0132224E080F815B0142249E780F80F
:1049A00016A015221CE080F817B0162241E780F807
:1049B00018A0172214E080F819B0182239E780F8FF
:1049C0001CA019220CE080F81DB01C2231E780F8F1
:1049D0001EA01D2204E080F81FB01E2229E7013A24
:1049E00002990D2903D103990139039124E7DDF8D8
:1049F00008E00EF1010ECDF808E01AE77B6996F8A1
:104A0000088003EB4818404605F11E010B2202F016
:104A100033FA95F8293088F80C30B9F1000F15D128
:104A2000384644B931680122FFF792F80546294615
:104A30004046102207E049464A46FFF789F80546F6
:104A4000294640462022FEF750FD00E05546DFF89B
:104A500084800899726858F82130796938469847F7
:104A60000130F6D03B8B23F001033B83B9F1000FFB
:104A700020D104B3216804F1140020310C2202F08B
:104A8000FBF9E56297F82B20FB6802FB05352563EF
:104A900004F1340004F12C01082202F0EDF9079B27
:104AA000C4F808906360089BC4F80C9084F83E300A
:104AB000022400E000243B8B980706D53846FEF719
:104AC00029FD02E06FF0030000E0204613B0BDE8CE
:104AD000F08F00BFEC86FF1F2DE9F041038B1646D7
:104AE0009A048AB004460D4627D5086806A9FEF741
:104AF0008BFD236A069A87B202EB0308B6B9082237
:104B0000BB0000929BB22046414604AAFEF74EFC31
:104B1000002862D1A92F06A804A98CBF0022012277
:104B2000FEF790FA40F6FF7303903CE020464146C2
:104B3000FEF74EFA002850D1E1E713F4804F0F68DA
:104B4000036A19D003EB172786B92B78022200924B
:104B50002046394606AA5B00FEF728FC00283CD117
:104B6000BDF8183003934FF6FF731CE03946FEF78B
:104B70002FFA002831D1E8E703EBD71776B92B6875
:104B8000042203F07F0300922046394603AA9B00CB
:104B9000FEF70CFC08BB6FF0704304E03946FEF7EB
:104BA00017FAD0B9EBE7039A61688A4201D99A42B1
:104BB00005D3204629680C22FEF7CAFF03902A6815
:104BC000636A9A420CD8039BE2682B6094F82B101E
:104BD00003FB01236B60002004E06FF0030001E0A1
:104BE0006FF006000AB0BDE8F0810000F8B5054698
:104BF0000C46164622B92846FEF7B6FD58B1F8BD58
:104C0000036858680021017741778177C177FEF703
:104C100046FC022EEFD1134F95F83E30616957F8EC
:104C200023302268204698470130F5D0238B286B2B
:104C300023F001032383A368984205D2208B00F060
:104C4000020080B240B9F8BD94F848103246FEF731
:104C500095FA0028F2DAF8BD2046BDE8F840FEF7E4
:104C600059BC00BFEC86FF1FF8B506464B69057FAF
:104C70000C460846B16903EB4515FEF7A9F907464E
:104C8000D8B9B3681A0A2B776A771A0C1B0EAA7761
:104C9000EB7728463946FEF702FC0A4D94F8483077
:104CA000616955F82330B269204698470130F5D044
:104CB000238B23F00103238301E06FF003073846C1
:104CC000F8BD00BFEC86FF1F2DE9F04F8A4EADF511
:104CD000037D0190306810F0020008D08748884BAF
:104CE00042691B6800219847441C00F0F784326831
:104CF000D10700F1ED83834D2B68222B00F2E6846F
:104D0000DFE813F023002300E404E404E404E404F3
:104D1000E404E404E404E404E404E404E404E40453
:104D2000E4043F00490076004E01E4048301BE0123
:104D3000E802F7021F0340035203E404E404E4041E
:104D4000E4047103AC03C303D7036C4C6769C7B9B0
:104D50004FF4007002F070FA4FF4A67323614FF421
:104D60000073694A2385694B60611A60684A644B25
:104D700084F848701A60674A674B1A60674A684B44
:104D80001A605E4B00221A60FEF720FC431C00F004
:104D9000A58410232B60C71C7ED011232B60002814
:104DA00040F09484554A536993F8C2011146E0B12A
:104DB00093F95200462818D093F93600462814D0AB
:104DC00093F8C80193F8C911000400EB016093F84F
:104DD000C71100EB012093F8C61143181360FEF7CA
:104DE000F5FB441C04D100F079BC00230B6001E00A
:104DF000033051D041494B69DC7D9A7D93F80CA07A
:104E000012EB04244FEA0A2A10D193F8264093F8B3
:104E10002720240404EB026493F8252004EB0224E9
:104E200093F824204FF00109144401E04FF00009E9
:104E30001F7DDA7C12EB07270DD193F8227093F8CF
:104E4000232093F821503F0407EB026793F82020BA
:104E500007EB05271744CC6193F810E0D1F80080E8
:104E600081F82AE0587B254A81F82B0093F80FC07F
:104E70009D7B05EB0C25ADB205EB080CBAF5007F68
:104E8000C1F820C005D320B10AFB00F1B1F5004FF5
:104E900006DD244802F044F9FEF77EFB00F016BC64
:104EA0000EFB04F4B2F818E0A2F828A02EF0080EC9
:104EB0001FFA8EFE05EB040A4EF02001CAEB070A2A
:104EC0001183BAFBF0FA4FF6F4718A452CD8B9F188
:104ED000000F29D10121516003F1240193F93A30E7
:104EE000322B0CBF4EF4005E4EF4804E4EF0200E7E
:104EF000A2F818E035E000BFB085FF1F4887FF1F0C
:104F0000B485FF1F9C87FF1F03340000B885FF1F77
:104F1000ED3300001B340000EC86FF1F79340000E5
:104F20004487FF1F02D2000093F831E093F830105D
:104F300093F82F9001EB0E2193F82EE04FEA0E4EDE
:104F40000EEB096E93F82D900EEB092E93F82C9032
:104F500018FA81F1CE44D1621160C2F804E003F185
:104F6000400153687D1B2D1B6444B5FBF0F503FB2A
:104F70001040138B556203F4C0439460D06013B1AA
:104F8000BD4B1F30D86007310B22BC4801F074FFC5
:104F9000BB4B12221A60FEF719FB013000F09E8312
:104FA000B848B94C02F0BCF8B34BB8481A8B42F081
:104FB00080021A8302F0B4F804F596784FF00109E4
:104FC0004FF0030A238FD90714D594F83A708FB99C
:104FD0002568204639463C2201F046FFA4F8389067
:104FE00084F83A7035B125602846A94902F0ECF8FA
:104FF000A4F836A03C344445E4D1336843F00103BF
:1050000033609F4B13221A6060E39B4F7C693E69BB
:1050100000214FF40072204601F026FF022384F89D
:10502000BF310C2384F8C0310B2384F8C2313823FC
:1050300084F8C331F82384F8C431B8233F3E84F8A0
:10504000C5313F2384F8C631330A84F8CB31330CA1
:1050500084F8CC31552384F8FE31AA2384F8FF313B
:105060008C4B84F8CA61360E84F8CD611B6879696F
:10507000384600229847002840F0228215232B60F2
:105080007D4EDFF8249274694FF4FE7200212046B1
:1050900001F0EAFEEB232370582363709023A37082
:1050A0007D49E01C02F090F84FF400733385FF2136
:1050B0000023E37202223F23A176F8212273237694
:1050C0006175318B11F4C04F59D03769A2743C23FC
:1050D0006370012323743B0A237501F400539BB2D0
:1050E000E774083F4BB140F25512B7FBF2F7FE2FC1
:1050F0004FF00602A27309D813E040F20112B7FB89
:10510000F2F7FE2F4FF00802A2730CD90622E274C8
:10511000FF2222755BB11423E374082323750C2747
:1051200006E00C2FF7D8002F08BF012700E0FE276C
:105130000023E3750123A77586F82B30552384F8E7
:10514000FE31AA2384F8FF31082204F136005349C6
:10515000DFF824A101F090FE338BC9F800709A04A7
:1051600045BF322384F83A3007F10803BB1DCAF863
:105170000830B3681F3304F12408F36059E0306944
:105180002377A0F13F03190A84F82110190C227427
:1051900084F822102022190EB3F5022FA27384F88E
:1051A000203084F8231001D8012310E0B3F1807F70
:1051B00001D808230BE0B3F1007F01D8102306E0EB
:1051C000B3F1806F02D886F82B2002E0402386F8E6
:1051D0002B3096F82B10012202EBC111A0F16003D5
:1051E0000B44B3FBF1F3190A84F82510190CC9F824
:1051F000003084F8243084F82610190E5B005F33E9
:1052000084F8271084F830200221062284F82C101C
:1052100084F83220B360082204F15200204901F0E2
:105220002BFE96F82B20B368A3EB420304F1400851
:10523000F36096F82B306373802388F800302923BD
:1052400088F8023002F030F988F8030002F02CF9F7
:1052500088F8040002F028F988F8050002F024F923
:1052600088F8060096F9493003BB08F107000D499C
:105270000B2201F001FE2BE04887FF1F9187FF1FE3
:105280009C87FF1F0FD20000BC85FF1F09C00000D4
:105290001ED20000EC86FF1F22D200002BD200009D
:1052A00034D200003DD20000A487FF1F002320213C
:1052B000F21808EB030092F84920C2712AB908EBF2
:1052C000030201330B2BD171F9D101330A2BEFDD2E
:1052D00016232B609648038B03F4C0433BB9954BD0
:1052E00041691B683F229847002840F0E980172356
:1052F0002B608F4C8F4B228B1B68616902F4C0427C
:105300002046002A0CBF452200229847064608B1D5
:10531000461CD6E0676931464FF40072384601F00A
:10532000A3FD04F149010B22384601F0A5FD082335
:10533000FB7238460121FEF7B2F87F4B1E6018233E
:105340002B607D4E7A4C336894F82B20934212D216
:10535000A268784920460F6861691A44B847014637
:10536000002835D13368606901334FF4007233602F
:1053700001F07AFD96E119232B60002333606F4B17
:1053800001221A706A4B1A8B5869530401D56C4973
:1053900002E0970402D56B49042201E06A490C221D
:1053A00001F06AFD1A232B606149634C0B8B226864
:1053B00049699E0454BF5F3206225D4E13F4804F4C
:1053C0005C4B30461B6818BF08229847014608B15D
:1053D000013176E070690C2201F046FD236801334B
:1053E00023601F232B605548584C534B0178246889
:1053F0001A684C43A2421C4616D3012903D8013136
:105400000170192351E04A48018BCC040AD511F4EC
:10541000C04F21F480540CBF5F3208321A600483FD
:10542000202342E0212340E0414B198B01F4C0418D
:1054300009B95F3200E008323E493D480E685969BB
:10544000B04700283CD12368013313F0FF0F2360DD
:1054500040F028813E4801F063FE23E1364C344899
:10546000226803699A4202D321232B600DE0314B5D
:1054700041691B68984718BB2368013313F0FF0F7D
:10548000236040F00F813348E5E7294C238B03F478
:10549000C04363B1304801F043FE238B98044CBFF6
:1054A0002E482F4801F03CFE0F232B60FAE0222308
:1054B0002B60204B1E481B6841694622984728B143
:1054C000013000F00B8132232B60FFE02548E9E733
:1054D000D10640F1FB80164B234FDE69186A39680C
:1054E0000644B14280F0E380761ADFF88490DFF85A
:1054F00084800A2E28BF0A26002E00F0D3801A4A84
:105500000B4C11684B1C1360204602AAD9F80030DE
:105510009847002840F0C480238B144D13F4804F2B
:1055200035D02B6802AF3A5832BB023329E000BFB6
:105530004887FF1FEC86FF1FF086FF1FA185FF1F16
:10554000D4D2000038D00000D8D20000A487FF1FBA
:1055500049D200004BD200004DD2000061D20000C1
:1055600065D2000069D20000A485FF1FAC85FF1F33
:10557000B485FF1FA087FF1F91B209B1120C00D1A3
:1055800001330430B0F5007FCCD12B6088E003F408
:1055900000539BB20BB9296879E0524B1868236A13
:1055A0000138C01A0323B0FBF3F203FB120018B159
:1055B00001280CBF02200120DFF840C12A68D8F87A
:1055C0000030DCF800E000247F2C5AD802AF01281C
:1055D00057F8241013D0022832D0C1F30B0000B9C1
:1055E0000132012B02D10023184634E03E48084026
:1055F00000B90132023BF6D08E4601203FE001F0B7
:105600000F0B0EF07F4A5BEA0A0A08BF0132012B3A
:1056100020D04FF6F07A01EA0A0ABAF1000F00D161
:105620000132022B16D0DFF8D8A001EA0A0ABAF13B
:10563000000F00D10132033B0CD08E4602201EE049
:105640005FFA81FB0EF0704A5BEA0A0A08BF01327A
:10565000012B03D100234FF4007410E0DFF8A4A065
:1056600001EA0A0ABAF1000F00D10132022BF1D08F
:10567000090D090501B90132033BEBD000200134CB
:10568000A2E71A482A600360CCF800E008E002AF05
:10569000FA5802B901310433B3F5007FF7D129601C
:1056A000013E29E74D20042101F07EFF0EE0104964
:1056B000104C22F010020A600F4A94F900001268A0
:1056C000BF211A6301F046FD00232370019B02A94C
:1056D000987B052201F004FA0028F7D10DF5037D2F
:1056E000BDE8F08FA485FF1F00F0FF00A087FF1F1B
:1056F000B085FF1FA885FF1FAC85FF1FE886FF1F31
:105700000000FF0F00FF0F002DE9F041036893F840
:105710003A70164B0546542404FB07342046696949
:10572000FDF756FC0646C8B92B7E62695B01D018AE
:10573000D35CE52B15D10E49DFF838800B2201F040
:105740009BFB58F8273061696A6920469847013009
:10575000F7D0238B23F00103238304E06FF00306CB
:1057600001E06FF009063046BDE8F0814887FF1F71
:105770007AD20000EC86FF1F2DE9F04F81469FB0E2
:1057800059F8043B93F83A20A44B4FF0540A0AFB13
:10579000023A00F11003039390F82A30019300239A
:1057A0000093019B03F0020780460E466424FFB27B
:1057B0005046D8F80810FDF70BFC0546002840F0CD
:1057C000DE8098F80C20DAF8141052018B18895CEE
:1057D00011B1E52906D009E0DB7A1B0700F1B180A1
:1057E000012516E1002F00F0AB8002E0002F40F011
:1057F000A880D87A00F03F0EBEF10F0F224654D198
:10580000002C52D011F0400F13D0E52901D1642CA7
:105810000FD1997F0139C9B2FD2905D8621E1EA991
:105820001144002001F8640C93F80DE0CDF800E07D
:1058300004E0597BDDF800E0714536D10D2A05DC26
:1058400005A8002101F010FB00242CE01EA9987F80
:105850001144A2F10D0401F8650C187F01F8660CE3
:10586000187E01F8670C987D01F8680C187D01F826
:10587000690C987C01F86A0C187C01F86B0C987B19
:1058800001F86C0C587A01F86D0CD87901F86E0C9F
:10589000587901F86F0CD8781EAA01F8700C2244D0
:1058A0005B7802F8643CE4B24BE0820706D50199CC
:1058B00001F0200202F0FF0B002A4DD000F0080298
:1058C00002F0FF00002A3CD193F80CE006F1090237
:1058D0000EF0080C02925FFA8CFC195C202951D161
:1058E000197A20290AD02E210EF0100E11700820EE
:1058F00001325FFA8EFE195C202958D10021117007
:10590000DA7A32729A7FD97F120402EB0162597FF0
:1059100002EB0122197F0A443260597E1A7E02EBA3
:105920000122B280D97D9A7D642C02EB0122F280A3
:105930004FD04FB91846FDF775FB009B984203D036
:1059400064244FF0000B07E005A92144029801F000
:105950003BFC64244FF0010B50464946FDF7F3FE33
:10596000073007D1BBF1010F14BF6FF006056FF0D0
:105970000F054EE0BBF1000F3FF41AAF49E06FF0A6
:10598000030546E0052908BFE521BCF1000F08D05A
:10599000A1F1410B5FFA8BFBBBF1190F9CBF2031CA
:1059A000C9B20130082802F8011B96D198E7BEF170
:1059B000000F08D0A1F1410C5FFA8CFCBCF1190F6B
:1059C0009CBF2031C9B201300B2802F8011B92D1D3
:1059D00094E7002FBED07E23737201223346997A5A
:1059E000080644BF80399972997A29B903984946C3
:1059F0000C2201F041FAADE748B22028D8BF21318E
:105A000002F10102D8BF99720A2A03F10103E6D11B
:105A1000ECE728461FB0BDE8F08F00BF4887FF1FA6
:105A20002DE9F04F00220F684A810C46097DA7B08E
:105A300011F0010F0CBF2C232F2301930DF1310323
:105A400080F82A100546E2810093E189A2899142FB
:105A500080F0518105F1040841460C2202A801F0B2
:105A60000BFA28460AA9FFF787FE064628B110F16F
:105A7000100F02D06FF00E003EE1B4F80A90019BC7
:105A80000098994401F0AAFB22894844904207DD1E
:105A9000404602A90C2201F0EFF96FF00D002BE156
:105AA000BDF82C90217D9DF83020BDF82E806275C8
:105AB00009F01F0BC9F3431A11F0010F4FEA5929DE
:105AC00009F2BC7907F1010177D0D00607D412F0B2
:105AD000010F0CBF4FF4D2724FF4927201E040F20A
:105AE000ED324FF00B0864204FF02D0EB8F1010895
:105AF00013D0930548BF01F8010C40B258BF01F81C
:105B000001EC722804D077280CBF7820722000E0C6
:105B10007720520092B20131E8E707F10A00784994
:105B200001F052FB9DF83030DF0602460BD52B68A2
:105B3000744993F83A30542000FB031393F82B1068
:105B4000188D484300E00A98414601F091F8034659
:105B50002022AAF1020A01301A70BAF10A0F07D8FE
:105B6000DFE80AF0080A0C0E10121416181A1C00AE
:105B7000654914E0654912E0654910E065490EE0A9
:105B800065490CE065490AE0654908E0654906E0B9
:105B9000654904E0654902E0654900E0654901F0B6
:105BA00013FB12210246584601F062F8102102460A
:105BB000484601F05DF8074677E0D0074CBF522217
:105BC0002D223A709DF8303013F0020F14BF482296
:105BD0002D220A709DF8302012F0040F14BF5320BC
:105BE0002D2048704B1C9DF8301011F0200F14BF71
:105BF00041212D215A1C597001325846122101F0C1
:105C000037F84FF02E0B024680F800B00221013227
:105C1000504601F02DF8024680F800B000214846B9
:105C2000013201F025F84FF02009024680F800907B
:105C3000122101324FEAD82001F01AF83A23024625
:105C400003700132C8F34510022101F011F89DF8EC
:105C50003030DA0607460AD5237DDB0703D4364900
:105C600001F0B2FA0746238A013323821DE00DF1C9
:105C7000140A52460A98102100F0FAFFC0EB0A00FD
:105C8000113003463A4613F1FF3302D302F8019B69
:105C9000F9E73844514601F097FA638A62680133A4
:105CA00063820A9B13440746636007F101092023BE
:105CB0003B704846009901F087FA227DC9EB000944
:105CC0001107074684F8169006D402460D2102F803
:105CD000021B0A21417017462268BA1A6281E289C2
:105CE0000132E281227D120744BF00223A70103651
:105CF0007FF4ABAEBEE6002027B0BDE8F08F00BF5A
:105D000086D200004887FF1F92D2000096D2000082
:105D10009AD200009ED20000A2D20000A6D20000BB
:105D2000AAD20000AED20000B2D20000B6D200006B
:105D3000BAD20000BED20000C2D200000F4B70B534
:105D40003C220E46002402FB0435298F89B9012329
:105D50002B8785F83A002EB1F01880B201F06CFA6A
:105D6000286000E02E60054B3C2000FB0430868656
:105D700070BD0134052CE6D1002070BDBC85FF1F2D
:105D800030B5ADF51D7D05460C464FF41C72002163
:105D9000684601F069F868462946224600F00AF88C
:105DA000049B23B1684621460022FEF7E5F80DF575
:105DB0001D7D30BD2DE9F843144692F83A308E4AE5
:105DC0000E46542101FB03230546188B020640F1C1
:105DD000078100226A61002E7BD0E78E96F90010C1
:105DE0002E2922D196F901102E291ED1216829B918
:105DF000268F46F0400626870E4616E0032F40F217
:105E0000F3800AB1013FBFB211F907C0BCF15C0FCA
:105E100005D196F90210013229B9023607E0BCF12A
:105E20002F0FEFD1F5E70336D8E7002A51D0228FA4
:105E3000032F42F040012187A9833BD92368002228
:105E400013F80790DA55238F206823F01003238777
:105E500003302146FFF794FF804618B1236803F80A
:105E60000790C1E096F90030BBB1AB8B23F0C003C3
:105E700043F08003238730462146FFF781FF18B1A6
:105E8000A5F81C80804608E0AB8BDB0505D52068B3
:105E9000711E384401F098F903E0AB8BD80503D5A7
:105EA000E7860520BDE8F883236803F8079040469D
:105EB000BDE8F883D1050CD523680022DA700323EE
:105EC000E38604F1200004F108010C2200F0D4FF65
:105ED000E7E7218F2E6021F4FC72A983228736B177
:105EE000327822B152B20A2A01D00D2A01D1012200
:105EF00010E05C2A01D02F2A0DD141F02001A983A6
:105F0000727822B152B25C2A01D02F2A01D1042228
:105F100000E002226A61AA8B12F0020F04F120064F
:105F20002DD15A68D968EA60012A626193F82B3052
:105F300006D810F4C04F03D01F390B44A36102E010
:105F400002FB0312A261002304F1140723773946F0
:105F50000C2204F1080000F08FFF304639460C2275
:105F600000F08AFF072323876B69206843F008034A
:105F70006B6120B1214901F027F90323E386AB8B44
:105F800013F0E40F1DD05A0603D5304604F1080182
:105F900012E01F0613D46B6913F0060F304609D0C8
:105FA00004F108010C2200F067FF6869042806D19B
:105FB000BDE8F88304F114010C2200F05DFF6E606F
:105FC00006E004F11401696030460C2200F054FF31
:105FD0006B6913F005000BD101222A61BDE8F8833B
:105FE0006FF00100BDE8F8836FF00200BDE8F883B0
:105FF0000020BDE8F88300BF4887FF1F1ED20000C5
:106000002DE9F3470023838743680446884690F8C8
:106010003E10D80715464BD5A268E368D31A01D1C4
:10602000002047E09D4288BF9DB2244BDFF890904E
:10603000542707FB013704F1340A002DF0D0E36840
:10604000C3F308039BB2C3F50076B6B2B54238BFBE
:106050002E4613B9B6F5007F1AD000963846A16BCC
:106060004246FDF7A3F980B9A28FE3683244A287C4
:106070003A8D3344B3FBF2F1AD1BE36002FB113305
:10608000ADB2B044002BD8D10BE06FF0030011E0AB
:1060900094F83E30A16B59F8233038464246984771
:1060A000E1E738465146FDF7D5FA0028C5D001E0B2
:1060B0006FF0080002B0BDE8F08700BF4887FF1FFF
:1060C000B485FF1F38B50C46096851B1FFF758FE7B
:1060D000051E09DB2168201D20310C2200F0CCFEBA
:1060E00002E06FF0100038BD284638BDF0B5254BF2
:1060F00091F83E20542606FB0236ADF5217D358B06
:1061000005F01005ADB207460C46002D31D14B68A5
:1061100013F0240F30D029464FF41C7204A800F06D
:10612000A3FE21680C22203101A800F0A5FE04A8DE
:1061300039462268FFF73EFE089BFBB12A4604A8B9
:106140002168FDF719FF851D18D12168069619A849
:1061500020310C2200F090FE206801A90C22203092
:1061600000F08AFE04A821464FF00042FEF73EFAF6
:1061700004E06FF0120001E06FF009000DF5217DE1
:10618000F0BD00BF4887FF1F38B54368DB060446F3
:1061900005D503690C4A02EBC30300225A706068FC
:1061A00010F0005509D094F83E20084B54212046A9
:1061B00001FB0231FEF758FD05462046002144222E
:1061C00000F052FE284638BDF486FF1F4887FF1FA7
:1061D0002DE9F04F554B90F83E804FF0540B0BFBE0
:1061E000083B00238387BBF818300446D806ADF57A
:1061F000017D0F46154600F18C806368990740F1D8
:106200008B80DFF834A1002D59D0E368C3F3080672
:10621000B6B236B9B5F5007F0ED2A268D31A9D4248
:106220000AD2434A94F83E30A16B52F823305846C4
:106230006A46984730B172E0684600214FF4007218
:1062400000F012FEC6F5007C6545CCBF1FFA8CF944
:10625000A94600A8304439464A4600F00DFE5AF8D7
:106260002830A26B5846694698470130F7D0E3685A
:10627000A2684B44934288BFA360E360A38F4E445F
:106280004B44C9EB0505B6F5007F4F44A387ADB27B
:10629000B9DBA26BDBF808300132A263D21A9BF89B
:1062A0002B30B2FBF3F103FB1122002AABD158468D
:1062B00004F13401FEF710FC0028A4D031E0A38FD4
:1062C0002BB16368DA0307D543F000536360002500
:1062D000184F04F12C0806E020465946FEF7C4FC8E
:1062E0000028F4D01DE07E1973786BB171684046C8
:1062F0002C31082200F043FF30B97368A268D968D6
:106300009A608A4238BFDA600835502DEBD1002000
:1063100007E06FF0120004E06FF0090001E06FF099
:1063200003000DF5017DBDE8F08F00BF4887FF1F1A
:10633000B485FF1FF486FF1FEC86FF1F0B8F43F40D
:10634000807370B50B8706460C46CD8EFFF718FD9F
:10635000031D092B2BD8DFE803F0352A352A082A3C
:106360002A05242D0325E5860136236813B396F903
:10637000002082B1032D02D95C225A5500E001D0E1
:106380000135ADB220683146284400F01DFF236876
:10639000C01AE0860EE0E586022D08BF03255A5597
:1063A00008E00323E38623680022DA7002E06FF03E
:1063B000020070BD04F1140004F120010C2200F071
:1063C0005BFD002070BD00002DE9F0472D4B0C4611
:1063D00090F83E105426012A06FB01360546C36894
:1063E00005D0022A10D0002A18BF002412E0002C89
:1063F00003DA62429A420CD804E08268D21A9442CC
:1064000028BF14461C4405E08268944201D2141B44
:1064100000E000249C4231D005F1340808D2404607
:1064200005F12C01082200F027FD0023EB6003E0BA
:10643000AB689C4228BF1C46B6F82890EF68C9F1AB
:10644000000A0AEA070704EA0A0A574515D2AA6BA6
:10645000B3680132AA63D21A96F82B30B2FBF3F17B
:1064600003FB11234F44002BEFD13046414601225C
:10647000FEF732FB0028E8D001E0EC600020BDE828
:10648000F08700BF4887FF1F2DE9F0410C46ADF5AE
:106490001C7D0746154600214FF41C72684600F02B
:1064A000E3FC23681A8F15F0200F14BF42F01C0282
:1064B00042F00C021A87684639462268FFF77AFCD8
:1064C000049B002B00F0AC8015F4804805D0BDF88B
:1064D0001C3043F01003ADF81C30684621682A4692
:1064E000FDF74AFD0228064659D1A046264658F82F
:1064F0002C1B0C22203104F1140000F0BDFC56F8D6
:10650000341B08222C31404600F0B6FC216830468E
:106510002C31082200F0B0FC22685368D97ACE07EB
:1065200048BF25F006056560987FD97F000400EB21
:106530000160597F00EB0120197F00264318A360FA
:10654000E66092F83A3011A984F83E3004F1200058
:106550000C2200F091FC9DF86E3215F4007184F865
:1065600040300BD094F83E202F4B542101FB0231D8
:1065700020460222FEF73AFBA66007E0280505D573
:1065800020460222FFF720FF002849D16A0442D5A5
:106590000120394622466B46FDF718F93BE06B05B2
:1065A00015D5871D39D121681F4A91F83A305420FA
:1065B00000FB0323203168440C22029300F05CFCB2
:1065C0006846214625F00042FEF710F828E020BB7F
:1065D00021680C22203104F1140000F04DFC45F03C
:1065E00080052368656093F83A3004F1200084F850
:1065F0003E3011A90C2200F03FFC9DF86E3284F869
:106600004030B8F1000F0AD03046394622466B467A
:10661000FDF7DCF801E0022002E0304600E04046F1
:106620000DF51C7DBDE8F0814887FF1F2DE9F84F6F
:106630000C461E460A60002A53D092F83A302E4982
:10664000542505FB03131B8BDD0602D516F0260F20
:106650004AD1F1063FD5294B4FF0000813F8077CCB
:10666000A3F108096FBB214626F01003FFF7DEFFF8
:10667000022805463BD1DFF888A004F12C0B0AEB79
:1066800007035A7872B90837502FF8D1C9F8044077
:1066900094F83F3089F80130666089F80060C4F8EA
:1066A000108026E0596858462C31082200F067FD1A
:1066B0000028E8D117F80A301B07E4D56FF00A0567
:1066C00017E008F10108B8F10A0F03F10803C5D17A
:1066D0006FF015050DE021463246BDE8F84FFFF793
:1066E000D3BE6FF00B0504E06FF0120501E06FF010
:1066F00005052846BDE8F88F4887FF1FFC86FF1F69
:10670000F486FF1F2DE9F0412C4B91F83A2092B00E
:1067100012AC542606FB02360B8F44F8441D43F09E
:1067200020030D460B87042221468046FFF7ACFE6E
:1067300048BB04F1140704F12C003946082200F08C
:106740009BFB30460799FCF743FC58BB9DF8202083
:10675000736952019B5C43B1E52B26D13046394623
:10676000FCF7F1FFC31DECD124E02B8F43F0300385
:1067700004222B8740462146FFF786FE0246C8B911
:10678000019B5B6807E0022814D1019B5B68DA7A01
:1067900012F001020CD1E521197020463146FEF7B6
:1067A00025FA07E06FF0030004E04FF0FF3001E04E
:1067B0006FF0090012B0BDE8F08100BF4887FF1FED
:1067C000F0B5204B91F83A20542606FB0236ADF581
:1067D0001D7D07460C46684600214FF41C7200F0F0
:1067E00043FB358B05F01005ADB22DBB238F04950F
:1067F00043F008032387684639462246FFF7DAFA52
:10680000049BDBB14FF4806268462146FDF7B4FB80
:10681000821D04D0002808BF6FF011000EE004F1C3
:10682000200115A80C22029600F026FB6846294696
:106830002A46FDF7DBFE01E06FF012000DF51D7D2D
:10684000F0BD00BF4887FF1FF8B5D30704D4234B22
:1068500053F82030322B3DD1214E542303FB0063EB
:106860001D8B05F01004A4B28CBB1E4F05F0400533
:10687000ADB247F8204012F0040F45F008041C8325
:10688000164C02D045F4804503E0970706D545F441
:10689000005545F008051D83152300E0142344F836
:1068A0002030140706D5542303FB00631A8B42F4EF
:1068B00080521A83542303FB00600B22493000F0FE
:1068C000DBFA4D20042100F06FFE0020F8BD6FF0D0
:1068D0001200F8BD6FF00100F8BD00BF9C87FF1FDC
:1068E0004887FF1FB085FF1F8268C3689A4270B552
:1068F000044601D8002070BD43689A0735D590F84A
:106900003E201D4B067FA169542505FB0235284614
:106910006B6903EB4616FCF75BFB014640BBE36883
:106920001A0AA360337772771A0C1B0EB277F377CB
:106930003046FCF7B4FD114E94F83E30696956F8C4
:106940002330A269284698470130F5D02B8BA06BE5
:1069500023F001032B83AB689842CBD395F8481002
:106960000222BDE87040FCF709BC6FF0090070BD61
:106970006FF0030070BD00BF4887FF1FEC86FF1F4C
:1069800070B5114B1C56E4B9104A114E42F8204024
:10699000104A1954542505FB00220421556A46F873
:1069A0002050156A0C4A42F820500C4A52F82050E8
:1069B00045F0100542F820504D2000F0F5FD20462E
:1069C00070BD6FF0160070BDA885FF1FAC85FF1F5E
:1069D000A087FF1F4887FF1FA485FF1FB085FF1FEB
:1069E00038B50B465424094933B904FB001011464D
:1069F000BDE83840FCF7ECBA054D55F8205004FBD3
:106A0000001011461A46A84738BD00BF4887FF1F2F
:106A1000B485FF1F2DE9F84FDFF84090DFF840B054
:106A20004FF0540808FB00F882460E46174609EB63
:106A3000080431465BF82A3020463A469847411C04
:106A40000546F6D059F808309F4204D16069228D7E
:106A5000314600F011FA2846BDE8F88F4887FF1F3D
:106A6000EC86FF1F024B542202FB0030704700BF30
:106A70004887FF1F37B50138C5B2054804682B01A8
:106A8000E018007B0095E4580323A04703B030BD15
:106A9000AC87FF1F08B5044B1870000100F0CCFB59
:106AA000024B186008BD00BFA887FF1FAC87FF1FFF
:106AB000FF2873B50E460DD008490138C5B20C68E1
:106AC0002B01E118087B0095E45811460223324659
:106AD000A04700E0002002B070BD00BFAC87FF1FE0
:106AE00037B50138C5B2054804682B01E018007BB2
:106AF0000095E4580423A04703B030BDAC87FF1FC6
:106B0000074A13B501381268C1B20B01D018007BD7
:106B100000910021D4580A460523A04702B010BDB9
:106B2000AC87FF1F37B50A4606490138C5B20C6865
:106B30002B01E118087B0095E45800210623A047AB
:106B400003B030BDAC87FF1F30B50C4B1D780C4B2C
:106B50001B6800221033AA420ED053F8104C844216
:106B600002F1010205D113F8044C8C4201D1D0B2DC
:106B700030BDD2B21033EEE7002030BDA887FF1F32
:106B8000AC87FF1F2DE9F74F054610468B4692460E
:106B90001C46FFF7D9FF014608B1002040E0FFF78F
:106BA000D3FF06460028F8D01F4B00F18058D3F8D9
:106BB00000902B8808F1FF384FEA081809EB080706
:106BC000ABB1204600F038FB0346786078B12A88E4
:106BD00010468DE80C0000F02FFB9DE80C0000280B
:106BE000DBD01860586098601044D860DA826B88F7
:106BF0008BB1204600F020FB0446B86058B16D8888
:106C0000284600F019FB0028C7D020606060A06013
:106C10002844E060E58249F808A0304687F80CB0C7
:106C200003B0BDE8F08F00BFAC87FF1F032807B596
:106C300006D0052812D0A8B9104600F081FE12E057
:106C40001389ADF804300023ADF806301368074A05
:106C5000197801A81823FFF795FF04E0104601F00A
:106C6000ABFB00E0002003B05DF804FBF96E000010
:106C70002DE9F043CE0604D52023137001F0FB016B
:106C80000132CD0705D5002803DA2D2313704042C9
:106C9000013201F0020701F0040C2D4B00240A26FA
:106CA000FFB25FFA8CFC4FF0200810B90A203025A3
:106CB00026E0302583420ED9B3FBF6F314B9012B3D
:106CC000F8D10FB1157004E0BCF1000FF2D082F8DA
:106CD00000800132EEE7B0FBF3F505F13009EDB2CB
:106CE000002B18BF012482F8009003FB150001322D
:106CF000B3FBF6F3D9E734B102F8015BB3FBF0F371
:106D0000002BF8D18CB911F0040F134602F10100E9
:106D100003D002462020187007E08C0702D50246F7
:106D2000302018703023137001320B0706D513463C
:106D30000D2003F8020B0A2050701A4601F04001A2
:106D400001F0FF0301B913701046BDE8F08300BFE6
:106D500000CA9A3BCB062DE9F04102D520231370DF
:106D600001320F0606D51346302403F8024B78246F
:106D700054701A4601F0400601F0200801F0080C9A
:106D800001F00701042928BF04214900F6B25FFA87
:106D900088F85FFA8CFC17460B46013BDBB2FF2BF1
:106DA00014D09D0020FA05F505F00F0505F130041B
:106DB000392C08D9B8F1000F02D005F1370402E0F0
:106DC00005F15704E4B207F8014BE6E75018BCF1AF
:106DD000000F04D00D2353540A234370023006B928
:106DE0000670BDE8F0810246013092F90030202B98
:106DF000F9D0013A002012F8013F59B22F290EDDD7
:106E0000D9B2A1F13003DBB2092B88BFA1F157033E
:106E10004FEA001088BF03F00F031843EBE77047F9
:106E200010B50022014610F8013BA3F13004E4B292
:106E3000092C04D9B3B12D2B08BF0122F2E7013987
:106E4000002011F8013FA3F13004E4B2092C06D868
:106E50005BB2303B03EB400303EBC000F1E712B140
:106E6000404210BD184610BD02440346934202D072
:106E700003F8011BFAE7704710B50023934203D0D3
:106E8000CC5CC4540133F9E710BD2DE9F843058A01
:106E90004768AA4238BF154604460E463DB3C3684C
:106EA0007A199A42426015D3C7EB03081FFA88F893
:106EB0000368C8EB05094B44436002F0C1F88EB18A
:106EC000394642463046FFF7D7FF06EB08002168F7
:106ED0004A4605E002F0B4F826B1304639462A4663
:106EE000FFF7CAFF02F0A4F8238A5B1B238202F09B
:106EF000A7F82846BDE8F883F8B51D460F461646A4
:106F00009DF8184002F094F8052D0ED0062D13D0F0
:106F1000042D1CD1104B1B6803EB04143946606828
:106F20003246BDE8F840FFF7B0BF0B4B1B6803EBE0
:106F3000041463681C8A0BE0074B1B6803EB041402
:106F400063681A6800249A605A601C8200E000247A
:106F500002F076F82046F8BDAC87FF1F2DE9F0411E
:106F6000044615460F4602F063F8218A628AE38AD6
:106F700088182844984202DD5D1AAD1AADB22A4441
:106F8000D4F808806282E26808EB05069642A660A3
:106F900006D3F31A2668A3609E1BAE1BB6B200E0B0
:106FA0002E4602F04DF8404639463246FFF764FF60
:106FB000B54204D02068B919AA1BFFF75DFF02F0A3
:106FC00037F8638AA28AAB4206D1238A2B441A443B
:106FD00000232282A38202E02A44A2825B1B6382F6
:106FE00002F02EF82846BDE8F0810000F8B504460E
:106FF0000D46002937D1027843789A4262D102F0D7
:1070000017F8A178314B32481970FFF79DFD3149CF
:107010000646087010B902F013F855E02E4B1868B8
:1070200000EB0616207956F80C3C1A8A561D0644C9
:10703000D88A864203DD0D7002F002F842E0063283
:107040001A8228469A68511C9960215C1170DA688E
:107050009968914228BF1A6800F1010028BF9A6020
:107060000628EFD1F8BD1B4B1E7866B9027843782D
:107070009A4229D1877816483946FFF765FD0646BA
:1070800010B3FFB205E0114A177800221A7001F020
:10709000D7FF114B1868E37800EB0616032B56F860
:1070A0000C0C04D1C28A038AD01A80B2F8BD2146E2
:1070B0002A46FFF753FF0421044678B200F074FA21
:1070C0002046F8BD2846F8BD3046F8BDAA87FF1F08
:1070D000F96E0000A987FF1FAC87FF1F30B528B9E4
:1070E0000846BDE830401146FFF780BFFF2803D0B7
:1070F000BDE83040FFF7BEBC002030BD10B50346F0
:107100000446E21A14F8010B92B20028F9D12AB110
:107110000846BDE810401946FFF7E0BF104610BD15
:10712000014B1978FFF7EABF0D82FF1F1FB56A46B2
:10713000FFF79EFD6846FFF7F3FF05B05DF804FB1F
:107140001FB56A46FFF706FE6846FFF7E9FF05B080
:107150005DF804FB07B5002370B18DF800308DF8A1
:1071600001308DF8020001238DF8041068460521D6
:107170008DF80330FFF73AFF03B05DF804FB30B53C
:107180000023934208D0C45C0133CD1815F8015C8C
:10719000A542F6D0012030BD002030BD013810F8E6
:1071A000013F3BB111F9012B5BB29342F7D008DDEF
:1071B0000120704791F90000003818BF6FF00000FF
:1071C00070474FF0FF3070470A78034603F8012BF1
:1071D00011F9012B0AB11846F6E770470023C25691
:1071E0000AB10133FBE71846704700000E4B13B598
:1071F00000221A800D4B0E4A19600E4B147819604C
:107200001A460378A34202D063B10430F9E74388F9
:10721000194411600DF107035522994202D801F873
:10722000012BFAE702B010BDB487FF1FB087FF1F24
:107230001B82FF1FB887FF1FF8B5104A104B11685B
:107240001C880C4414F0030F17460E4A1CBF24F090
:107250000304043412681E4623189A4205460AD9CC
:107260002A4620460021FFF7FFFD3B68E31A1D4434
:1072700035802046F8BD0020F8BD00BFB087FF1F55
:10728000B487FF1FB887FF1FF8B5104A104B05469B
:107290001C8810680444481E044217461E4602D04B
:1072A0004B421C400C440B4A126863199A420AD99B
:1072B0002A4620460021FFF7D7FD3B68E31A1D440C
:1072C00035802046F8BD0020F8BD00BFB087FF1F05
:1072D000B487FF1FB887FF1F044B1A681346981A1C
:1072E00013F8011F552980B2F9D07047B887FF1FE6
:1072F000034B1868034B1B68C01A80B2704700BF6D
:10730000B887FF1FB087FF1F044B1868044B1B682A
:10731000C01A044B1B88C01A80B27047B887FF1F81
:10732000B087FF1FB487FF1F2DE9F047594F5A4E12
:1073300000233B603360594B90461A7882460C78A4
:10734000002C4DD064B2944241D10B4693F90140D8
:107350005D1AEDB203F101090CB14B46F6E71420BA
:1073600068430430FFF768FF03463060E843484451
:10737000A14642784AB3514652B2D1F800E0BEF17C
:10738000000F20D09EF900C094451AD14A68C3F876
:1073900000E05A600A891A810AB10134E4B2B1F8F6
:1073A0000AE08A89A3F80AE09A81897BD973BEF141
:1073B000000F00D11AB109F101095FFA89F91433FC
:1073C00001E01031D9E70130D3E71A600AE04B1C25
:1073D0001946013391F900000028F9D11946AEE7AA
:1073E000A14625463368002B48D0B9F1000F2FD0B5
:1073F0000C2000FB09F0043080B2FFF71DFF264B84
:1074000038601B684FF0000E4FF0010C4FF6FF7A0A
:107410001A68AAB15A8932B1524508BFA3F80AE0E6
:107420005A89426002E0998909B1416001214268AC
:107430000AB180F809C009B140F80C3B1433E7E702
:107440000FFA89F94FEA091300EB8900C01A386076
:1074500004EB0800C0B2FFF71DFB7CB13468FF26C7
:1074600023685BB123893BB1032001212246FFF74A
:10747000DDFBA07300B9A6731434F1E7084801F0EE
:10748000C7FD084B00221A6002F0E4FA2846BDE866
:10749000F08700BFC887FF1FBC87FF1F1B82FF1F2D
:1074A000C087FF1FC487FF1F064A108840F30003F0
:1074B00023F4974323F07F0383EA500080B21080C7
:1074C000704700BFC087FF1F1F4B73B51C680025A6
:1074D000143454F8143CA4F114069BB314F8053C7E
:1074E00013F00D0F2CD001F0A3FD34F8083C1BB9AC
:1074F00014F8053CDB071DD414F8043C9BB18DF84F
:1075000000508DF8015054F8142C12788DF8035067
:107510008DF802200020694605228DF80430FFF71F
:10752000DDFD04F8045C14F8053C13F00A0308BF01
:1075300004F8053C01F084FD54F8103C30469847AF
:107540001434C6E702B070BDBC87FF1F38B50D4BC1
:107550001C68054601F06CFD04F1140353F8142C6B
:1075600072B113F8051C11F00D0F07D092F900202D
:10757000AA4203D001F064FD012038BD1433EDE7C9
:10758000104638BDBC87FF1F064B1B681A683AB10E
:1075900092F90020824201D1D87B70471433F5E77D
:1075A00080207047BC87FF1F38B5154B1C682368C7
:1075B00023B393F9003083421ED1B1B9114B1D683A
:1075C0009DB12B688BB19C420DD101F031FDA38997
:1075D0001BB10D4A126813446B600023E373BDE8CE
:1075E000384001F02DBD0C35EBE7480702D5E37BB1
:1075F0001A0703D4E17338BD1434D8E738BD00BF8F
:10760000BC87FF1FC887FF1FC487FF1FF8B5184B33
:107610001C680D4617464CB3164B1E6833682BB3D7
:1076200093F9003083421FD12368E3B19E4218D101
:1076300001F0FEFCF37B23F00203F37327721FB902
:10764000B58125B9657208E0002D08BF01250A4BF8
:107650001B681D44012365606372BDE8F84001F0BA
:10766000EFBC0C34E0E7F8BD1436D7E7F8BD00BF37
:10767000C887FF1FBC87FF1FC487FF1F38B5114B8A
:107680001D68EDB1104B1C682368CBB193F9003035
:10769000834213D12B6883B19C420CD101F0C8FC0A
:1076A00000232B726B72E37B43F00203E373BDE8AC
:1076B000384001F0C5BC0C35ECE738BD1434E3E7C5
:1076C00038BD00BFC887FF1FBC87FF1F154A164B78
:1076D00011681B68013130B5104611600BB30C33D3
:1076E000042453F80C2CE2B113F8031CB9B105685B
:1076F00053F8081C8D4212D1D17B8D0705D40D079C
:1077000058BFD47313F8041C117492892AB153F82A
:10771000081C0A4443F8082C01E003F8032C0C333E
:10772000DFE730BDC487FF1FC887FF1F37B590F85C
:1077300033300546B3B1028B8A4213D800248DF84A
:10774000023001238DF803302046DD2369460522EF
:107750008DF800408DF801408DF80430FFF7BEFC35
:1077600085F8334003B030BD2DE9F04191F8343055
:1077700013F0010C05460C4605D00A8B0B8DD31A6D
:107780000B8300230B8594F830309A0714D0DB0765
:1077900028464CBF1121132102F038FCC0B200284A
:1077A00040F09E8094F8303023F0030343F0400310
:1077B00084F83030BDE8F08103F0200202F0FF08C9
:1077C000002A40F08880268B4EB923F040032846DB
:1077D00084F8303002F00AFC2046314677E0E06A57
:1077E000E16810F480600A781BD003F0040000F018
:1077F000FF0728B123F0040384F83030474611E036
:1078000094F83200824205D094F83180904509D135
:10781000012E07D043F0040384F8303002460127DC
:1078200000E00746BCF1000F33D062698B199A4221
:1078300004D8521A92B2002A52D000E03246E38BAA
:10784000284FB6EB530F09D957F82530DB8CB01A07
:10785000984203DBB2EB560F88BF520894F83030E1
:1078600043F0400384F83030284602F06FFDE368AF
:10787000626903449342E36024BFA368E36057F85E
:1078800025300646D98C2046FFF750FF2685BDE8F7
:10789000F0812846114602F0B9FB236801332360CA
:1078A00094F8303043F0400384F83030C7B9E368CF
:1078B000626901339342E36024BFA368E360238BD2
:1078C000013B2383074B53F82530D98C2046BDE874
:1078D000F041FFF72BBF2846BDE8F04102F086BB20
:1078E000BDE8F081D887FF1F38B505463820FFF77F
:1078F000A3FC044608B9002038BD2846FFF79CFCCD
:10790000A0600028F7D043192061E0606361E5833F
:10791000204638BD10B50C46083102F043FD228BDD
:10792000238DD31A03442383E368181AA368E06005
:10793000984202D2E38B1844E0600023238510BDF7
:107940002DE9F84304460E463F48217AFFF7FCF83C
:107950000146054610B1700705D46FE0FFF7F4F853
:10796000054600286DD005F18053384A3649126823
:10797000DFF8E080013B1B0116F0020F02EB03076A
:10798000D15007D0E08894F80890FFF7ADFF48F891
:107990002900B86016F0010F2D4E06D0A088FFF721
:1079A000A3FF237A786046F82300227A294B58F8FF
:1079B00022208AB12168D162227A617B53F8222089
:1079C00082F83410227AE18853F82230E27B4A436D
:1079D000642192FBF1F2DA84227A1D4B56F82220C0
:1079E0002AB3217B82F83310A188227AA67B53F830
:1079F00022004E43642296FBF2F68684207AE67BD0
:107A000053F82000714391FBF2F2C284227A53F8BA
:107A100022102268CA62227A617B53F8222082F8FF
:107A20003410217AA27A53F8213083F83220237A55
:107A30003B73207A214602F07FFB02E00846BDE856
:107A4000F8832846BDE8F8838D7C0000AC87FF1FD3
:107A5000CC87FF1FD887FF1F2DE9F0417A4B53F8E1
:107A600021407A4B94F8342053F82150E36A0F46B2
:107A700002F00201064601F0FF08F1B1E18B258B0F
:107A8000206916074CBF4A080A4615442583DD05C0
:107A90006369104444BF02F1FF3292B2984228BF9A
:107AA000C1EB0001206128BF21613846216902F045
:107AB0007BFC238C01332384BBE01A0512D594F898
:107AC0003020500704D522F0040284F8302014E05E
:107AD00094F83210B14205D142F0040284F830200B
:107AE000BDE8F08113F0800807D094F83180B8EB3E
:107AF0000601D1F1000858EB01089A0625D5132E8E
:107B000012D195F83430DC0703D538462946FFF703
:107B100001FF95F8303043F0200385F830306B6872
:107B200001336B60BDE8F081112E0ED195F8303035
:107B3000980640F1878023F0200385F830303846DE
:107B40002946BDE8F041FFF70FBE2268D90402F1D3
:107B50000102226019D52A8BEB8B9A420CD82B6933
:107B60001E702B696A69013393422B6124BFAB6895
:107B70002B612B8B01332B8395F8303013F0600F82
:107B800003D138462946FFF7EFFDE28B238BB8F18E
:107B9000000F3CD19A420BD90133238323691E7015
:107BA0002369626901339342236124BFA36823617F
:107BB000E36A13F0600F23D094F83020D2061FD46C
:107BC000218BA28C91421BD39E060AD595F83030AA
:107BD00043F0020385F8303038462946FFF7C4FDEC
:107BE00005E038464FF40071EA6A02F02DFA94F885
:107BF000303043F0100384F8303063680133636041
:107C0000E26A48F2800313409BB1BDE8F081218C09
:107C10009A4201F1010121840BD9013323832369A5
:107C20001E702369626901339342236124BFA368F4
:107C3000236194F8330028B140B20421BDE8F0413B
:107C4000FFF7B2BCBDE8F081CC87FF1FD887FF1FCC
:107C50000D4B53F8203093F8302041B1910611D5E7
:107C600022F0200283F830201946FFF77DBD42F054
:107C7000200283F8302093F83420D20702D5194629
:107C8000FFF748BE704700BFD887FF1F2DE9F843B4
:107C9000984606460D4614469DF8207001F0C8F936
:107CA000A8F10203082B00F23881DFE813F0090085
:107CB00077009B0069000501360136013601E100BD
:107CC000994B1B683FB203EB071715F4805F14BF95
:107CD000BF687F68002C51D0230605D53046214669
:107CE000FA6A02F0B1F949E060050BD52146304649
:107CF000FA6A02F017FB0546C5F300213046FFF78C
:107D0000A7FF0BE1E10717D597F834309A070FD595
:107D1000FA8B1807FB6A48BF5208D90544BF02F125
:107D2000FF3292B27A843046396902F03DFB08E0B6
:107D3000304602F00BF904E0A30702D5304602F00A
:107D40004BF9600703D5304602F0B0F804E0210794
:107D500002D5304602F0F0F814F0100FFB6A02D0A2
:107D600043F4805303E0A20602D523F48053FB6260
:107D7000660644BF05F07F0587F83350BD8DCDE022
:107D8000694B1B6803EB071748F280027B68D96ACE
:107D90000A400AB11D8CC1E01D8BBFE0624B1B681D
:107DA00003EB0717BF683DB9FD8B3B8BED1AA5426E
:107DB000C0F2B380ADB2B1E001F042F929462246EB
:107DC00007F10800FFF7CAF8054601F031F997F806
:107DD000303013F0600F40F0A18030463946FFF795
:107DE000C3FC9BE0DFF84091D9F800304FEA071858
:107DF000434429465F68224607F10800FFF745F82B
:107E000097F8343013F0080F054648460BD03B8CEA
:107E1000DC0708D4BA68FB8BF96802EB530399427C
:107E200028BF1346FB60FA6A12F0600F78D097F80B
:107E30003030D90674D53C8BF98C8C4270D823F045
:107E4000100387F8303097060CD507684744304652
:107E5000B96891F8303043F0010381F83030FFF712
:107E600083FC5DE030464FF4807102F0EDF857E09E
:107E70002D4B1B683FB2012C03EB071704D9023CC2
:107E8000BB68A4B27DB902E07B6865B907E0012C4C
:107E900005D91D605D607B681D605D603EE000256A
:107EA00043F824503AE003EB84040023E25CEA54F4
:107EB0000133042BFAD130E03FB21B4D24B12B68C3
:107EC00003EB0717BB6821E02A683F013A44536877
:107ED00093F83010CC0619D521F0100183F830103A
:107EE0009168CA6A900609D591F8303043F00103D1
:107EF00081F830303046FFF737FC04E030464FF46D
:107F0000807102F0A1F82B681F447B689A680025F5
:107F10001A61DA601D831D8400E0002501F090F8ED
:107F20002846BDE8F88300BFAC87FF1F024B53F81B
:107F30002010FFF719BC00BFD887FF1F40B183692D
:107F400093F82420501C83F8240003EB4203998308
:107F5000704711F0010F30B500F1020408D0057828
:107F6000134623F8025B407845EA002515801A463F
:107F700011F0020F04F1020008D02578134623F80F
:107F8000025B647845EA042515801A464B0705D53F
:107F900003781380417843EA0123138030BD000049
:107FA0002DE9F8439946374B089E1B68282404FBAB
:107FB00009340746E38A002B61D1A58AF36822833E
:107FC0008A4234BF90468846A84538BF4546A4F843
:107FD000168065821860B1682B484A6873684FEA5A
:107FE000054E42F080020EEA0000104318604B6814
:107FF000E06883F040034B608B6883F040038B6044
:108000002946FFF79BFF6760E28A638A9A4206D09F
:10801000E3683BB19B6993F82430012B02D9E08AD5
:10802000BDE8F8834846314601F080FD0028F6D1CE
:10803000F36815482F44C5EB0808A58A1F60B1688E
:1080400073684A681FFA88F8A84538BF45464FEA62
:10805000054E42F080020EEA0000104318604B68A3
:10806000E06883F040034B608B6883F040038B60D3
:108070002946FFF763FF638A2B446382C4E700202D
:10808000BDE8F883E887FF1F0000FF032DE9F041FA
:1080900088B01D4680460E4617469DF8384000F0D1
:1080A000C7FFAB1E042B00F2A180DFE803F003231F
:1080B000701C9000524B1B6824B203EB041416F49E
:1080C000805F14BFA36863687C0608D59A6992F83C
:1080D0002110C80744BF06F07F0682F820609B6924
:1080E00093F8214085E0464B1B6803EB041463685A
:1080F0001C8A7EE0424B1B6803EB0414A5685DB943
:1081000003AC4046214601F011FD18B900943046F9
:10811000394636E02C466CE0AB6993F8214014F008
:10812000010466D036B9EC8A2B8AE41ABC425FDBC4
:10813000A4B25EE000F084FF31463A462846FEF7DE
:108140000DFF044600F074FFAB6993F82130590627
:108150004FD403AE4046314601F0E8FC002848D138
:108160006B68EA68D21AAB6993F8211041F04001BC
:1081700083F8211092B20096944228BF1446686892
:10818000A1B20A464346FFF70BFF044631E01C4B01
:108190001B6803EB04143A46656831462846FEF72F
:1081A00074FEAB6993F821305A07044623D500F0DA
:1081B0003FFFAB6993F8212022F0040283F82120CD
:1081C000AB69987E01F076FD0028F9D011E00C4BE8
:1081D0001B6824B203EB04140FB1A36800E06368CA
:1081E0001A6800249A605A601C8202E0002400E0B1
:1081F000344600F025FF204608B0BDE8F08100BFFE
:10820000AC87FF1F2DE9F04F87B007460DF1160030
:10821000884691461E46FAF7BBFE00244FF0010B3C
:108220000178BDF81620521A92B2ADF816204378A4
:108230000192042B10D0052B20D0022B45D143797D
:10824000BB4205D0D7F1010438BF0024002C3CD03C
:1082500001244FF0000B38E0002C36D0B8F1FF0FAE
:1082600002D08378434530D1B9F1FF0F02D0C378F3
:108270004B4529D1002E31D0022426E02CB326B361
:10828000A51ED5F1000C5CEB050C35462B68B3B18F
:108290009A7890F802A082EA0A0252060DD1BCF147
:1082A000000F12D193F805C01B7943EA0C23B5F8EF
:1082B00004C09C4509D2AB8007E00835E6E7BCF175
:1082C000000F02D0286000E00324019B0844002B2B
:1082D000A6D1BBF1000F0CBF3046002007B0BDE8AF
:1082E000F08F37B5836993F820300546BBB1028A19
:1082F0008A4214D800248DF8023001238DF803300F
:108300002046DD23694605228DF804308DF80040B3
:108310008DF80140FEF7E2FEAB6983F8204003B020
:1083200030BD0000F8B504468078E77866790B46E2
:1083300000F07F010AB2550105EBC2020A4D2D681B
:108340001544227920F07F00384342EA062201F0EA
:1083500023FCE3780BB9112303E095F8223043F0B6
:10836000010385F82130F8BDE887FF1F00F07F0189
:1083700038B5104A0BB25C0104EBC30314681C440B
:1083800000221346E568FF2001F006FC002384F874
:108390002130E38284F824301DB12B822B68AB603E
:1083A0006B60A36823B100221A821A689A605A602F
:1083B00038BD00BFE887FF1F2DE9F04105462A4F71
:1083C000A97B2A4A3C6804301C23FEF7DBFBAE7B0A
:1083D00080466EB136B2730103EBC6063444AB89F6
:1083E000A3826B89DE0614D5202384F8223010E0A6
:1083F0006B7C282001335843FEF71EFF082383823D
:10840000AB7C3860044680F820302946304601F0C5
:1084100091FC174A08F180531268013B02EB0312EA
:108420009368E36013B19C612B892382AB7BA376B5
:10843000AB7B6BB1EB7B5BB119B24C0104EBC101BF
:108440003C680C44A376AB7B84F82330AB89A382D1
:108450005368A3601BB19C61AB7C84F820302B680F
:1084600040462360BDE8F081E887FF1F8D80000053
:10847000AC87FF1FF8B51546194A0E461168282229
:1084800050430C180F5817B9A06838B9F8BD3046DA
:1084900029461A46B847072820D1F5E794F8200066
:1084A00018B140B20421FFF77FF894F82120A368A7
:1084B00002F0040101F0FF0779B9D88A198A411A3C
:1084C000A94206DB184631462A46FEF747FD3846E4
:1084D000F8BD42F0040284F821200120F8BD00BF5D
:1084E000E887FF1FF0B5A1B00E46802200210546A7
:1084F0006846FEF7B9FC3046FF2100226B46FFF7C5
:1085000081FE40B3154F00245DF8040020B355B937
:108510001EB98078FFF72AFF1BE000AB234499883F
:10852000FFF700FF15E0837803F07F035A0102EBA9
:10853000C3033A681344012D93F821200BBF22F0A6
:10854000010222F0020242F0020242F0010283F82C
:1085500021200834D8E7012021B0F0BDE887FF1FB3
:108560002DE9F0439446A5B00D461E4606282AD8AC
:10857000DFE810F00F017702720207007E028C0222
:108580009202A24B1B68282707FB0C37FC8AFD6868
:108590001CBBC5B12C8AC4B16A68EB689A4202D38D
:1085A000E98A521A6A606868191A89B2A14228BF1A
:1085B000214600960A466346FFF7F2FCAB6928465F
:1085C000198AFFF78EFE00246FE2AB6993F8212031
:1085D00022F0400283F8212067E27B8AA342C0F0A8
:1085E0009D80002D78D02B8A002B75D0AA6992F837
:1085F0002410908B012901F1FF31C8BFB2F81EE0B1
:1086000082F82410C0EB0303A969C8BFA2F81CE0DC
:108610009BB22B8291F824206FF0010E501C01EBCD
:10862000420800220EFB00F09646023A824207D032
:1086300008EB0209B9F81C90CE441FFA8EFEF4E74D
:10864000734535D1002BB9D1BCF1000F04D097F898
:10865000212012F0300F17D0BB8AB4FBF3F203FBDA
:1086600012439BB27BB9B36870685A6842F08802C3
:1086700002605A6882F040025A609A6882F04002B2
:108680009A60012300E000236A681444EA686C6081
:10869000944202D3EA8AA41A6C600022FA82002B68
:1086A0008CD191F8213023F0400381F8213085E707
:1086B0006A68E96814448C426C6002D3EA8AA41A9E
:1086C0006C606868091ACEEB030389B28B42B8BFAD
:1086D00099B20023FB826CE7BB8AB4FBF3F203FB85
:1086E00012439BB2BBB93B8BA34206D1BCF1000F36
:1086F00011D097F82130DB060DD4B36871685A6841
:1087000042F088020A605A6882F040025A609A6811
:1087100082F040029A600024FC82C6E1E41ABA8A20
:10872000A4B2944228BF1446A5B1AB6993F82420A3
:10873000998B012AC8BFD88B02F1FF3283F824201D
:10874000C8BF98832B8A5B1A2B82AB692846198A8B
:10875000FFF7C7FD798A7A68F3680A441A60B3683C
:1087600071685A6842F08000294A26043240024368
:108770000A605A6882F040025A609A6882F04002A9
:108780009A6021462846FFF7D9FB7B8A1C447C82ED
:1087900019E70C781D4B24F08004D3F800800027E3
:1087A000012CA8F81670994600F09380022C00F076
:1087B0000281002C40F049814B78092B7ED8DFE8FC
:1087C00003F0787D7D7D7D45057D74488B78C87884
:1087D000CF7943EA00208B7943EA072700F47F43EF
:1087E000B3F5007F18D006D8B3F5807F27D104A851
:1087F000FAF7C8FB1BE0B3F5407F11D0B3F5C06FAB
:108800001DD1009603480A2114E000BFE887FF1F2E
:108810000000FF0342D3000004A8FAF7B9FB06E00A
:10882000C0B204A9FAF7BAFB002800F03D81BDF8F8
:10883000101000963A460023FFF7B2FB35E1D8F856
:108840000030002B00F03081681C3DE08B78B37461
:1088500029E08978974E00203170FFF743FE0446E7
:1088600010B1002333701FE1D9F8003093F8206075
:10887000CEB1A91C01220DF11600FEF7FDFA7523F9
:108880008DF8133002238DF814302046FE2304A9FE
:1088900007228DF810408DF811408DF812608DF888
:1088A0001530FEF71BFC0324FFE0009681480121F0
:1088B00002E08148009602210A46BCE7D8F8003061
:1088C000002B00F0F1800846318A002298470446C8
:1088D000EBE091F80190B9F10A0F01F1020044D0E8
:1088E000B9F10B0F04D0B9F1000F40F0AE8058E0A1
:1088F000704D2B78002B00F0D780032103AAFFF7DF
:1089000028FB9DF80E403946802204A8FEF7ACFAF9
:1089100028782146FF2204ABFFF774FC083704AB2C
:108920003B4453F8084C1CB1A078FFF71FFDF5E756
:108930009DF80E709DF80C602146802204A8FEF779
:1089400093FA28783946324604ABFFF75BFC0028DF
:1089500000F0AA80083404AB234453F8080C002824
:10896000A1D00021FFF7DEFCF4E7524D2B78002B5D
:1089700000F09A80022104AAFFF7EBFA28789DF80C
:10898000101022463B46FFF73DFC002800F08C808B
:1089900021462246009603303B46FFF701FB3C464A
:1089A00083E0444B1B78002B7ED002210096434885
:1089B0000A464B463EE04F78012F3ED8881C04AA59
:1089C0002146FFF7C6FA3B4BBDF810001B780BB9E8
:1089D000002869D1282300F01F0203FB0282012F27
:1089E00092F8213018D11F077FF5EDAD23F0080371
:1089F00082F82130D8F80030002B3FF4E4AD24ACED
:108A0000C0B204F8840D01F04DF8D9F800302046CA
:108A10001B680021042259E703F0080202F0FF035B
:108A2000009622B1022126480A46002302E00221D4
:108A300022480A46FFF7B4FAC5E5D8F80030002B03
:108A400032D008460322082140E7D8F800305BB353
:108A50002846318A3A4639E71A8A12B96046022313
:108A600003E0328A604629460123FFF703FD2EE723
:108A70009B7C33B1134B1B68CC2193F92000FEF78C
:108A800069FB00200146FFF72DFD9CE50D4B1B689F
:108A9000CB2193F9200004E00A4B1B6893F92000D6
:108AA000CA21FEF757FB8EE50424204625B0BDE819
:108AB000F08300BFE687FF1FE487FF1F4ED300004F
:108AC0004CD30000E887FF1F054B1B68282202FBE0
:108AD000003090F82130194380F82110704700BF12
:108AE000E887FF1F034B1B68282202FB003090F829
:108AF00023007047E887FF1F014B1860704700BFD5
:108B0000EC87FF1F00F0A6BA08B56C20FEF71EFD2B
:108B100018B9BDE8084001F0CBBD08BD2DE9F04310
:108B2000414C424D40F2B3720423571EBFB2BE0700
:108B30000ED1A84210D9A0F1F170A0F50540023382
:108B4000DBB2062B02D8013292B2EEE7073BF7E721
:108B5000A0420AD8002400E001240022DFF8F0C07F
:108B6000DFF8CC80DFF8EC900CE000F17E4000F5FF
:108B7000F61000F548600133DBB2062BE3D9073B62
:108B8000FAE702226CB1012A0BD1484519D9A0F5A8
:108B90001810A0F56E501D33DBB2062BF1D9073B40
:108BA000FAE71CF8025008FB05F6B04209D9801B11
:108BB0002B44DBB2062B01D9073BFAE70132D2B2D4
:108BC000E0E71B4C0126A0420BD9A0F5A8300136E6
:108BD000A0F5C070F6B20133DBB2062BF3D9073B28
:108BE000FAE70024B0F5616F04D90134A0F56160A3
:108BF000E4B2F7E700253C2803D901353C38EDB253
:108C0000F9E771B10B4901320A700B4A16700B4A31
:108C100013700B4B18700B4B1D700B4B1C700B4BD8
:108C20001F80BDE8F08300BF8033E1010085E201D1
:108C3000805101002182FF1F1A82FF1F1C82FF1F2B
:108C40004889FF1F6C8BFF1FC488FF1F1E82FF1FF8
:108C5000B4D30000803B26002DE9F047B0F8048033
:108C6000042340F2B2740022444504F0030617D2F4
:108C700001344EB902F1F17202F505420233DBB262
:108C8000062BF1D9073BFAE702F1F07202F59932AF
:108C900002F5C0720133DBB2062BE5D9073BFAE7D8
:108CA0008579DFF8B8C0DFF8B8906C1E54B1013C8C
:108CB00014F80C7009FB07223B44DBB2062BF5D9F4
:108CC000073BFAE75EB9022D09D902F5A83202F591
:108CD000C0720133DBB2062B01D9073BFAE790F8EB
:108CE00007C00CF1FF394B44DBB2062B01D9073B1F
:108CF000FAE7867A477AC47A30B24FEA800A80016E
:108D0000CAEB00004FF4616A0AFB0700DFF850A0CD
:108D100020440AFB090909EB020079B1084AA2F8CC
:108D20000080084A1570084A82F800C0074A177088
:108D3000074A1670074A1470074A1370BDE8F08797
:108D40001E82FF1F2182FF1F1A82FF1FC488FF1F80
:108D50006C8BFF1F4889FF1F1C82FF1FB4D30000CC
:108D600080510100704770477047704770477047E7
:108D70007047704770470000034B4FF400621A6061
:108D800000200221FEF768BE24800040034B4FF410
:108D900080621A6000200121FEF75EBE2480004040
:108DA000034B4FF4007200201A600146FEF754BED8
:108DB000248000400B4B10B520220B4C1A60236816
:108DC000022023F004032360FFF7B0F823685A075A
:108DD00007D443F004032360044B1A7842F04002A6
:108DE0001A7010BD24800040688BFF1F03C006402E
:108DF0000B4B10B510220B4C1A602368012023F096
:108E000002032360FFF792F82368990707D443F021
:108E100002032360044B1A7842F040021A7010BD1E
:108E200024800040688BFF1F03B006400B4B10B539
:108E300008220B4C1A602368002023F001032360F2
:108E4000FFF774F82368D80707D443F001032360C1
:108E5000044B1A7842F040021A7010BD2480004082
:108E6000688BFF1F03A0064038B51C4A1C4D1278C2
:108E70002B789006DBB211D41A4A12781A40910668
:108E80000CD5194C194B20789B7802211840FEF71D
:108E9000E3FD2B78DBB21A0748BF22780F4A114C4A
:108EA00092F90020002A07DB227822F03F021342C9
:108EB00002D00220FFF73AF823785D060CD5084A65
:108EC0001278540608D5074A23F040031370084B64
:108ED0001A6822F004021A6038BD00BF0BC00640B9
:108EE00004C0064003C0064007C00640BC88FF1F00
:108EF000688BFF1F38B51C4A1C4D12782B789006E2
:108F0000DBB211D41A4A12781A4091060CD5194CCA
:108F1000194B20785B7801211840FEF79DFD2B78D6
:108F2000DBB21A0748BF22780F4A114C92F9002091
:108F3000002A07DB227822F03F02134202D00120F0
:108F4000FEF7F4FF23785D060CD5084A1278540624
:108F500008D5074A23F040031370084B1A6822F023
:108F600002021A6038BD00BF0BB0064004B00640D4
:108F700003B0064007B00640BC88FF1F688BFF1F88
:108F800038B51D4A1D4D12782B7802F02002DBB255
:108F900002F0FF0182B91A4A12781A4090060BD5E6
:108FA000184C194B20781B781840FEF755FD2B788C
:108FB000DBB21A0748BF22780F4A114C92F9002001
:108FC000002A07DB227822F03F02134202D0002061
:108FD000FEF7ACFF23785D060CD5084A12785406DC
:108FE00008D5074A23F040031370084B1A6822F093
:108FF00001021A6038BD00BF0BA0064004A0064065
:1090000003A0064007A00640BC88FF1F688BFF1F17
:10901000064B10B51C68238841F27B22002B08BF49
:1090200013460380FEF740FA208010BDC88BFF1F57
:1090300072B6024B1A6801321A607047B888FF1F77
:10904000034A1368013B136003B962B6704700BF5F
:10905000B888FF1F08B5094B1B88DB070AD5FFF747
:10906000E7FF074B4AF202621A804BF280421A80F5
:10907000FFF7E6FF034B20221A6008BD00200540E1
:109080000C2005408CF00F4008B5054B1A681A609B
:10909000FFF7CEFFFEF71AFBBDE80840FFF7D0BF91
:1090A00000000440F8B52D4E33680446154653B908
:1090B0002B4F2C4A27F00107D85B985202333C2BE8
:1090C000FAD1294B336029480278284B1206FBD588
:1090D0001A7812F0300F1CBF30221A70244B092C62
:1090E0001C700BD002D8062C08D01AE0412C11D0ED
:1090F000432C16D10A681F4B1A700FE01D4B0A0C47
:109100001A70062C4FEA112203F8012C03F8021CF6
:1091100007D103E00A68174B1A7002E02B68164A61
:109120001360FFF785FF336810489847FFF788FF03
:10913000412C0ED1114B1A78013B1B781B0443EADA
:1091400002630D4A127813430D4A127843EA022350
:109150002B60064B187800F03100F8BD3488FF1FF3
:109160000E82FF1FF887FF1FF987FF1F00000240D4
:109170000700024006000240080002400B000240C7
:1091800009000240F8B5444B1D68444B1A7801327F
:10919000D2B23B2A1A7063D900221A70404B197858
:1091A0000131C9B23B29197038D91A703D4B197871
:1091B0000131C9B21729197024D91A703A4A3B48AB
:1091C000117803780131C9B211700133DBB2062B7B
:1091D00001D9073BFAE71D29037007D1344B1978F1
:1091E000022903D10121117003221A70314B1B682F
:1091F0001B0707D5304BDC6824B1FFF719FFA047E8
:10920000FFF71EFF2B4B1B689F0607D52A4B5C6997
:1092100024B1FFF70DFFA047FFF712FF254B264CA7
:109220001A6812F0020F1F4606D0666826B1FFF7D3
:10923000FFFEB047FFF704FF204A13781E060FD445
:10924000013BDBB213703A68D00709D55BB201333A
:1092500006D1246824B1FFF7EBFEA047FFF7F0FE2C
:10926000154B1C691E4624B1FFF7E2FEA047FFF72D
:10927000E7FE104B1B6859070CD5114B1B689D422C
:1092800008D1B46834B1FFF7D3FEA047BDE8F84079
:10929000FFF7D6BEF8BD00BF00D003404889FF1FCE
:1092A0006C8BFF1FC488FF1F1A82FF1F1C82FF1FC9
:1092B0002182FF1F4488FF1F748BFF1F2082FF1F26
:1092C0004C8AFF1F094B1A6822F4803222F04102B7
:1092D00010B51A60064B1C6834B1FFF7A9FEA04711
:1092E000BDE81040FFF7ACBE10BD00BF00600340FA
:1092F000708BFF1F10B5084B1B7801229A40074B5B
:109300001A60074B1C6834B1FFF792FEA047BDE816
:109310001040FFF795BE10BDF087FF1F248000406E
:10932000AC88FF1F036810B51C061CD5144B33F81E
:109330001130DA0404D5C3F30B039BB2036012E0CF
:1093400080230129036004D0022907D059B90D4BAD
:1093500005E00C4B1A6822F0007203E00A4B1A6811
:1093600022F080721A60094B53F8214034B1FFF7A4
:109370005FFEA047BDE81040FFF762BE10BD00BF12
:10938000B088FF1F3C800440308004403888FF1FB5
:1093900001480221FFF7C6BF00800B4001480121B0
:1093A000FFF7C0BF0090034001480021FFF7BABF9C
:1093B0000080034003782DE9F04707460D4603F08F
:1093C000FF0613B30124DFF84890A246344217D0B9
:1093D0000F2D26EA040608DDA5F110030AFA03F3AF
:1093E000012B03D1FFF750FE00E03C7059F82580B7
:1093F000B8F1000F04D0FFF71BFEC047FFF720FEB7
:1094000064000135E4B2002EE0D1BDE8F08700BF72
:109410004C88FF1F08B507480021FFF7CBFF06481F
:109420000821FFF7C7FF05481021BDE80840FFF7F6
:10943000C1BF00BF05C0074006C0074007C00740C6
:109440002DE9F843134FDFF854803C68FCB1124E0D
:109450003C600125254215D0D6F80090FFF7E8FDC5
:1094600008EB060303F14043A3F59A2309F43029DE
:109470001B689847B9F5002F08BF3D6024EA050432
:10948000FFF7DEFD6D000436002CE3D1DDE7BDE81B
:10949000F88300BFA0D0044000D00440CC89FF1F57
:1094A0002DE9F843134FDFF854803C68FCB1124EAD
:1094B0003C600125254215D0D6F80090FFF7B8FD95
:1094C00008EB060303F14043A3F5982309F4302980
:1094D0001B689847B9F5002F08BF3D6024EA0504D2
:1094E000FFF7AEFD6D000436002CE3D1DDE7BDE8EB
:1094F000F88300BFA0C0044000C004404C89FF1F97
:109500002DE9F843134FDFF854803C68FCB1124E4C
:109510003C600125254215D0D6F80090FFF788FD64
:1095200008EB060303F14043A3F5962309F4302921
:109530001B689847B9F5002F08BF3D6024EA050471
:10954000FFF77EFD6D000436002CE3D1DDE7BDE8BA
:10955000F88300BFA0B0044000B00440E88AFF1FB9
:109560002DE9F843134FDFF854803C68FCB1124EEC
:109570003C600125254215D0D6F80090FFF758FD34
:1095800008EB060303F14043A3F5942309F43029C3
:109590001B689847B9F5002F08BF3D6024EA050411
:1095A000FFF74EFD6D000436002CE3D1DDE7BDE88A
:1095B000F88300BFA0A0044000A00440C888FF1F9B
:1095C0002DE9F843134FDFF854803C68FCB1124E8C
:1095D0003C600125254215D0D6F80090FFF728FD04
:1095E00008EB060303F14043A3F5922309F4302965
:1095F0001B689847B9F5002F08BF3D6024EA0504B1
:10960000FFF71EFD6D000436002CE3D1DDE7BDE859
:10961000F88300BFA090044000900440548AFF1FCC
:109620002DE9F84F064690461D460F46FFF700FD10
:10963000364B374C1A684FF00C0909FB06F94A44BF
:10964000A260926812F0400F9B4605D105F110030D
:10965000636005F1140304E005F11803636005F18C
:109660001C03DFF8ACA0E3603846D8F8041032469B
:109670005346FEF775FF0328074606D004281BD083
:1096800001282CD1FFF7DCFC3CE0DAF80810DAF80E
:1096900004204B6843F0800313604B6883F0400361
:1096A0004B608B6883F040038B60D8F8003043F048
:1096B0008003C8F8003022E026B984232B61AB6117
:1096C000304609E03046FFF70DFA124B1B6803EBFA
:1096D000401384221A619A610821FFF7F5F9DBF83B
:1096E000002002EB090399680B4B0B4021680B43E8
:1096F00043F080012360C8F8001042F80930FFF7FA
:109700009FFC00273846BDE8F88F00BFF487FF1F95
:10971000D48AFF1F508AFF1F0800FF032DE9F0477E
:10972000AA4E3746AA4DDFF8CC822C7898F8003044
:109730001C4000F0488134F0080900F08780FFF7F2
:1097400077FCE3074AD5A34AA34833232B70137849
:1097500043F00203137098F8003023F0300388F8C8
:1097600000309E4B19688B6823F040038B60002308
:109770000B601178137101F0FD01117098490122FD
:109780000A70984A13701371137103700371037296
:1097900003730374037503760377137182F8303013
:1097A00082F8343082F838300B7803F0040303F089
:1097B000FF08002BF8D18C4B8C4A1B68DFF83CA2C9
:1097C0009A6040321A600420424653464146FEF7F2
:1097D000C7FE834B8AF812800D221A70A00711D59C
:1097E0003378590703D5824B5A6801325A603B7867
:1097F0009A0703D57E4B1A6801321A60062333702C
:1098000002232B70E3060CD530232B70794B1A788A
:10981000002142F020021A7005200A460B46FEF78E
:109820009FFEA0060CD530232B70724B1A780021B6
:1098300022F020021A7006200A460B46FEF790FE20
:109840005FFA89F9FFF7FCFB85F8009021077FF5A7
:109850006AAF694A644B1578147818682D0929B2E3
:1098600014F0080F00EB4113644C20D08A0009016A
:10987000891A5A4A12681144A1608A68520604D4AF
:1098800003F110026260143303E003F11802626016
:109890001C33E360FFF7CCFB2A46584B0021032022
:1098A000FEF75EFEFFF7CCFBA27C554B7EE0127804
:1098B00002F0040202F0FF0E22B103F108024FF0A1
:1098C000400E00E01A46C4F800E0D2F800E0CEF303
:1098D000094CA4F810C00EF03C04042C02D0342C27
:1098E0002BD065E0DFF8F48008018C00041BD8F869
:1098F000000000EB040E8900DEF808E01EF0080FFF
:109900001CBF005900F080093548415C08BF4FF08A
:1099100080092846CD064CBF01210221FFF780FEB9
:10992000D8F800301A59B9F1000F02D022F08002A5
:1099300001E042F080021A5141E000241C619C6168
:109940002E4CDFF898E024684FEA810C4FEA0118AA
:1099500014F0400FDEF80040CCEB080C6444D4F85F
:1099600008C0284C0CEA040404D1046044F0C0048C
:10997000846003E0846044F0C0040460880009014E
:109980000C1ADEF8001021444820486028460021C7
:10999000FFF746FE012805D0104B1B681A5942F00C
:1099A00080021A510B4B1A7802F0DF021A7006E09F
:1099B00084221A619A6128460821FFF785F8044B32
:1099C00008221A70AEE6BDE8F08700BF8820074085
:1099D0008020074094200740D0200740F487FF1FD5
:1099E000C0200740C4200740508AFF1F880008009D
:1099F0008C8BFF1F8420074090200740D48AFF1FD4
:109A0000982007400800FF03104B1B6840330901F2
:109A100043F8202000F1604303F56443C9B2197094
:109A200020220B4B90FBF2F29200034002F16042C5
:109A3000002B02F5614203DA013B63F01F0301339F
:109A4000012101FA03F31360704700BF08ED00E045
:109A50001F0000800E4B1A6810B542F001020D4C39
:109A60001A60802323600C4B05221A6055200B4A94
:109A70000621FFF7C9FF236843F040032360084B2A
:109A800031221A60236843F00103236010BD00BF38
:109A90003880044000000440040004408990000025
:109AA00008000440134B20F0800210B51C685101DF
:109AB000000604EB010313D50F48104900680C247D
:109AC00004FB0200446824F0400444600020186154
:109AD000986111F8223023F0020301F8223010BD02
:109AE000625822F0040262509A6822F004029A60DE
:109AF00010BD00BF508AFF1FF487FF1FC020074022
:109B000008B548B101280AD001300BD10021082244
:109B10000548FDF7A9F905E0034B186808BD024B9D
:109B2000586808BD002008BD8C8BFF1F38B5174B47
:109B30001D68174B13F820305A070C4624D5154BD7
:109B40001B680C2202FB00338B6005EB4015FFF70E
:109B50006FFAA3689B685B0604D405F11003636089
:109B6000143503E005F1180363601C356368E56094
:109B7000186810F0800403D0FFF762FA022038BDA5
:109B8000FFF75EFA204638BD012038BD508AFF1F1E
:109B9000C0200740F487FF1F2DE9F04F9C46404B43
:109BA000DFF80C81D3F800900C468B002701FF1AD8
:109BB0003C4B1646D3F800A04A0118F8211009EBD7
:109BC000020521F00C010AEB070B08F82410FF280E
:109BD0004FF00001A9612961A96085B049F8021020
:109BE000CBF808109B464AF807102F4B06D11A787D
:109BF00022F030021A7008F824104EE093F800A00A
:109C00004AF0100A83F800A0DBF8003020F0800A48
:109C1000BAF1010F3B4402D15960242303E008212B
:109C2000596005234821000631D4686880B966452B
:109C300038BF66463046039101920293FDF7FCFA65
:109C400068603046FDF7F8FA029B019A0399E860D4
:109C5000164836043040014341F0800021F04001B5
:109C6000A86041F0800049F80200DBF800201744AA
:109C700043F0080CB960BAF1000F01D1634603E06C
:109C800003F0FB0343F0180308F8243005E0BAF1B1
:109C9000000FF9D043F01003F6E705B0BDE8F08FF0
:109CA000508AFF1FF487FF1F842007400000FF0336
:109CB000C02007401C4B2DE9F0411D6803B205EBA5
:109CC00043159A001C01194BA41A1A68125912F074
:109CD000400F0CBF083500262A6808BF402612F046
:109CE0008007984619D16968C2F309420123FEF73B
:109CF000C1FB012814D0D8F800301A1938469168F1
:109D00000B4A0A4032431E5906F0800642F0800199
:109D1000324329601A51BDE8F0810120BDE8F0818D
:109D20000220BDE8F08100BF508AFF1FF487FF1FAB
:109D30000800FF032DE9F0414D4B4E7C1A6842F0BC
:109D400040021A6003F5203301361A6822F080427F
:109D500042F000421A600B7C012B0C46F6B209D18E
:109D6000444B1A6842F4A0221A605A6C42F0050271
:109D70005A6408E0404B1A6842F400521A603F4BA4
:109D80004FF4E0621A603E4B1A68102E28BF10266E
:109D900042F480220C201A607043FDF74DFA394AD4
:109DA000394B1060197841F08001197017461A7804
:109DB0001506FCD4354D02232B704FF40071700151
:109DC000FDF762FA324B334A1860000A1070598866
:109DD0001175D9781176304900220A7028312A701D
:109DE0000A701D460B7803F0040303F0FF06002BF6
:109DF000F8D10820D5F80080FDF71EFAC8F8040055
:109E00000820D5F80080FDF717FA2B68234AC8F818
:109E10000C009A6040321A603B684FF008129A605A
:109E20001F4B0D221A70ED2203F8B02CFF2203F80D
:109E3000402CBF2203F8382C49201A4A0621FFF78C
:109E4000E3FD194B8B2203F87C2C062203F8742CBB
:109E500001221E7003F86C2C6389DC0705D50A4BC0
:109E600040221A70102203F8042CBDE8F08100BFD4
:109E700000F00140048004403880044068D0044071
:109E800034800440F487FF1F0C21074094200740D2
:109E9000508AFF1F9C200740982007408800080038
:109EA000C02007401D970000002107401A4B0128E1
:109EB00010B553F820401CD00ED3022827D1174BE1
:109EC0001A6842F480521A60154B4FF440721A60BF
:109ED00031200A21134A18E0104B1A6842F48062BC
:109EE0001A60114B4FF440721A602D200C210F4A5A
:109EF0000BE00A4B1A6842F400621A600C4B4FF4F4
:109F000040721A600B4A2F200B21FFF77DFDE3788A
:109F100043F00803E37010BD54D5000038800440BE
:109F20000CC00440698E000044A00440818F0000F2
:109F300010B00440F58E0000034B53F82030DA785F
:109F400002F03702DA70704754D500001A4B01282E
:109F500010B553F820401CD00ED3022827D1174B40
:109F60001A6842F480521A60154B4FF440721A601E
:109F700031200A21134A18E0104B1A6842F480621B
:109F80001A60114B4FF440721A602D200C210F4AB9
:109F90000BE00A4B1A6842F400621A600C4B4FF453
:109FA00040721A600B4A2F200B21FFF72DFDE3783A
:109FB00043F02403E37010BD54D500003880044002
:109FC00008C00440698E000040A00440818F00005A
:109FD0000CB00440F58E0000034B53F82030DA78C3
:109FE00022F02402DA70704754D50000064B53F873
:109FF000203093F90B20002A05DBDA7802F07F028B
:10A0000042F04002DA70704754D5000030B50C4B76
:10A0100053F820301A7912F0800F4FF001020DD062
:10A02000084C02FA00F01A79DA782568D97162F0E2
:10A030007F020543DA702560002030BD104630BD38
:10A0400054D50000688BFF1F334B53F8203030B5D8
:10A05000002B60D05A7B11F4C05F02F0F9024CD0A3
:10A060000C0528D5012814D00AD302281AD12B4C6C
:10A07000256845F4805525604FF44075284C10E064
:10A08000264C256845F4806525604FF44075254CC5
:10A0900007E0224C256845F400652560224C4FF40A
:10A0A000407525608D0405D54C044CBF42F002027A
:10A0B00042F006025A73CD041FD5012814D00AD3EA
:10A0C00002281AD11548046844F4805404604FF4FF
:10A0D0004074164810E01148046844F48064046039
:10A0E0004FF44074124807E00C48046844F40064DC
:10A0F000046010484FF44074046094070BD4C80700
:10A1000003D55A7B42F008025A738A0703D55A7B5B
:10A1100022F008025A7330BD54D500003880044044
:10A1200000C0044008A0044004B0044004C004403F
:10A130000CA0044008B004406C4B01282DE9F0410C
:10A1400005460F4653F8204009D003D302280BD010
:10A15000BDE8F081664B1A6842F4806208E0644B07
:10A160001A6842F4006203E0614B1A6842F48052BC
:10A170001A603B68580605D528464FF4C0510022A6
:10A18000FFF762FF012DFB7A06D80B2B0CD8594A3A
:10A19000594932F8132005E00B2B08D8574A584983
:10A1A00032F81320CB5C04E00C23EA2201E0062302
:10A1B0007522A372C2F30423D2B2237062703A688C
:10A1C000504912F0010F02F0060307D07F204855D6
:10A1D0005BB151074CBF0323022306E0FF20485523
:10A1E0001BB152074CBF13231223A3707B7BDB07E9
:10A1F00031D5454B5E5D730103F1804303F5104398
:10A2000000220121E01D9980DA809A8218619A610A
:10A21000DA600A2299609A833C4B595D3C4B304688
:10A2200053F82520FFF7F0FBE37A63F07F03E37236
:10A23000384B1A6842F002021A6006F180466B0041
:10A2400006F50436033363F07F033370E37863F07D
:10A250007F03E37003E0E37A03F07F03E3727B7B29
:10A260009E073DD52C4B13F805802C4B595D2C4B8C
:10A27000404653F82520FFF7C7FBE37A43F020035D
:10A28000E372244B1A684FEA481642F0020208F1C2
:10A29000804801351A606D0008F5043365F07F05CC
:10A2A0001D70BB8806F1804606F510469AB2F28210
:10A2B000002101220734B180F383B282F18034603F
:10A2C000B2607A7B12F00C0F04D015074CBF062247
:10A2D0000222B28300225B42F260B361BDE8F081EA
:10A2E000E37A23F02003E372BDE8F08154D5000047
:10A2F0003480044050D3000068D3000074D30000C1
:10A300001BD40000BC88FF1FC7D4000007D4000086
:10A3100040D500003C8004403CD5000018D400002B
:10A320000CD40000084B53F82030480703D55A7B63
:10A3300042F001025A730A0703D55A7B22F0010248
:10A340005A734FF48070704754D50000114B70B5AC
:10A3500053F82040104B26791D5CE6786B0103F121
:10A36000804303F5104326F04006E67094B2DC8289
:10A37000DA831960094B01211C6801FA00F00443DB
:10A380001C60074B186801FA05F528431860104651
:10A3900070BD00BF54D50000C7D40000688BFF1FFC
:10A3A0000C800040002070470B4A52F82020D278E1
:10A3B000520710D4094A125C530103F1804303F59C
:10A3C00010431961064B012101FA02F21968114389
:10A3D0001960FFF7BBBD704754D500003CD50000A5
:10A3E0000C80004038B520F4FF64451824F00704C1
:10A3F000092021460022FEF755FE30B92B1BB3F58C
:10A40000006F03D904F50064F2E7012038BD0000B5
:10A410002DE9F74F16460F46244C51B9236899078A
:10A4200001D100203EE023F0030323604FF0040835
:10A4300004E020F00303236000F00308DFF87090CD
:10A44000DFF868A009F1040BC8F10405B54228BF84
:10A45000354609EB0803184639462A460193FCF7AE
:10A460000BFD019B2B445B452F44C5EB060612D325
:10A47000062021680E4AFEF715FE054688B9DAF86F
:10A4800000300B480433FF210422CAF80030A846EC
:10A49000FCF7EAFC02E023681D442560002ED3D1BE
:10A4A000BFE7012003B0BDE8F08F00BF4888FF1F61
:10A4B000C088FF1F034608461946FCF7DDBC0000B4
:10A4C000F8B5037B23F0E003013B0446092B00F2BF
:10A4D0008A80DFE803F007054D46498A96233C4110
:10A4E00000263FE04B4B4C4D1A6842F000521A6078
:10A4F0004A4B00221A60027B12F0200F1E4606D043
:10A5000000690121FEF70AFB23692B6003E00121AA
:10A51000FEF7A2FB28601023336064E0404B1B78F9
:10A52000C372404B1B8883803F4B1B7883713F4B2A
:10A530001B78C3713E4B1B7803723E4B1B784372F2
:10A540003D4B1B788372344B1B6803614BE0002149
:10A55000FEF782FB206146E000690021FEF7DEFA8B
:10A5600041E00126013600E000260136013600E018
:10A570000026013694F90C30002B08DA2F4B01220B
:10A5800002FA06F61A6822EA06021A602BE0214B4C
:10A59000224D1A6842F000521A602F681E4B17F0C5
:10A5A000010707D000222A601A604FF440721A6136
:10A5B0000120F8BD2168224A42F826102F60186851
:10A5C0000121FEF7ABFA1D4B012202FA06F61A68CA
:10A5D00032431A6043201B4A0221FFF715FA1A4A38
:10A5E000102313602B600020F8BD144B1A68002163
:10A5F00022F004021A60FEF72FFB144B00261860AD
:10A60000B4E7827A124B013A02F03F021A70002638
:10A61000B0E700BF3C80044000D0034014D00340AA
:10A620004889FF1F1E82FF1F2182FF1F1A82FF1F02
:10A630001C82FF1FC488FF1F6C8BFF1F4488FF1FF5
:10A64000748BFF1F859100001CD003404C8AFF1FB4
:10A650002082FF1FF0B5104B1E78104B1F78104B57
:10A660001D78104B1A78104B1C78104B1B8840F249
:10A67000DA7C63450DD9ED0245EA471542EA4412FA
:10A68000A3F2BC73354342EA432305800B800020CC
:10A69000F0BD0120F0BD00BF4889FF1F6C8BFF1F7C
:10A6A000C488FF1F1A82FF1F2182FF1F1E82FF1F07
:10A6B000474B1968480710B544D5464A1268002A26
:10A6C0003CD1454A1268520510D5444A107840F0F2
:10A6D000400010704248047844F04004047012783E
:10A6E000D40703D51A6822F004021A603A4B1B689B
:10A6F000180511D53B4B1A7842F040021A703A4ABD
:10A70000107840F0400010701B78DA0704D5304B09
:10A710001A6822F004021A602F4B1B68DB0411D563
:10A72000324B1A7842F040021A70314A107840F0E9
:10A73000400010701B78DC0704D5254B1A6822F006
:10A7400004021A602B4B1A7830BF214B1B68580744
:10A750000DD41F4B1960204B1A6812F4806F1A46F3
:10A7600021D01F4B197801F0BF0119701BE0224B5B
:10A770001B7813F0280FECD0204B214C27201870A9
:10A780004C20587023781E4813F0200FFAD003781D
:10A790005B06FCD5174B1A70194A137803F00C03AB
:10A7A0000C2BFAD1D5E713681C0504D50E4B1A788B
:10A7B00002F0BF021A70084B1B68D80404D50C4B7A
:10A7C0001A7802F0BF021A70BDE81040FEF738BCDC
:10A7D00010ED00E0688BFF1F3480044005A00640A8
:10A7E00000A0064005B0064000B0064005C0064087
:10A7F00000C006400040064000E00740044006401C
:10A800000640064008B56C20FCF7BEFE10F00900BB
:10A8100046D0244B1B789A0603D5234B1B785B0646
:10A8200035D4224B1B68580739D51F4B1A7812F0C4
:10A83000470F2ED01B4A1178890604D51B7803F0E8
:10A840000703022B27D013781A0705D5164B1B7860
:10A8500003F00703032B20D0124B1B789B071ED558
:10A86000114B1B7803F00703042B18D1104B1878F9
:10A8700000F00300022806D0032806D001280CBFF0
:10A880000720062008BD082008BD092008BD0320B8
:10A8900008BD022008BD042008BD052008BD012018
:10A8A00008BD00BF00E0074001E0074010ED00E0F8
:10A8B00002E0074020F0E003092B5AD8DFE803F05C
:10A8C00005080C101E252C343E486C20002152E057
:10A8D0002A4B00221A700CE0284B00221A7043E029
:10A8E000274B1A7842F020021A705A7842F0C002C0
:10A8F0005A70244B1A6822F0040239E0204B1A786F
:10A9000042F020021A7082222DE01D4B1A7842F08C
:10A9100008021A70032226E0194B1A7842F002024C
:10A920001A7020F01F001CE0154B1A7820F01F0051
:10A9300042F002021A7040F0010012E0104B1A7847
:10A9400020F01F0042F002021A7040F0020008E0FE
:10A950000B4B1A7820F01F0042F002021A7040F0F0
:10A960000300987004225A70064B1A6842F00402E1
:10A970001A606C200121FCF717BE00BF01E0074000
:10A9800000E0074010ED00E0014A024B1A60FEE7CC
:10A990000400FA050CED00E010B5124A1249134804
:10A9A000891A00238B4203D01C5CD4540133F9E78D
:10A9B0000F4B104A9342184605D10F4A0F49002306
:10A9C000891A184608E00E490023891A8B42F4D0F0
:10A9D000C45CD4540133F9E78B4202D0D054013324
:10A9E000FAE710BDF081FF1F2282FF1F60D5000033
:10A9F00010040000100400002482FF1FCC8BFF1FF6
:10AA00003CB4000008B5494B1A6842F480521A6001
:10AA1000474A484B1A60484B1A6822F060021A6095
:10AA2000043B4CF220511B6813F0400F434B4DF692
:10AA3000281219801A800BD04FF4C87223F8082C02
:10AA4000002223F80A2C40F2C11223F80E2C03E056
:10AA50003B4B4FF4E9721A803A4B08221A70A3F16B
:10AA60000113A3F5104324221A70A02203F8012C2D
:10AA7000354A137813F0020F334BFAD01A78D00608
:10AA8000FCD41A7802F00C02082AFAD12F4B2E4976
:10AA900027221A704C225A700B782B4A13F0200F81
:10AAA000FAD013785906FCD5294A2A4B1A602A4B4A
:10AAB00028221A70244A137803F00C030C2BFAD1C5
:10AAC000264B274A27491360274ADA60274A1A612A
:10AAD000274A5A61274A9A61274A1A63274A9A6085
:10AAE000274A9A63274ADA62274A3C3343F8041F0D
:10AAF0009342FBD1FFF750FF244B254800221A60F8
:10AB0000FF210422FCF7B0F9F5F73EFE214A224B63
:10AB1000224823491A60FCF769FB22482249062291
:10AB2000FCF702FCFCF7D0FCFCE700BF38800440D7
:10AB30000301600080C00440D4F00F400E200540A7
:10AB40000020054002D00740064006400440064071
:10AB50000000130144800440004006400080FF1FB5
:10AB600008ED00E0758D0000658D0000678D000028
:10AB7000698D00006B8D00006D8D00006F8D0000F1
:10AB8000718D0000738D0000AC81FF1F00800040BC
:10AB9000C088FF1FFC7F0020C88BFF1F4CD5000022
:10ABA000CC8BFF1FCCD400008CD3000000F580209C
:10ABB00049300003012342F4807231B10B421CBFC3
:10ABC0000260994304305B00F7E770472DE9F74FC7
:10ABD00002798346092A00F20B84DFE812F00A00AA
:10ABE000980209048C0109043703C003090409040D
:10ABF000BE008279530613D4170614D412F0080F3E
:10AC000002F0100506D0002D0CBF4FF410254FF4B4
:10AC100030250AE0002D14BF4FF42025002504E064
:10AC20004FF4002501E04FF44025960702D545F08A
:10AC3000030503E0540748BF45F00205DBF8088030
:10AC40009BF80790B14EDFF810A300270124B8F15C
:10AC5000000F00F0CD8314EA080F7BD0B9F1040F88
:10AC600000F2C683DFE809F0031831465B00DBF829
:10AC70000020A7497A5057209BF80510A54AFEF7F7
:10AC8000C3FE326842F40072326000202A46214638
:10AC9000FFF78CFFA04A13E0DBF800209F497A50B1
:10ACA00058209BF805109E4AFEF7AEFE326842F42B
:10ACB0008062326001202A462146FFF777FF994AD9
:10ACC000116821EA0401116042E0DBF80020964996
:10ACD0007A5059209BF80510944AFEF795FE326889
:10ACE00042F40062326002202A462146FFF75EFFEE
:10ACF0008F4AE5E7DBF800208E497A505A209BF80E
:10AD000005108D4AFEF780FE326842F480523260B0
:10AD100003202A462146FFF749FF884AD0E7DBF89F
:10AD20000020874BFA505B209BF80510854AFEF700
:10AD30006BFE326842F40052326004202A462146FB
:10AD4000FFF734FFDAF8002022EA0402CAF80020F4
:10AD500028EA04086400043779E7C1798468FF2988
:10AD600022D1794A117821EA04011170017AD17057
:10AD7000764901225CB1DBF80800024204D0DBF81E
:10AD8000000024EA0204086452000431F2E79BF850
:10AD900005106F4A1520FEF737FE6B4ADBF80810E6
:10ADA00013780B43137023E3827902F018000838FC
:10ADB000C0B2102896BF674D4FF0000815F800800C
:10ADC000900705D412F0040F0CBF0022022200E00D
:10ADD0000322042900F20C83DFE801F00319242F79
:10ADE0003A004A49086840F4007008600020214693
:10ADF000FFF7DCFE484A1168DFF86491534B21EA03
:10AE000004011160012600254FF0030C31E03F4999
:10AE1000086840F48060086001202146FFF7C6FE04
:10AE2000404AE8E73949086840F4006008600220B9
:10AE30002146FFF7BBFE3E4ADDE73449086840F48F
:10AE40008050086003202146FFF7B0FE3B4AD2E75E
:10AE50002E49086840F40050086004202146FFF79E
:10AE6000A5FE3D4AC7E7DBF80820164204D176006C
:10AE70000135002CF7D1BBE29BF8072005EB42120D
:10AE800019F80270FF2F33D0F90807F0030ABF0842
:10AE900007F1804707F5F827304A4FEA4A0A0A4483
:10AEA00039780CFA0AF021EA000139709BF8071092
:10AEB000DBF8000005EB411108FA0AFA19F8011055
:10AEC00043F82100012001F0070100FA01F1C9B2A5
:10AED000117015201E4A9BF805108DE80810FEF72A
:10AEE00093FD3A784AEA020A87F800A09DE8081024
:10AEF00024EA0604BBE741798A09012A00F086802A
:10AF000030D3022A00F0A38072E200BF38800440F0
:10AF1000548AFF1FC195000014F00F40C888FF1F1E
:10AF20006195000054F00F40E88AFF1F0195000072
:10AF300094F00F404C89FF1FA1940000D4F00F4003
:10AF4000CC89FF1F4194000004C007404C88FF1FBC
:10AF50001594000095D3000014F10F4005C0074080
:10AF600027D40000A54A106840F0807010609BF85C
:10AF7000052022F0C002072A00F23A82DFE802F040
:10AF8000040D163B2029323B9D4A106840F40070A6
:10AF900010604FF450709B4A10E0994A106840F4DA
:10AFA000007010604FF45070974A07E0944A1068A0
:10AFB00040F400601060954A4FF48860106023E010
:10AFC0008F4A106840F4007010604FF45070904A3F
:10AFD000F4E78B4A106840F4007010604FF4507032
:10AFE0008C4AEBE7864A106840F4007010604FF41A
:10AFF0005070894AE2E7824A106840F4007010609D
:10B000004FF45070C2F8E00F844A41E07B4A106868
:10B0100040F0007010609BF8052032F0C0020BD0A9
:10B02000012A40F0E581764A106840F40070106013
:10B030004FF450707A4A07E0714A106840F400708B
:10B040001060784A4FF450701060774A20E0774AD9
:10B05000106840F0807010609BF8052032F0C0024C
:10B060000CD0012A40F0C481654A106840F4007099
:10B0700010606F4A4FF45070106008E0604A10682A
:10B0800040F4007010604FF45070C2F8F00F694A3D
:10B09000C020C2F884009BF80A0000F018001828AD
:10B0A00001F03F010FD164484FF0807504688D4076
:10B0B00024EA05040460C46A44F40074C4625F486E
:10B0C00040F2034404609BF90A000131002802EBBE
:10B0D000C100B4BF2424282444600020D0649BF81D
:10B0E0000A00BBF8084010F0200FBBF8060003D0A0
:10B0F00064089460400801E0013C946002EBC101E7
:10B1000088609BF80A3003F03F03136070E1847B92
:10B110008268012C0FD002D3022C1DD068E1B0F957
:10B120000C10002935491CDB08683C4D40F080704C
:10B1300008603E201FE0B0F90C1000292F4904DA06
:10B140000B6823F000730B6052E10868364D40F045
:10B15000007008603F200EE0B0F90C100029334960
:10B1600003DA0B6823F08073EDE70868314D40F097
:10B17000807008604020002129602E6833064FF05F
:10B18000C00648BF2960C5F88460E9644FF6FF76C1
:10B190000021B24206D9072902D001315208F8E74E
:10B1A0004FF6FF72BBF80C70254EAA6089B2FF06FD
:10B1B00026F8141044BF41F4805126F81410DBF82F
:10B1C0000020204941F824205AB11F4B9BF805105C
:10B1D00053F82420FEF718FC36F8143043F04803E7
:10B1E00003E036F8143043F0080326F8143036F83C
:10B1F0001430C3F30B039BB22B60F9E03C80044096
:10B20000388004400C900440109004400CB004407E
:10B210001C900440009004400490044000800340CF
:10B22000249004402090044000900340308004406B
:10B230002C90044000800B400C8004404890044057
:10B24000B088FF1F3888FF1FA8D30000826815064A
:10B2500008D5827D002A40F0CB80674A116821F42E
:10B26000805111609BF81620002A40F0C180624A8C
:10B27000116841F480511160DBF8082012F00105DB
:10B280000AD012F0020F14BF40250025540703D442
:10B29000002D14BF6025202512F0080F18BFBBF841
:10B2A0001400564918BF088012F4407F4DD0002288
:10B2B00081F822209BF81740640104F1804404F5D2
:10B2C00010440221A180A28240F20112E280DBF848
:10B2D0000C202260DBF80020A160A2B1DBF808009E
:10B2E000C00548BF0621A1839BF81610444840F8CA
:10B2F00021209BF81700434A50549BF80510424AFE
:10B30000FEF782FB00E0A2833C4A22610022A26198
:10B31000DBF8102051425208E160E28391B23B4ACF
:10B32000E182116841F0020111609BF8172002F1DF
:10B33000804202F50432B02111709BF81710344A94
:10B3400001208840116801431160DBF808305B067A
:10B350002A4B48BF45F0800583F8215048E090F81B
:10B36000214090F82020240244EA1214120302F42F
:10B37000E04244F080041443244A116841F48001FF
:10B3800011600189234A1160418991600021116196
:10B39000C288570404D544F4004444F002040FE08A
:10B3A0001604026848BF44F002044AB11A49482012
:10B3B0000A609BF80510194AFEF726FB44F02004AA
:10B3C000BBF80620D50508D5BBF81C20144902B1EE
:10B3D000013A0A60134A01211160134A44F0010145
:10B3E00011609BF821300F2B04BF44F480341460AB
:10B3F00003B0BDE8F08F00BF2C80044000C00C40BB
:10B40000AC88FF1FF087FF1FF59200003C800440CE
:10B410000C80004004600340708BFF1FC592000049
:10B4200054610340506103400060034002440346FE
:0CB43000934202D003F8011BFAE77047BA
:10B43C00436F6E6E656374696F6E2074696D6564BD
:10B44C00206F75740D0A00A348313000436F6D6D89
:10B45C00616E64206C696E6520626C6F636B6564F1
:10B46C000D0A000051B5000001000000FFFF0300B1
:10B47C00058000005BB500000080FF1F000001008C
:10B48C000580000063B500007DB500007E0400005F
:10B49C00070000006FB5000053B40000040000006A
:10B4AC00000100000000000000000000000000008F
:10B4BC0000000000150078002000000017005D005F
:10B4CC000A0000000041444D494E00202075546193
:10B4DC00736B6572264B494E45544953000000006E
:10B4EC0000000000000000000000501403030000E6
:10B4FC00325F00000D0A0A48656C6C6F2C20776F68
:10B50C00726C642E2E2E204B494E455449530D0A15
:10B51C0000574F4B454E202D2000676F696E6720FA
:10B52C00746F204C535320616761696E0D0A007271
:10B53C006573746F72696E672057414954206D6F43
:10B54C0064650D0A00666C6173682E62696E007228
:10B55C00616D2E62696E0066617669636F6E2E692D
:10B56C00636F003947656E65726174652E62696E32
:10B57C000000000100010010100000010020006814
:10B58C00040000160000002800000010000000203D
:10B59C00000000010020000000000000100000006E
:10B5AC00000000000000000000000000000000216E
:10B5BC0065F25F2065F1EF2065F2EF2165F22F0057
:10B5CC00000000000000000000000000000000006F
:10B5DC00000000000000000000000000000000005F
:10B5EC00000000000000000000000000000000202F
:10B5FC0065F2CF2065F1FF2165F2FF2065F2FF2097
:10B60C0065F1AF2166F20F000000000000000000A1
:10B61C00000000000000000000000000000000001E
:10B62C00000000000000000000000000000000000E
:10B63C000000002165F24F2065F2EF2065F1FF203C
:10B64C0065F2CF2166F20F0CC1FF3F000000000035
:10B65C0000000000000000000000000000000000DE
:10B66C0000000000000000000000000000000000CE
:10B67C00000000000000002165F20F2065F22F0C85
:10B68C00C2FF4F0BC1FFEF0BC1FFFF0CC1FFEF0B54
:10B69C00C1FF2F00000000000000000000000000AF
:10B6AC00000000000000000000000000000000008E
:10B6BC00000000000000002065F15F2065F1DF163E
:10B6CC0093F85F0BC1FFCF0BC1FFFF0BC1FFFF0B4B
:10B6DC00C1FFFF0BC1FF9F00000000000000000035
:10B6EC00000000000000000000000000000000004E
:10B6FC000000002165F29F2065F1FF2065F1FF201D
:10B70C0065F1FF2165F2AF0FB2FC5F0BC1FFEF0BD0
:10B71C00C1FFCF11AAFB3F2165F29F2065F25F00AC
:10B72C00000000000000000000000000000000000D
:10B73C00000000000000002165F24F2165F2EF20AF
:10B74C0065F1FF2065F1FF2065F1CF0000000021BD
:10B75C0065F21F2065F2FF2065F1FF2065F1FF20E7
:10B76C0065F1CF2165F22F00000000000000000001
:10B77C00000000000000000000000000000000219C
:10B78C0065F29F2166F22F0CC2FF5F0BC1FFEF0B1E
:10B79C00C1FFEF1693F85F2165F2CF2065F1FF2012
:10B7AC0065F2FF2065F1FF2065F22F00000000001C
:10B7BC00000000000000000000000000000000007D
:10B7CC000000000BC1FF0F0BC1FFCF0BC1FFFF0B24
:10B7DC00C1FFFF0CC1FFFF0CC1FFAF1D72F36F2146
:10B7EC0065F29F2165F20F000000000000000000D0
:10B7FC00000000000000000000000000000000003D
:10B80C0000000000000000000000000CC1FF4F0C05
:10B81C00C1FFEF0BC1FFFF0BC1FFCF1693F81F2029
:10B82C0065F23F0000000000000000000000000076
:10B83C0000000000000000000000000000000000FC
:10B84C000000000000000000000000000000000CE0
:10B85C00C1FF0F0CC1FF2F2065F28F2165F2FF2075
:10B86C0065F1FF2165F2EF2065F12F00000000006B
:10B87C0000000000000000000000000000000000BC
:10B88C000000000000000000000000000000000BA1
:10B89C00C1FF5F0BC1FFEF1693F85F2065F1CF205E
:10B8AC0065F1FF2065F2FF2065F1FF2065F1CF0007
:10B8BC00000000000000000000000000000000007C
:10B8CC00000000000000002065F23F0CC2FF9F0B3F
:10B8DC00C1FFFF0BC1FFFF0BC1FFFF0BC1FFAF1D72
:10B8EC0074F45F2165F2EF2165F29F2165F20F0080
:10B8FC00000000000000000000000000000000201C
:10B90C0065F14F2165F2EF2065F2FF2065F1CF0F55
:10B91C00B1FC5F0BC1FFEF0BC1FFFF0BC1FFFF0BB6
:10B92C00C1FF9F00000000000000000000000000AC
:10B93C0000000000000000000000000000000020DB
:10B94C0065F12F2065F1EF2065F1FF2065F1FF20F7
:10B95C0065F1FF2165F29F0CC1FF9F0CC2FF2F0008
:10B96C0000000000000000000000000000000000CB
:10B97C0000000000000000000000000000000000BB
:10B98C00000000000000002165F25F2065F1FF213E
:10B99C0065F2CF2165F22F000000000000000000CE
:10B9AC000000000000000000000000000000000F7C
:10B9BC00FF000003FF000081FF0000C07F0000C0FB
:10B9CC003F0000800F0000C1030000F0010000F8F0
:10B9DC00030000FE070000FF010000FF000000FC58
:10B9EC00000000F0070000F00F0000FC3F0000001A
:10B9FC0033C6000036C600000012000046C6000028
:10BA0C004BC600000200000045787465726E616CD4
:10BA1C00000820080031000000312E3500320000F3
:10BA2C000000000033C6000036C600000012000003
:10BA3C001DCC000026CC0000050000003BCC000013
:10BA4C0044CC0000050100005CCC000065CC00007B
:10BA5C000502000079CC000081CC00000503000039
:10BA6C009CCC0000A5CC000005040000C5CC000057
:10BA7C00D4CC000005150000EFCC0000FDCC00007C
:10BA8C000516000088C900001ACD00000511000041
:10BA9C0016C9000000C900000000000046C60000E6
:10BAAC004BC6000002000000455A504F525400741F
:10BABC00616D7065720057444F470057616B657537
:10BACC0070207265736574003F3F3F0033C6000001
:10BADC0036C600000012000055C900005DC9000008
:10BAEC00010A000071C9000078C9000001010000C2
:10BAFC0016C9000000C900000000000046C6000086
:10BB0C004BC60000020000004A54414700706572A9
:10BB1C006970686572616C206661696C757265002C
:10BB2C00556E646572766F6C746167650000000019
:10BB3C0033C6000036C600000012000046C60000E6
:10BB4C004BC600000200000033C6000036C60000E1
:10BB5C000012000046C600004BC6000002000000A8
:10BB6C004C6F636B75700000CDC2000034CD0000CB
:10BB7C00000400007EC100004CCD00000005000058
:10BB8C00E1C2000067CD00000006000076CD000089
:10BB9C0078CD00000007000092CD000094CD00008D
:10BBAC00000900007BC10000B3CD0000000A0000BA
:10BBBC0055C40000C2CD0000000E000057C40000A8
:10BBCC00D1CD0000000F0000ECCD0000EECD000048
:10BBDC000010000009CE000026C600000011000075
:10BBEC0016C9000000C900000000000046C6000095
:10BBFC004BC600000200000033C6000036C6000031
:10BC0C000012000088C9000094C900000602000060
:10BC1C00A7C90000B1C90000060A0000BEC9000097
:10BC2C00C7C9000006090000D9C90000E2C900001C
:10BC3C0006080000F6C90000FEC90000011F000044
:10BC4C001ECA000025CA00000120000041CA0000E5
:10BC5C0047CA00000100000054CA00005DCA000081
:10BC6C00011A000016C9000000C900000000000005
:10BC7C0046C600004BC6000002000000436C6F6318
:10BC8C006B206C6F737300506F7765722D6F6E0045
:10BC9C0057616B657570000033C6000036C6000036
:10BCAC00001200001BC9000026C90000051C000082
:10BCBC0036C9000042C90000051D000016C900006D
:10BCCC0000C900000000000046C600004BC6000082
:10BCDC000200000074BB00000F0C00007FC50000C8
:10BCEC00B8BD0000140200008EC5000030BA000080
:10BCFC00160B0000A1C50000F8BD00000F0F0000DE
:10BD0C00B3C5000004BC0000110B0000C6C5000048
:10BD1C00D8BA000011050000D5C50000A4BC000075
:10BD2C000D050000E4C500003CBB00000D02000046
:10BD3C00F1C500000CCE00000D180000FEC500007F
:10BD4C0054BB00000F0200000FC60000FCB900003D
:10BD5C000F02000023C60000333030000000003614
:10BD6C00303000000000313230300000003234300E
:10BD7C0030000000343830300000003936303000EC
:10BD8C0000003134343030000031393230300000B2
:10BD9C003338343030000035373630300000313134
:10BDAC0035323030003233303430300033C600009E
:10BDBC0036C600000012000046C600004BC600004C
:10BDCC00020000004F444400004556454E004E4FC3
:10BDDC004E4500486F7374206465627567676572C1
:10BDEC0000536F66747761726500000033C6000003
:10BDFC0036C600000012000069CA00006CCA0000C0
:10BE0C00010F000099CA00009CCA0000011000003C
:10BE1C00C8CA0000CBCA000001110000FBCA000018
:10BE2C00FECA0000011B000016CB000019CB00005D
:10BE3C00011C000030CB000033CB0000011D0000C2
:10BE4C0085C9000048CB0000011E00006ACB000031
:10BE5C0072CB00000102000090CB000098CB0000D8
:10BE6C00010B0000B2CB0000BCCB000001040000B1
:10BE7C00D3CB0000DECB000001050000FBCB0000A3
:10BE8C0000CC0000010C000016C9000000C9000025
:10BE9C000000000046C600004BC600000200000077
:10BEAC004E4F4E450000000052545300000000005D
:10BEBC00584F4E0000000000536F66747761726536
:10BECC002076657273696F6E20000A0A0D000A0DE8
:10BEDC003D3D3D3D3D3D3D3D3D3D3D3D3D3D3D3D86
:10BEEC003D3D3D0A0D00206B427974657300206264
:10BEFC0079746573004E6F204469736B20726561B1
:10BF0C0064790D0A00496E76616C6964206469720B
:10BF1C006563746F72790D0A004469726563746F9E
:10BF2C00727920000D0A0A005B445D00207B636F70
:10BF3C00756C64206E6F7420626520756E64656C20
:10BF4C006574656421217D00207B756E64656C656C
:10BF5C007465647D002066696C657320776974680C
:10BF6C0020002062797465730D0A00206469726583
:10BF7C0063746F726965732C200020667265650DA1
:10BF8C000A0046696C652F6469726563746F727917
:10BF9C00206E6F7420666F756E640D0A007772697F
:10BFAC007465206661696C6564004E65772066690E
:10BFBC006C65206C656E677468203D20000D0A521C
:10BFCC00454144204552524F52206F636375727243
:10BFDC0065640046696C65206E6F7420666F756EC3
:10BFEC00640D0A0052656164696E67207365637441
:10BFFC006F722000204641494C454421210D0A0016
:10C00C0057726974696E6720736563746F722873F5
:10C01C0029200020536563746F72207772697465F0
:10C02C00206572726F72210A0D00202D204F4B0A71
:10C03C000D00466F726D617474696E6720464154D1
:10C04C00003132200031362000333220006E6F7404
:10C05C0020706F737369626C650D0A00696E2070D5
:10C06C00726F6772657373202D20706C65617365D8
:10C07C0020776169742E2E2E0D0A004D616B6520A0
:10C08C00646972206661696C65640D0A00437265AF
:10C09C006174652066696C65206661696C65640D08
:10C0AC000A004E6577206E616D65206D697373694A
:10C0BC006E670D0A004E6F7420666F756E640D0A04
:10C0CC000052656E616D65206661696C65640D0A70
:10C0DC0000446972204E4F5420656D7074790D0ABE
:10C0EC000044656C657465206661696C65640D0A55
:10C0FC000046696C65207375636365737366756C54
:10C10C006C79207472756E63617465640020636C65
:10C11C00757374657273206672656564005472750C
:10C12C006E636174696F6E206661696C65640D0A7B
:10C13C0000496E76616C696420706174680D0A0048
:10C14C000D0A53442D6361726420006E6F74206479
:10C15C00657465637465640D0A006E6F7420666F98
:10C16C00726D617474656400205344484300313629
:10C17C00003132003332002077726974652D707291
:10C18C006F746563746564004279746573207065BF
:10C19C007220736563746F723A00436C75737465C7
:10C1AC00722073697A653A004469726563746F72C0
:10C1BC007920626173653A00464154207374617250
:10C1CC00743A004641542073697A653A004E756D95
:10C1DC00626572206F6620464154733A004C4241AE
:10C1EC003A00546F74616C20636C75737465727370
:10C1FC003A00496E666F20736563743A0046726547
:10C20C006520636C7573746572733A004E6578744F
:10C21C0020667265653A004E65772064617465200E
:10C22C007365740D0A000A0D415250207265736FCC
:10C23C006C7665640A0D000A0D41525020726573CC
:10C24C006F6C7574696F6E206661696C65640A0D3C
:10C25C00000A0D53657269616C206E756D626572B2
:10C26C003A2000446576696365206964656E74697B
:10C27C006669636174696F6E3A200030203D20520C
:10C28C00554E0031203D20574149540032203D206D
:10C29C0053544F500033203D20564C505200342004
:10C2AC003D20564C50530035203D204C4C5300360D
:10C2BC00203D20564C4C53300037203D20564C4CE2
:10C2CC0053310038203D20564C4C53320039203D20
:10C2DC0020564C4C533300205B6163746976655D6A
:10C2EC00004C61737420726573657420636175739F
:10C2FC0065203D20000A0D53797374656D206D65C2
:10C30C006D6F7279207573653A0A0D00467265651A
:10C31C002068656170203D20000A0D556E757365AF
:10C32C006420737461636B203D20000D0A546865B2
:10C33C002064657669636520686173206265656E4B
:10C34C00206F7065726174696E6720666F72200071
:10C35C0042616420706F7274206E756D6265720D2F
:10C36C000A000D0A506F72742064697265637469F7
:10C37C006F6E3A20004F55545055540D0A00494EDB
:10C38C005055540D0A00496E76616C696420706FCB
:10C39C0072740D0A00506F727420697320696E708C
:10C3AC0075740D0A00506F72742073746174653A61
:10C3BC002000310D0A00300D0A000D0A3F3F0D0A16
:10C3CC0023004D656D6F727920446973706C6179CF
:10C3DC000D0A0046696C6C0D0A0057726974650D84
:10C3EC000A004572617365640D0A004572617365DC
:10C3FC00206661696C6564210D0A000A0D4279653D
:10C40C00204279650A0D00496E636F727265637420
:10C41C002064617461206C656E6774680D0A000D90
:10C42C000A53657269616C20636F6E666967757219
:10C43C006174696F6E0D0A0042617564203D2000C5
:10C44C00696E76616C69642100370038002042699E
:10C45C0074730D0A002073746F70206269742873F2
:10C46C00290D0A00466C6F7720636F6E74726F6CC7
:10C47C002000486967682077617465722000250D7B
:10C48C000A004C6F77207761746572200055534217
:10C49C00204572726F7220436F756E746572730DE6
:10C4AC000A002D204352432D3136206572726F7273
:10C4BC00733A002D204352432D35206572726F72F2
:10C4CC0073203A00555342204572726F7220436FAD
:10C4DC00756E746572732072657365740D0A004E07
:10C4EC0065772074696D65207365740D0A00656E3F
:10C4FC0061626C650064697361626C65000D0A4968
:10C50C006E76616C6964207377697463680D0A00D8
:10C51C00496E636F72726563742073657269616CC6
:10C52C002073706565640D0A00496E636F727265E5
:10C53C006374207061726974790D0A00496E636FBF
:10C54C0072726563742073746F7020626974730DFA
:10C55C000A00496E636F727265637420666C6F7744
:10C56C0020636F6E74726F6C0D0A000A0D0D004D16
:10C57C0041430020202020204D61696E206D656EA6
:10C58C007500204C414E20636F6E66696775726151
:10C59C0074696F6E0020202053657269616C206392
:10C5AC006F6E6669672E0020496E7075742F4F751B
:10C5BC0074707574206D656E750020202041646D5B
:10C5CC00696E2E206D656E75002020205374617489
:10C5DC00732E206D656E750020202020555342204F
:10C5EC006D656E750020202020493243206D656EEC
:10C5FC00750020204469736B20696E7465726661E6
:10C60C006365004654502F54454C4E455420636F7F
:10C61C006D6D616E64730020202043414E20636F6A
:10C62C006D6D616E647300757000676F20746F20A0
:10C63C006D61696E206D656E750071756974004C65
:10C64C006561766520636F6D6D616E64206D6F64DE
:10C65C00650075744641542F6361726420696E667F
:10C66C006F005B706174685D2073686F772064691C
:10C67C00726563746F727920636F6E74656E74008B
:10C68C0064697264005B706174685D2073686F77B5
:10C69C002064656C65746564206469726563746F8D
:10C6AC00727920636F6E74656E74006469726800D1
:10C6BC005B706174685D2073686F7720686964646F
:10C6CC00656E20636F6E74656E7400696E666F665E
:10C6DC00005B706174685D2073686F772066696CAD
:10C6EC006520696E666F00696E666F64005B7061D1
:10C6FC0074685D2073686F772064656C657465641D
:10C70C0020696E666F006364005B706174685D2005
:10C71C006368616E6765206469722E20282E2E2056
:10C72C00666F7220757029005B706174685D206E95
:10C73C00657720656D7074792066696C6500777219
:10C74C00697465005B706174685D20746573742036
:10C75C00777269746520746F2066696C65006D6B07
:10C76C00646972006E657720656D707479206469F8
:10C77C0072005B66726F6D5D205B746F5D2072651D
:10C78C006E616D65007472756E63007472756E63A4
:10C79C0061746520746F205B6C656E6774685D20D6
:10C7AC005B706174685D007072696E74005B7061BF
:10C7BC0074685D207072696E742066696C652063A4
:10C7CC006F6E74656E74005B706174685D20646577
:10C7DC006C6574652066696C65206F722064697283
:10C7EC002E00756E64656C00756E64656C657465A1
:10C7FC00205B6E616D655D005B2D31362F31325DD6
:10C80C00205B6C6162656C5D20666F726D6174207B
:10C81C0028756E666F726D61747465642920646925
:10C82C00736B005B2D31362F31325D205B6C616296
:10C83C00656C5D2066756C6C20666F726D61742022
:10C84C0028756E666F726D617474656429206469F5
:10C85C00736B0072652D666F726D6174005B2D31A8
:10C86C00362F31325D205B6C6162656C5D207265C8
:10C87C00666F726D6174206469736B2121212121B3
:10C88C000072652D66666F726D6174005B2D3136BA
:10C89C002F31325D205B6C6162656C5D2066756C5E
:10C8AC006C207265666F726D6174206469736B21A4
:10C8BC00212121210073656374005B686578206E0B
:10C8CC00756D6265725D20646973706C617920733B
:10C8DC006563746F72007365637477005B68657869
:10C8EC00206E6F2E5D205B706174742E5D205B6317
:10C8FC006E745D00446973706C6179206D656E7542
:10C90C002073706563696669632068656C70007577
:10C91C0073625F6572726F72730053686F77205524
:10C92C005342206572726F7273007573625F636E2F
:10C93C00745F727374005265736574205553422092
:10C94C00636F756E746572730075705F74696D6575
:10C95C000053686F77206F7065726174696E672021
:10C96C0074696D65006D656D6F72790053686F77D2
:10C97C00206D656D6F7279207573650073686F77C4
:10C98C005F636F6E6669670053686F7720636F6EC5
:10C99C0066696775726174696F6E0073686F775F33
:10C9AC0074696D6500646973706C61792074696D6C
:10C9BC0065007365745F74696D65005365742074EC
:10C9CC00696D652030313A32323A35360073657410
:10C9DC005F64617465005365742044617465203232
:10C9EC00333A30323A323031300073686F775F6CE3
:10C9FC00700053686F77206C6F7720706F7765725B
:10CA0C00206D6F646520616E64206F7074696F6E49
:10CA1C0073007365745F6C70005B6F7074696F6E1C
:10CA2C005D20536574206C6F7720706F7765722072
:10CA3C006D6F64650072657365740052657365741F
:10CA4C0020646576696365006C6173745F727374DE
:10CA5C00005265736574206361757365006D6400C5
:10CA6C004D656D6F727920446973706C6179205BD0
:10CA7C00616464726573735D205B3C6C3E7C3C77D7
:10CA8C003E7C3C623E5D205B6E756D5D006D6D00A5
:10CA9C004D656D6F7279204D6F64696679205B61AD
:10CAAC006464726573735D205B3C6C3E7C3C773ECA
:10CABC007C3C623E5D205B76616C5D006D66004D7A
:10CACC00656D6F72792046696C6C205B6164647271
:10CADC006573735D205B3C6C3E7C3C773E7C3C62BA
:10CAEC003E5D205B76616C5D205B6E756D5D0073E9
:10CAFC00640053746F7261676520446973706C6174
:10CB0C0079207B6173206D647D00736D0053746FAD
:10CB1C0072616765204D6F64696679207B61732053
:10CB2C006D6D7D0073660053746F7261676520468E
:10CB3C00696C6C207B6173206D667D0053746F7221
:10CB4C00616765204572617365205B616464726521
:10CB5C0073735D205B6C656E2D6865785D00736525
:10CB6C00745F6464720053657420706F7274207407
:10CB7C00797065205B312E2E345D205B3C693E7CE8
:10CB8C003C6F3E006765745F646472004765742097
:10CB9C006461746120646972656374696F6E205B93
:10CBAC00312E2E345D00726561645F706F7274009B
:10CBBC005265616420706F727420696E7075742098
:10CBCC005B312E2E345D0077726974655F706F7205
:10CBDC00740053657420706F7274206F7574707567
:10CBEC0074205B312E2E345D205B302F315D007351
:10CBFC00617665005361766520706F727420736581
:10CC0C007474696E672061732064656661756C74F9
:10CC1C00007365745F62617564005365742073659D
:10CC2C007269616C20626175642072617465007355
:10CC3C0065745F73746F70005365742073746F70D8
:10CC4C0020626974732028312F312E352F32290040
:10CC5C007365745F626974730053657420646174E6
:10CC6C006120626974732028372F3829007365742A
:10CC7C005F70617200536574207061726974792001
:10CC8C00284556454E2F4F44442F4E4F4E452900B4
:10CC9C007365745F666C6F770053657420666C6F98
:10CCAC007720636F6E74726F6C2028584F4E2F5222
:10CCBC0054532F4E4F4E4529007365745F68696756
:10CCCC00685F77617465720053657420666C6F776A
:10CCDC00207374616C6C20282529205B312E2E3931
:10CCEC00395D007365745F6C6F775F776174657223
:10CCFC000053657420666C6F772072657374617273
:10CD0C007420282529205B312E2E39395D0053687B
:10CD1C006F772073657269616C20636F6E666967EB
:10CD2C0075726174696F6E00436F6E6669677572B8
:10CD3C0065204C414E20696E7465726661636500B6
:10CD4C00436F6E6669677572652073657269616C95
:10CD5C0020696E7465726661636500476F20746F3D
:10CD6C0020492F4F206D656E75003400476F20747D
:10CD7C006F2061646D696E697374726174696F6E32
:10CD8C00206D656E75003500476F20746F206F76CF
:10CD9C006572766965772F737461746973746963EE
:10CDAC0073206D656E7500476F20746F205553426C
:10CDBC00206D656E7500476F20746F2049324320DB
:10CDCC006D656E7500476F20746F20757446415405
:10CDDC00206469736B20696E7465726661636500AB
:10CDEC0039004654502F54454C4E455420636C69C1
:10CDFC00656E7420636F6D6D616E6473006100000D
:10CE0C0033C6000036C60000001200000DC700003B
:10CE1C005EC600000B0B00007AC700006EC6000057
:10CE2C000B0000008CC6000091C600000B17000020
:10CE3C00B7C60000BCC600000B200000D7C600001F
:10CE4C00DDC600000B190000F3C60000F9C6000097
:10CE5C000B1C000012C7000015C700000B010000DE
:10CE6C0065C7000034C700000B0200004AC7000071
:10CE7C0050C700000B0400006AC7000070C7000018
:10CE8C000B0300008AC700007EC700000B0C0000DB
:10CE9C0091C7000097C700000B160000B3C7000035
:10CEAC00B9C700000B050000F0C70000D3C7000095
:10CEBC000B070000EEC70000F4C700000B1B0000BE
:10CECC0062C8000004C800000B09000090C80000F4
:10CEDC002FC800000B1100005FC8000069C80000DB
:10CEEC000B0A00008DC8000098C800000B1200004F
:10CEFC00C1C80000C6C800000B080000E2C8000052
:10CF0C00E8C800000B15000016C9000000C900009D
:10CF1C000000000046C600004BC6000002000000E6
:10CF2C0056312E342E303038000902200001010415
:10CF3C00C000090400000208065005070501024064
:10CF4C0000000705820240000055534243000000D8
:10CF5C002AD000002ED000008ACF0000E7CF0000BE
:10CF6C000CD0000022D000000300000012010002CF
:10CF7C00000000082504FC0300010102030110035A
:10CF8C004D0079002000500072006F006400555372
:10CF9C00422052657365740A0D0055534220537537
:10CFAC007370656E6465640A0D00555342205265BA
:10CFBC0073756D650A0D00456E756D6572617465EE
:10CFCC0064202800290A0D000080000000000000E9
:10CFDC000A000000000000000000000000800001BA
:10CFEC001F000000755461736B65722055534274B9
:10CFFC006F53442D4361726420202020312E303039
:10D00C000A0343006F006E00660000000008000178
:10D01C00F80003000200080349006E0074000403CA
:10D02C0009040A034D0061006E007500F8FFFF0053
:10D03C004E6F6E2D666F726D61747465642000693D
:10D04C006E7465726E616C20666C6173680D0A009B
:10D05C0046696C653A20004469726563746F727935
:10D06C003A20002069732053464E0D0A0020697344
:10D07C00204C464E20000D0A5374617274696E6721
:10D08C0020617420656E74727920002028636C75A1
:10D09C0073746572200044656C65746564204C463D
:10D0AC004E0D0A00456E640D0A00466972737420B9
:10D0BC006F626A6563742066726F6D2000466972D8
:10D0CC007374206F626A656374206572726F720D7F
:10D0DC000A004C464E206F626A656374206572725A
:10D0EC006F720D0A0044617461203D00496E7661D7
:10D0FC006C6964204C464E2061747472696275745C
:10D10C00652121004C464E20636F6E74656E742051
:10D11C007A65726F206572726F72202D2000206EFE
:10D12C006F74207A65726F21210D0A0053464E20D0
:10D13C00616C696173204353206D69732D6D61744B
:10D14C00636821210D0A0053464E2046696C652008
:10D15C006C6F636174656420617420656E747279A0
:10D16C0020000D0A53464E206E616D65202800721A
:10D17C006561642D6F6E6C790068696464656E001E
:10D18C0073797374656D00766F6C756D65204944A9
:10D19C00006469726563746F7279006172636869A7
:10D1AC007665003F3F3F0029203D200020416C69FF
:10D1BC006173204353203D20000D0A46696C6520A5
:10D1CC006C656E677468203D200020737461727406
:10D1DC00696E6720696E20736563746F7220002915
:10D1EC002046415420736563746F722000206F6673
:10D1FC006673657420004D616C666F726D6564209A
:10D20C002D20004469736B2044206D6F756E74651E
:10D21C006400443A5C004D53444F53352E30004665
:10D22C0041543136202020004641543332202020F6
:10D23C00004E4F204E414D4520202020002A005802
:10D24C00004469736B20666F726D61747465642041
:10D25C004641543100320D0A00360D0A0044697300
:10D26C006B20666F726D61747465640D0A00554EA7
:10D27C0044454C45544554585400203120353032E7
:10D28C002035303220004A616E00466562004D61E7
:10D29C007200417072004D6179004A756E004A75DA
:10D2AC006C0041756700536570004F6374004E6FDE
:10D2BC00760044656300203C4449523E20202020E7
:10D2CC002020202020202000F8FFFFFFF8FFFF0F78
:10D2DC00FFFFFFFFFFFFFF0F000100000000000039
:10D2EC00000101000000021010101010101010109E
:10D2FC0010010101010100000404040404040404ED
:10D30C0004040404040404040404040404040404D1
:10D31C000404200220000000080808080808080877
:10D32C000808080808080808080808080808080871
:10D33C000808002000000A0600020000004001005E
:10D34C0001000000983A4C1DA60E5307A903D40106
:10D35C003801EA0075004E002700130000000000A1
:10D36C001018100C060402114C1DA60E5307A9032D
:10D37C00D401EA009C0075003A0027001300090054
:10D38C00015775616D4D6C0000010000000000003C
:10D39C00000200000000000000030000A993000040
:10D3AC009D930000919300001F1C1F1E1F1E1F1F2A
:10D3BC001E1F1E1F48544D004A5047004749460047
:10D3CC00435353004A530042494E00424D500049CA
:10D3DC00434F0057646F6700617070004D61737349
:10D3EC005374006D61696E74656E6163650075736D
:10D3FC0062006C6F77506F7765720007070700004B
:10D40C00A18D00008D8D0000798D000007070700AD
:10D41C00000010180C080613021118FFFFFFFF0381
:10D42C00FFFFFFFFFFFFFFFF04FFFFFFFFFFFFFFFB
:10D43C00FFFFFFFFFFFFFFFFFFFFFF05FFFFFFFFEA
:10D44C00FFFFFFFFFFFFFFFFFFFFFFFFFFFFFFFFE0
:10D45C00FFFFFFFFFFFFFFFFFFFFFFFF06FF0708B8
:10D46C00090AFFFFFFFF0BFFFFFFFFFFFFFFFFFF9F
:10D47C00FFFFFFFFFFFFFFFFFFFFFF0CFF0DFF0E86
:10D48C00FF0FFFFFFFFFFFFFFFFFFFFFFFFFFFFF90
:10D49C00FFFFFFFFFFFFFFFFFFFFFFFF0001FF028A
:10D4AC00FFFFFFFFFFFFFFFFFFFFFFFFFFFFFFFF80
:10D4BC00FFFFFFFFFFFFFFFFFFFFFF03040500005F
:10D4CC00DFD30000058B0000000000000400010009
:10D4DC00E4D30000990500004500020000000000A4
:10D4EC00E8D30000C94C00004500FFFF000000001D
:10D4FC00EFD30000E11100002500FFFF0000000049
:10D50C00FAD30000112B00002500FFFF00000000E3
:10D51C00FED30000098B0000000000000000010099
:10D52C0000000000000000000000000000000000EF
:10D53C00090A0B002D8E0000F18D0000B58D000046
:10D54C00010000500000000000A0064000B00640A2
:04D55C0000C00640C5
:10D56000FF00000001000000550000000100000065
:10D5700055534253000000000000000000FF8021CE
:10D58000017001780906FCD5704701010400B2075B
:02D59000FF0199
:0400000300000410E5
:00000001FF
